:020000040801F1
:10C00000D08C0020B9C20108897202088B72020824
:10C010009D7202089F720208A172020800000000CF
:10C02000000000000000000000000000CBC201087A
:10C03000A372020800000000CFC2010851460208A6
:10C04000D3C20108F34E0208D3C201080F3F020811
:10C05000D3C20108D3C20108C13C0208E13C020876
:10C06000033D0208233D0208453D0208BB36020895
:10C07000FD3602083F3702088B370208A138020854
:10C08000F138020841390208D3C20108D3C20108BD
:10C09000D3C20108D3C20108D3C20108653D02081A
:10C0A000D3C20108D3C20108D3C20108D3C2010818
:10C0B000594802087B4802089D480208D3C201087B
:10C0C000D3C20108D3C20108D3C20108D3C20108F8
:10C0D000D3C201087B310208EB3102085B3202084F
:10C0E000A73D0208473F0208D3C20108D3C2010896
:10C0F000D3C20108D3C20108D3C20108D3C20108C8
:10C10000D3C20108D3C20108BF480208D3C2010844
:10C11000CB3202083F330208E14802080349020813
:10C1200091390208DF3902082F3A02087B3A0208E7
:10C1300000F002F800F0B0F80AA090E8000C824489
:10C140008344AAF10107DA4501D100F0A5F8AFF266
:10C15000090EBAE80F0013F0010F18BFFB1A43F0E5
:10C1600001031847580D0100780D01000A444FF0F3
:10C17000000C10F8013B13F0070408BF10F8014B46
:10C180001D1108BF10F8015B641E05D010F8016B8B
:10C19000641E01F8016BF9D113F0080F1EBF10F8EF
:10C1A000014BAD1C0C1B09D16D1E58BF01F801CB12
:10C1B000FAD505E014F8016B01F8016B6D1EF9D595
:10C1C0009142D6D3704700000023002400250026AA
:10C1D000103A28BF78C1FBD8520728BF30C148BFEA
:10C1E0000B6070476E290BF0118470290BF0F784F7
:10C1F00066290FF0DC8065290FF0D98067290FF0E0
:10C20000D68061290FF0D58003681B0A28BF41F052
:10C21000800169290BF0BE8364290BF0BB8375296B
:10C220000BF0B8836F290BF0848478290BF0C3845A
:10C23000E9290CF07982E4290CF07682F5290CF0DA
:10C240007382EF290BF08184F8290BF0C284036814
:10C25000DB0928BF41F0800163290CF0308273298B
:10C260000CF03582E3290CF05382F3290CF058824C
:10C27000002070471FB50CF0F1FA040000200021E7
:10C280000EF0C0F9401C6060002000210EF0D0F9D3
:10C29000E0601FBD10B510BD0CF0AEFD1146FFF7FC
:10C2A000E9FF00F0E0FB0CF0DAFD03B4FFF7F2FF6A
:10C2B00003BC06F032FD00000948804709480047EA
:10C2C000FEE7FEE7FEE7FEE7FEE7FEE7FEE7FEE746
:10C2D000FEE7FEE704480549054A064B70470000A3
:10C2E000AF73020831C10108D05C0020D08C00205F
:10C2F000D06C0020D06C002038B508F051FB4FF412
:10C30000007006F003F90446002000906A462146BA
:10C31000FB4806F065FAB0B920460BF0B3FD217872
:10C3200028290CD194F82510262908D1221812F8B2
:10C33000051C242903D112F8031C292907D0214602
:10C34000F0A006F021F9204606F01AF938BD62780F
:10C35000412A15D0632A08D02146F2A006F014F92C
:10C36000F8A1522002F02BFBEDE782B22146FC48F7
:10C3700006F0E7F90028E6D0FAA006F05FF9E2E758
:10C380002146FDA006F000F9DDE738B508F008FB0E
:10C390004FF4007006F0BAF80446002000906A4698
:10C3A0002146EF4806F01CFA20B9BDF800102046DF
:10C3B00001F067FC204606F0E3F838BD10B508F040
:10C3C000EFFABDE8104001F03DBD38B508F0E8FADD
:10C3D000F14C2078400729D54FF4806006F096F89C
:10C3E0000546002000906A462946EC4806F0F8F918
:10C3F000C8B9BDF800202946E94805F096FC032895
:10C4000011D0BDF800202946E54805F08EFC032830
:10C4100009D0207820F004002070E2A006F00EF988
:10C42000E0A004F010FD284606F0AAF838BD7CB55F
:10C4300008F0B6FA4FF4806006F068F8064600206F
:10C44000019001AA3146DC4806F0CAF9002851D112
:10C45000DAA1304606F002FB0546002D46DB4FF41C
:10C46000007006F053F804464FF480700090711984
:10C4700000230A22204606F022FA20460BF002FD95
:10C48000217828290CD194F82510262908D12118C3
:10C4900011F8052C242A03D111F8031C292907D0EF
:10C4A0002146CAA006F070F8204606F069F821E09F
:10C4B0006178412915D0432908D02146CAA006F049
:10C4C00063F8D1A1522002F07AFAEDE782B2214658
:10C4D000A34806F036F90028E6D0A2A006F0AEF890
:10C4E000E2E72146CFA006F04FF8DDE73146D5A0C0
:10C4F00006F0A4F8304606F043F87CBD70B508F0AD
:10C500004FFAA548007840072DD5D548044605F0D8
:10C510006CF9D348401F054604F04EFE2B462246D8
:10C52000D0A1482002F04BFA102005F0EFFF06469C
:10C530002B46D3A2102130460BF0AEF9304602F064
:10C54000F2F8102130460BF092FD2346CEA21021C6
:10C5500030460BF0A1F9304602F0C8F83046BDE88D
:10C56000704006F00DB870BD38B508F019FA4FF4F8
:10C57000807005F0CBFF0446002000906A462146FB
:10C58000C34806F02DF990B9BDF80010204605F01B
:10C5900048FC814A78B1022823D0032828D00428F7
:10C5A00014D0BCA006F04AF8BAA004F04CFC204617
:10C5B00005F0E6FF38BD107820F004001070BAA036
:10C5C00006F03CF8B8A004F03EFCF0E7107820F04C
:10C5D00001001070B9A006F031F8B8A004F033FCE7
:10C5E000E5E7BAA006F02AF8B8A004F02CFCDEE7D4
:10C5F000BBA006F023F8BAA004F025FCD7E703F0AF
:10C60000A9BE38B508F0CCF94FF4806005F07EFF84
:10C610000446002000906A462146B54806F0E0F83E
:10C6200018B92146B3A005F0AFFF204605F0A8FFDA
:10C6300038BD38B508F0B4F94FF4806005F066FFF6
:10C640000446002000906A462146AF4806F0C8F82C
:10C6500018B92146ADA005F097FF204605F090FFE0
:10C6600038BD2DE9F04108F09BF94B4EAC4C4FF032
:10C6700000053078C10708D0810706D5410704D5E9
:10C68000000702D52570BDE8F0812078401CC0B2BB
:10C690002070022804D9A3A004F0D5FB0AF028FEDC
:10C6A0003078C0070CD1A5A001F0FCFF04F023FEF8
:10C6B000032822D0A3A004F0C6FBA6A005F064FFC7
:10C6C0003078C1071AD0800718D4A5A001F0EAFF7E
:10C6D0001E2005F01BFF07461E21384605F09DF879
:10C6E00003280CD0384604F0AEFB307820F001006F
:10C6F000307004F021FE384636E180E139E186E110
:10C70000B00F0020555342CAD5B5BDCFC2D0D027F7
:10C71000B7C727B7A8CAFDBEDDD6A13A2573202E1C
:10C7200000000000555342CAD5B5BDCFC2D0D0CE0F
:10C73000B4D6AAC0E0D0CDCAFDBEDDD6A13A2573DD
:10C74000202E0000555342CAD5B5BDCFC2D0D0CEA1
:10C75000B4D6AAC0E0D0CDCAFDBEDDD6A10000008F
:10C76000AC0600207355736572636D645175657511
:10C7700065D2E7B3F6A3A100555342C9CFCEBBBBE8
:10C78000FAC8B7C8CFCAD5B5BDCAFDBEDDD6A13A75
:10C790002573202E0000000031000020AA0B00208D
:10C7A0009A0100205463702053656E644461746183
:10C7B0002045727221000000901E00202B51495527
:10C7C00052433A202272656376220000544350CAD5
:10C7D000D5B5BDCFC2D0D027B7C727B7A8CAFDBE31
:10C7E000DDD6A13A25732000544350CAD5B5BDCF3C
:10C7F000C2D0D0CEB4D6AAC0E0D0CDCAFDBEDDD660
:10C80000A13A257320000000544350CAD5B5BDCFCE
:10C81000C2D0D0CEB4D6AAC0E0D0CDCAFDBEDDD63F
:10C82000A100000054637020736572766572C8B70A
:10C83000C8CFCAD5B5BDCAFDBEDDD6A13A25732085
:10C840000000000054435020CFC2D0D0CAFDBEDD4E
:10C85000BDE2CEF6CAA7B0DC3A2573200000000086
:10C86000F21B00204353513A25732C2045433230AC
:10C8700020566F6C746167653A25736D5600000031
:10C8800025736D56000000004353512573000000CE
:10C890009622002054637020756E6B6E6F776E2049
:10C8A000757263202E0000005463702073657276E9
:10C8B000657220636C6F736564202E005463702072
:10C8C000504450206465616374202E0054637020CE
:10C8D000696E636F6D696E672066756C6C202E00E3
:10C8E00054637020696E636F6D696E67202E00005F
:10C8F000BC1700205273343835207265636461744C
:10C90000613A2573202E0000B61300205273323393
:10C910003220726563646174613A2573202E0000D1
:10C9200000000020CFB5CDB3CDF8C2E7B1C0C0A3A1
:10C93000A3ACD6D8C6F4CFB5CDB32100CED5CAD6D8
:10C94000D6D03A00C4A3BFE9B0B2D7B0D2ECB3A3FB
:10C9500021000000CED5CAD6CAA7B0DC0000000076
:10C96000C8EBCDF8D6D03A0005F00EFE384605F0FB
:10C9700007FE3078C10714D0810712D5400710D4C4
:10C9800097A001F08FFE02F000F8032844D0307821
:10C9900020F00400307096A005F0F6FD97A004F09A
:10C9A00052FA3078C10711D081070FD500070DD496
:10C9B00005F00FFC03283BD0307820F008003070E1
:10C9C00092A005F0E1FD95A004F03DFA97A005F0D6
:10C9D000DBFD3078C1073FF456AE81077FF553AEDB
:10C9E0004107FBD50007F9D5944804F0FEFE9348B3
:10C9F000401F04F0E1FB01F0B4FE257043E63078FF
:10CA000040F0010030708EA005F0BEFD58E6307891
:10CA100040F0020030706EE6307840F00400307074
:10CA20008AA14C2001F0CBFF8EA005F0ADFDB8E748
:10CA3000307840F0080030708DA001F033FE02F035
:10CA40007FF807468CA14C2001F0B9FF032F04D0DA
:10CA50008EA004F0F8F90AF04BFC96A005F094FDC6
:10CA600000F09EFAB2E708B54FF4E0314FF00060F5
:10CA700008F07BFA07F094FF4FF4407008F040FA9A
:10CA8000904800F047FB904800F0D0FB8F4800F042
:10CA9000A6FA8F4803F0E0FC07F082FF00F026FAC8
:10CAA00001F053FA8B4C01230A224FF47A7120785B
:10CAB00007F05DFE8849207807F03EFE07F070FF22
:10CAC000AFF26140009000234FF4FA72022183A07C
:10CAD0000AF030FE834C60600AF044FEAFF2AD40D5
:10CAE00000900123642202217FA00AF023FEA060AF
:10CAF0000AF038FEAFF2F540022300906422194696
:10CB00007CA00AF017FEE0600AF02CFEAFF2115094
:10CB1000009003236422022179A00AF00BFE206119
:10CB20000AF020FEAFF2BF5000900423322202210F
:10CB300075A00AF0FFFD60610AF014FEAFF24360D9
:10CB4000009005234FF47A62022172A00AF0F2FDF0
:10CB5000A0610AF007FEAFF22970009006230A22B6
:10CB6000022170A00AF0E6FDE0610AF0FBFDAFF2E1
:10CB7000A570009007230A2202216DA00AF0DAFDB9
:10CB800020620AF0EFFDAFF2CB7000900823322252
:10CB900001216AA00AF0CEFD60620AF0E3FDAFF663
:10CBA0001500009009233222012167A00AF0C2FD7E
:10CBB000A0620AF0D7FDAFF6BF0000900A2314224E
:10CBC000012164A00AF0B6FDE0620AF0CBFD6349E2
:10CBD000634801F069FE01F080FEFEE77047000047
:10CBE000C1ACBDD3544350B7FECEF1C6F73A0000F6
:10CBF000544350C1ACBDD3CAA7B0DC00544350C1AC
:10CC0000ACBDD3CAA7B0DC2100000000485454508A
:10CC1000B3F5CABCBBAFCAA7B0DC0000485454503F
:10CC2000B3F5CABCBBAFCAA7B0DC2100CACDB7C53B
:10CC300045433230D7CAD4B421000000F21B002093
:10CC4000CED5CAD6B3C9B9A621000000446576691D
:10CC500063652074637020636F6E6E6574636564D2
:10CC600021000000544350C1ACBDD3B3C9B9A600E4
:10CC7000D7A2B2E1D6D03A00446576696365205206
:10CC800065676973746572210000000048747470F0
:10CC9000B3F5CABCBBAF4F4BA3ACD7A2B2E1C7EB55
:10CCA000C7F3CAA7B0DCA3ACD6D8C6F4CFB5CDB312
:10CCB00021000000D3B2BCFED7A2B2E1B3C9B9A62D
:10CCC00021000000B20A0020440000206F0600206E
:10CCD0002465030030000020A1CF01084E65745484
:10CCE00061736B0000000020527332333254617361
:10CCF0006B00000052733438355461736B000000D0
:10CD00004C65645461736B00546370557263546175
:10CD1000736B000054637048656172745461736B87
:10CD200000000000546370446F776E5461736B00B1
:10CD300054637055705461736B0000004D656E75DF
:10CD40005461736B0000000055636D645461736B34
:10CD5000000000005573625461736B00B5770208E0
:10CD60007177020800B585B01322A34968460BF01D
:10CD7000FFF89DF80900401C8DF809009FA000886D
:10CD8000ADF80B00684607F0B5FB9B4804F05BF874
:10CD90009BA004F058F80AF0ABFA05B000BD70B5DE
:10CDA00005460C467B2008F085FA012804D122466E
:10CDB00098A128460BF0A4F97C2008F07BFA012802
:10CDC00004D1224696A128460BF09AF97D2008F05E
:10CDD00071FA012804D1224694A128460BF090F95B
:10CDE0007E2008F067FA012804D1224693A1284644
:10CDF0000BF086F97C2008F05DFA88B97D2008F0F8
:10CE000059FA68B97E2008F055FA48B97A2008F036
:10CE100051FA012804D122468CA128460BF070F962
:10CE2000BDE8704008F06DBB10B504460B2204F15C
:10CE300019000BF065F9002084F8250010BD10B52D
:10CE400004460B2204F125000BF05AF9002084F867
:10CE5000310010BD30B5A1B07F480AF0FBFC7F481F
:10CE60000AF0F8FC7E4C7F48211DFFF7E8FF7D4B60
:10CE70000B22253300217CA00AF0ECFC7948193004
:10CE8000054606F0DBFF29467648FFF7CDFF294629
:10CE90007AA00AF0DFFCA1787CA030390AF0DAFC35
:10CEA0000121704806F0D3FF6E4A18217CA00AF0D9
:10CEB000D1FC6C480B2131300446FFF770FF22464D
:10CEC0000B217CA00AF0C6FC63480AF0C3FC802159
:10CED00001A80BF0EEF823467BA2802101A80AF0FE
:10CEE000DBFC01A803F0AFFF21B030BD10B507F0A7
:10CEF000B0FB03F085FF002005F010FE0D2007F0C9
:10CF000067F9FFF7A7FFAFF2A311022006F0C6FFF3
:10CF100000F070FF03F019FA03F07DFA07F0E6FE67
:10CF200003F098FB4FF4E134204603F0C5FA2046A5
:10CF300003F0F4FABDE8104007F0B3BF2DE9F0416B
:10CF4000654D4FF48078404605F0E0FA0746634EA1
:10CF50007068C0F30F240BE042463946284607F0BC
:10CF600021FD3A465EA14C2001F029FD05F58075B2
:10CF7000641EA4B2F0D2414638460BF078F83279FC
:10CF80003946284607F00EFD3A4655A14C2001F0DF
:10CF900016FD384605F0F4FABDE8F04103F0E8BEAE
:10CFA00010B5524C207807F051FC5148007870B908
:10CFB0002C481022104913380AF009FF60B100F024
:10CFC0009DFF284814220C4913380BF099F820785B
:10CFD000BDE8104007F02BBC01F06DFBF7E7002126
:10CFE00040F8191F41608160C160016141611938D9
:10CFF00019210BF03CB80000445B002030310000E8
:10D000005274635F416C725F43616C6C6261636B0D
:10D0100021000000D6D8C9CFB5E7C6F4B6AF0000EE
:10D02000C8EDB8B4CEBBC6F4B6AF0000B6C0C1A25E
:10D03000BFB4C3C5B9B7C6F4B6AF0000B4B0BFDA69
:10D04000BFB4C3C5B9B7C6F4B6AF0000D3B2B8B465
:10D05000CEBBC6F4B6AF0000BCC9020800CA0208C5
:10D06000B20A00206F0600200D0A426F6F74B0E60E
:10D07000B1BE203A20252A2E2A7300000D0A415005
:10D080005020B0E6B1BE203A202573000D0A52753B
:10D090006E4170704E756D3A20415050256400000D
:10D0A0000D0AC9E8B1B8B1E0BAC5203A20252E2A48
:10D0B000730000000D0AD6D8C6F4D4ADD2F2203ADF
:10D0C00020252E2A73000000D6D8C6F4D4ADD2F2A3
:10D0D0003A25732E0000000000F80708C41B00204A
:10D0E000B1BEB5D86C6F673A2573000030000020E0
:10D0F00048000020F8220146F94807F0F6BC10B5B8
:10D10000F8210AF0B4FFBDE81040F822F549F448D0
:10D1100007F048BC7CB50446F34805F009FB2046FF
:10D12000FFF7EDFF5B202070302060703120A07091
:10D13000E070207CFF2809D104F110004021054651
:10D140000AF095FFE9A128460AF06DFE94F8500018
:10D15000FF2809D104F15000402105460AF087FF5D
:10D16000E4A128460AF05FFE94F89000FF2809D158
:10D1700004F19000402105460AF079FFDEA128461F
:10D180000AF051FE94F8D000FF2809D104F1D00034
:10D19000102105460AF06BFFDBA128460AF043FE8A
:10D1A00094F8E000FF2816D0A8B1CE49DA48E03163
:10D1B00001F0CEFB94F8F000FF2817D0B0B1C949B8
:10D1C000D548F03101F0D1FB5D2084F8F70020460E
:10D1D000BDE87C408EE704F1E000102105460AF02E
:10D1E00046FFC9A128460AF01EFEE3E70020C4F866
:10D1F000F000A4F8F400009001900A22694641F67C
:10D20000583005F0B4FB694604F1F0000AF00BFE5B
:10D21000DAE701460322C14807F067BC002202801A
:10D22000827001460322BD4807F0BCBB10B504461E
:10D230002046FFF7F3FF2046BDE81040E9E72DE95F
:10D24000F04105460F46032640F2492005F05EF9FD
:10D2500004463B464FF40077B1A2394604F126005C
:10D260000AF01AFB002801DDB8420BDD40F29E22D5
:10D27000ACA1B1A005F0E2F9204605F081F9022049
:10D28000BDE8F08128222270642190FBF1F2303257
:10D29000A27090FBF1F201FB12020A2192FBF1F263
:10D2A0003032E27090FBF1F201FB1200303020715D
:10D2B000A84908786071401CC0B20870392801D9AB
:10D2C000302008700422A4A1A01D0AF019FF01213A
:10D2D00004F10A0006F0BBFD3B2184F82210B5F8EA
:10D2E0002310A4F82310262184F8251068784328F9
:10D2F00014D072216170032299A120460AF055FDD5
:10D3000020460AF0BFFD401C82B22146002005F0F5
:10D3100044FE204605F034F93046B1E752216170F1
:10D3200003228FA120460AF040FD20460AF0AAFD04
:10D3300082B221468B4805F004FA0028E9D04FF468
:10D340002E7278A188A005F079F9E2E753207047A2
:10D350002DE9F04707463C46A0782179303800EBAC
:10D36000C00202EB001001EB8001E0786FF02F02A9
:10D37000303800EB800002EB40000D18DFF860A1B0
:10D38000F8225849504607F00DFB4FF4807630469E
:10D3900005F0BCF88046534B7BA2F03399463146EA
:10D3A00040460AF079FA064694F82300312804D161
:10D3B000611991F82610242902D030281DD021E0CF
:10D3C000102148460AF053FE2A4604F12601484639
:10D3D0000AF096FEF8224349504607F086FBC6F550
:10D3E000807108EB06004B466CA20AF055FA5324F4
:10D3F00041463846FFF723FF05E0601990F8260004
:10D40000242806D04924404605F0BAF82046BDE855
:10D41000F087532441463846FFF711FFF3E72DE923
:10D42000F04707463C46A0782179303800EBC0022F
:10D4300002EB001001EB8001E0786FF02F02303832
:10D4400000EB800002EB40000D18DFF894A0F822FA
:10D450002449504607F0A6FA4FF48076304605F08E
:10D4600055F880461F4B52A2E0339946314640465C
:10D470000AF012FA064694F82300312804D1611903
:10D4800091F82610242902D030281DD021E0102147
:10D4900048460AF0ECFD2A4604F1260148460AF007
:10D4A0002FFEF8220F49504607F01FFBC6F580718A
:10D4B00008EB06004B4643A20AF0EEF9532441461E
:10D4C0003846FFF7BCFE05E0601990F826002428D6
:10D4D00005D04924404605F053F8204697E77BE005
:10D4E00000880108B20A0020AC0600202F41424DFE
:10D4F0000000000041424D0053686F7033343437F0
:10D5000039343734390000003132312E34312E377E
:10D51000392E3837000000009A01002000900108E1
:10D520002573000055534552434D445C7573657235
:10D53000636D642E6300000025732C25643A7570BA
:10D5400044617461427566207370696C6C6F7665B6
:10D5500072A3A100340000204D41433A00000000B6
:10D5600024582900AA0B002025732C25643A7354F3
:10D570006370305175657565207370696C6C6F767A
:10D580006572A3A1000000002A4745542A20546375
:10D5900070506F72743A5B25735D21002A534554B5
:10D5A0002A20546370506F72743A5B25735D2100BA
:10D5B0002A4745542A2054637049503A5B25735DCD
:10D5C000210000002A5345542A2054637049503AE0
:10D5D0005B25735D21000000532441463846FFF768
:10D5E0002EFE77E72DE9F04707463C46A0782179E3
:10D5F000303800EBC00202EB001001EB8001E07854
:10D600006FF02F02303800EB800002EB40000D1865
:10D61000DFF8F4A3F822FB49504607F0C3F94FF4B2
:10D620008076304604F072FF8046F64BF7A2D03386
:10D630009946314640460AF02FF9064694F82300F1
:10D64000312804D1611991F82610242902D03028FC
:10D650001DD021E0102148460AF009FD2A4604F1B8
:10D66000260148460AF04CFDF822E649504607F0EC
:10D670003CFAC6F5807108EB06004B46E8A20AF0BA
:10D680000BF9532441463846FFF7D9FD05E06019F0
:10D6900090F82600242805D04924404604F070FF65
:10D6A0002046B4E6532441463846FFF7C8FDF4E768
:10D6B0002DE9F04707463C46A0782179303800EB49
:10D6C000C00202EB001001EB8001E0786FF02F0246
:10D6D000303800EB800002EB40000D18DFF828A383
:10D6E000F822C849504607F05DF94FF4807630467D
:10D6F00004F00CFF8046C34BCEA2903399463146CE
:10D7000040460AF0C9F8064694F82300312804D1AF
:10D71000611991F82610242902D030281DD021E06B
:10D72000402148460AF0A3FC2A4604F12601484657
:10D730000AF0E6FCF822B349504607F0D6F9C6F5E0
:10D74000807108EB06004B46C0A20AF0A5F85324EE
:10D7500041463846FFF773FD05E0601990F8260052
:10D76000242805D04924404604F00AFF20464EE60E
:10D77000532441463846FFF762FDF4E72DE9F047B0
:10D7800007463C46A0782179303800EBC00202EB16
:10D79000001001EB8001E0786FF02F02303800EBD1
:10D7A000800002EB40000D18DFF85CA2F8229549DA
:10D7B000504607F0F7F84FF48076304604F0A6FEA6
:10D7C0008046904BA7A250339946314640460AF016
:10D7D00063F8064694F82300312804D1611991F8C2
:10D7E0002610242902D030281DD021E040214846AF
:10D7F0000AF03DFC2A4604F1260148460AF080FC66
:10D80000F8228049504607F070F9C6F5807108EBA0
:10D8100006004B4699A20AF03FF853244146384689
:10D82000FFF70DFD05E0601990F82600242805D0CB
:10D830004924404604F0A4FE2046E8E5532441462E
:10D840003846FFF7FCFCF4E72DE9F04707463C4675
:10D85000A0782179303800EBC00202EB001001EB18
:10D860008001E0786FF02F02303800EB800002EB8F
:10D8700040000D18DFF890A1F8226249504607F0E9
:10D8800091F84FF48076304604F040FE80465D4BC0
:10D8900080A2103399463146404609F0FDFF064606
:10D8A00094F82300312804D1611991F82610242915
:10D8B00002D030281DD021E0402148460AF0D7FB95
:10D8C0002A4604F1260148460AF01AFCF8224D497E
:10D8D000504607F00AF9C6F5807108EB06004B4682
:10D8E00072A209F0D9FF532441463846FFF7A7FC3E
:10D8F00005E0601990F82600242805D04924404608
:10D9000004F03EFE204682E5532441463846FFF7A8
:10D9100096FCF4E72DE9F84307463C46DFF8E8902B
:10D92000F8223849484607F03DF84FF480752846FC
:10D9300004F0ECFD06466348804606F07FFACDF819
:10D940000080DFF8C08060A2294698F80230304697
:10D9500009F0A2FF054694F82300312804D167A1FD
:10D96000A01C05F07BF820B194F82300302821D0CA
:10D9700025E094F82600302807D0312805D0322839
:10D9800003D0332801D050241AE088F80200F8228E
:10D990001C49484607F0A9F898F80230C5F580718F
:10D9A000701957A209F078FF532431463846FFF723
:10D9B00046FC05E051A1A01C05F050F830B1492407
:10D9C000304604F0DDFD2046BDE8F883532431469F
:10D9D0003846FFF734FCF3E72DE9F04707463C46AD
:10D9E000DFF82490F8220749484606F0DBFF4FF4A1
:10D9F0008075284604F08AFD0646DFF8088098F80E
:10DA000001308FE0B20A0020008801082A474554FF
:10DA10002A2046747049503A5B25735D210000004E
:10DA20002A5345542A2046747049503A5B25735D49
:10DA3000210000002A4745542A2046747050617323
:10DA400073776F72643A5B25735D21002A534554E6
:10DA50002A2046747050617373776F72643A5B2545
:10DA6000735D21002A4745542A204674705573651A
:10DA7000726E616D653A5B25735D21002A534554D2
:10DA80002A20467470557365726E616D653A5B2528
:10DA9000735D21002A4745542A20467470466F6CF6
:10DAA0006465723A5B25735D210000002A5345547A
:10DAB0002A20467470466F6C6465723A5B25735D0C
:10DAC00021000000880600202A4745542A2052756C
:10DAD0006E4170704E756D3A5B41505025635D200C
:10DAE000212020202A4745542A2041707056657213
:10DAF00073696F6E3A5B25735D2021003030310011
:10DB00002A5345542A2052756E4170704E756D3AF5
:10DB10005B41505025635DD6D8C6F4BAF3C9FAD03C
:10DB2000A721000083A22946304609F0B5FE05462C
:10DB300094F82300312805D1AFF24001A01C04F075
:10DB40008DFF20B194F8230030281DD022E094F8F6
:10DB50002600302803D0312801D050241BE088F85B
:10DB60000100F8227949484606F0BFFF98F80130D5
:10DB7000C5F58071701976A209F08EFE53243146E6
:10DB80003846FFF75CFB06E0AFF29001A01C04F002
:10DB900065FF28B14924304604F0F2FC204636E403
:10DBA000532431463846FFF74AFBF4E7F0B58DB011
:10DBB0000446F82265496B4806F0F4FE6AA104F1B8
:10DBC000260004F04BFF18B149240DB02046F0BDEB
:10DBD0004FF40076304604F099FC07466448054649
:10DBE00006F02CF95948F030A0F12002A0F1E00332
:10DBF000CDE90932A0F11001CDE90B105D4A603882
:10DC0000A2F10903CDE905329039CDE90710111FC2
:10DC1000A0F18C029038C378CDE9022501930491DC
:10DC2000817800914378544A3146384609F034FEF1
:10DC300039462046FFF703FB5324384604F0A0FC86
:10DC4000C3E770B504464DA104F1260004F006FFB9
:10DC500010B15025284670BD53254AA12046FFF734
:10DC6000EEFA642006F039FD00F086FE642006F02E
:10DC700034FD03F061FB4CA003F0E5F809F038FB3C
:10DC8000E8E710B5044694F824003038112835D25E
:10DC9000DFE800F0090D1115191D2125292D343457
:10DCA0003434343431002046FFF7CBFF27E02046E0
:10DCB000FFF77CFF23E02046FFF78EFE1FE02046A3
:10DCC000FFF728FE1BE02046FFF7BEFD17E02046C9
:10DCD000FFF754FD13E02046FFF7EAFC0FE0204673
:10DCE000FFF780FC0BE02046FFF799FB07E020469A
:10DCF000FFF72EFB03E0FFF729FB00E04E202E4943
:10DD0000502809D049280DD04E2811D14968204605
:10DD1000BDE81040FFF793BA89682046BDE810407F
:10DD2000FFF78DBAC9682046BDE81040FFF787BAF3
:10DD300010BD00002A4745542A20496170466C6195
:10DD4000673A5B25635D212000000000B20A0020D5
:10DD50002A5345542A20496170466C61673A5B2515
:10DD6000635D2100008801084745545F4941500028
:10DD700088060020F61B002050CA0208434D445F6D
:10DD8000525354002A5345542A2055736572206318
:10DD90006F6E74726F6C206465766963652072655E
:10DDA0007374617274210000D6D8C6F4C3FCC1EE4E
:10DDB000C8EDD6D8C6F42100340000204949062019
:10DDC000487070474749072048707047454905200B
:10DDD0004870704743490920487070474149032003
:10DDE000487070473F490C20487070473D490B20F0
:10DDF0004870704710B502F0BBFAAFF20F010C206B
:10DE000005F02DFFAFF223010B2005F028FFAFF244
:10DE10003301092005F023FFAFF247010D2005F083
:10DE20001EFFAFF25701072005F019FFAFF26B019B
:10DE30000F2005F014FFAFF27B01BDE81040062073
:10DE400005F00DBF27484278011D0D2A48D2DFE8B2
:10DE500002F0474747174727372F471F47070F004D
:10DE6000027802EB420201EB8202527802702EE04D
:10DE7000027802EB420201EB82029278027026E005
:10DE8000027802EB420201EB8202D27802701EE0BD
:10DE9000027802EB420201EB82021279027016E074
:10DEA000027802EB420201EB8202527902700EE02C
:10DEB000027802EB420201EB82029279027006E0E4
:10DEC000027802EB420201EB8202D2790270002258
:10DED0004270007800EB400001EB80008068004752
:10DEE000704700004800002008B5FEA00023009005
:10DEF00003220C21184602F0E4FC08BD38B51E20B0
:10DF000004F004FB04460522FC4920460AF0F8F818
:10DF10000122002310211046009402F0D2FC1E21A1
:10DF200020460AF0A4F8F5490A220B3920460AF0E7
:10DF3000E7F8002302220C210120009402F0C1FC2A
:10DF40002046BDE8384004F01BBB10B5FFF7D6FFF4
:10DF5000BDE81040C8E708B5E9A0012300901A46C3
:10DF60001021002002F0ADFCE8A000230090022266
:10DF70001021184602F0A5FCE7A000230090032220
:10DF80001021184602F09DFC08BD08B5DCA0002356
:10DF9000009001221021184602F093FCDBA00090B3
:10DFA000012302221021002002F08BFCDAA00023C2
:10DFB000009003221021184602F083FC08BD08B52A
:10DFC000CFA00023009001221021184602F079FC16
:10DFD000CEA00023009002221021184602F071FC0E
:10DFE000CDA00090012303221021002002F069FC43
:10DFF00008BD08B5C5A000230090012210211846D5
:10E0000002F05FFCC4A000230090022210211846F9
:10E0100002F057FCC3A0009001230322102100202E
:10E0200002F04FFC08BD08B5C1A0012300901A46BC
:10E030001021002002F045FCC0A000230090022225
:10E040001021184602F03DFCBFA0002300900322DF
:10E050001021184602F035FC08BD08B5B4A0002315
:10E06000009001221021184602F02BFCB3A0009072
:10E07000012302221021002002F023FCB2A0002381
:10E08000009003221021184602F01BFC08BD08B5C1
:10E09000A7A00023009001221021184602F011FCD5
:10E0A000A6A00023009002221021184602F009FCCD
:10E0B000A5A00090012303221021002002F001FC02
:10E0C00008BD08B59DA0002300900122102118462C
:10E0D00002F0F7FB9CA000230090022210211846BA
:10E0E00002F0EFFB9BA000900123032210210020EF
:10E0F00002F0E7FB08BD08B599A0012300901A467D
:10E100001021002002F0DDFB98A0002300900222E5
:10E110001021184602F0D5FB97A00023009003229F
:10E120001021184602F0CDFB08BD08B58CA00023D5
:10E13000009001221021184602F0C3FB8BA0009032
:10E14000012302221021002002F0BBFB8AA0002341
:10E15000009003221021184602F0B3FB08BD08B559
:10E1600086A0012300901A461021002002F0A9FB8E
:10E1700085A00023009002221021184602F0A1FB86
:10E180007DA00023009003221021184602F099FB85
:10E1900008BD08B579A0002300900122102118467F
:10E1A00002F08FFB78A000900123022210210020B2
:10E1B00002F087FB70A00023009003221021184674
:10E1C00002F07FFB08BD08B572A0012300901A463B
:10E1D0001021002002F075FB71A0002300900222A4
:10E1E0001021184602F06DFB71A00023009003225D
:10E1F0001021184602F065FB08BD08B565A0002394
:10E20000009001221021184602F05BFB64A00090F0
:10E21000012302221021002002F053FB64A00023FE
:10E22000009003221021184602F04BFB08BD08B5F0
:10E2300058A00023009001221021184602F041FB53
:10E2400057A00023009002221021184602F039FB4B
:10E2500057A00090012303221021002002F031FB7F
:10E2600008BD08B556A0012300901A4610210020D1
:10E2700002F027FB55480023009002221021184687
:10E2800002F01FFB5148403809F0FCFD102809D965
:10E290004E4800233038009003221021184602F027
:10E2A00010FB08BD34A00023009003221021184663
:10E2B00002F007FB08BD08B545A0012300901A46EF
:10E2C0001021002002F0FDFA404800234030009069
:10E2D00002221021184602F0F4FA3C48403809F0B6
:10E2E000D1FD7BE04D454E552020202020202020D0
:10E2F00020202020204241434B0000004F5B0020A3
:10E3000046545020D0C5CFA20000000054435020F6
:10E31000D0C5CFA200000000C9E8B1B8C9FDBCB6A5
:10E3200000000000C9E8B1B8D0C5CFA200000000CD
:10E33000B2E9D1AF465450D5CBBAC500B2E9D1AF9E
:10E34000465450C3DCC2EB00B2E9D1AF4654502072
:10E3500020495000B2E9D1AF465450C2B7BEB60012
:10E36000B2E9D1AF5443502020495000B2E9D1AFB7
:10E37000544350B6CBBFDA0020000000B2E9D1AF61
:10E38000B5B1C7B041505000C1A2BCB4C9FDBCB6C4
:10E3900041505000B2E9D1AF4D4143494400000023
:10E3A000B2E9D1AF41505020B0E6B1BE000000004C
:10E3B000B2E9D1AF424F4F54B0E6B1BE0000000009
:10E3C000465450D5CBBAC53A00000000020B0020DD
:10E3D000465450C3DCC2EB3A00000000102808D9B4
:10E3E000F7480023009003221021184602F069FA32
:10E3F00008BDAFF27C0000230090032210211846D4
:10E4000002F05FFA08BD08B5EEA0012300901A469D
:10E410001021002002F055FAE9480023B0300090A6
:10E4200002221021184602F04CFAE548103809F093
:10E4300029FD102808D9E24800230090032210216A
:10E44000184602F03EFA08BDAFF2D4000023009057
:10E4500003221021184602F034FA08BD38B5DBA0BB
:10E46000012300901A461021002002F02AFAD44C11
:10E470000023103C022210211846009402F021FAD9
:10E48000204609F0FFFC102808D9CD480023009051
:10E4900003221021184602F014FA38BDAFF22810FA
:10E4A0000023009003221021184602F00AFA38BD1A
:10E4B00008B5C9A0012300901A461021002002F0DF
:10E4C00000FABF480023C0300090022210211846F5
:10E4D00002F0F7F9BA48103809F0D4FC102808D92E
:10E4E000B7480023009003221021184602F0E9F9F2
:10E4F00008BDAFF27C1000230090032210211846C3
:10E5000002F0DFF908BD08B5B5A0012300901A4656
:10E510001021002002F0D5F9A9480023D030009046
:10E5200002221021184602F0CCF9A548103809F053
:10E53000A9FC102808D9A24800230090032210212A
:10E54000184602F0BEF908BDAFF2D41000230090C7
:10E5500003221021184602F0B4F908BD38B5A3A073
:10E56000012300901A461021002002F0AAF9102081
:10E5700003F0CCFF04469248A0A2203810218378F3
:10E58000204609F089F90023022210211846009440
:10E5900002F097F9AFF2202000230090032210210F
:10E5A000184602F08EF92046BDE8384003F0E8BF77
:10E5B00010B58349312020394870F822944806F07C
:10E5C00094FA94A003F0E0FF022006F086F8BDE87C
:10E5D000104008F08DBE38B593A0012300901A4674
:10E5E0001021002002F06DF9192003F08FFF04467E
:10E5F0000121204605F02BFC002302220C211846A5
:10E60000009402F05EF904F115000023009003224B
:10E610000C21184602F055F92046BDE8384003F0B9
:10E62000AFBF38B582A0012300901A461021002008
:10E6300002F047F90C2003F069FF0446204605F07C
:10E64000FDFB0023022210211846009402F039F944
:10E65000AFF2DC200023009003221021184602F0C4
:10E6600030F92046BDE8384003F08ABF08B573A0F2
:10E67000012300901A461021002002F022F9504890
:10E6800000231C38009002221021184602F019F9CC
:10E69000AFF21C300023009003221021184602F034
:10E6A00010F908BD08B5002300901A46102118463D
:10E6B00002F007F908BD38B5634C2078C1074FF068
:10E6C00010000AD0009061A300220221382002F03D
:10E6D000CDF82068401C206038BDAFF26433009054
:10E6E00000220221382002F0C1F8F2E71CB50446EE
:10E6F00010210022009156A31146104602F0B6F8F0
:10E7000056490022CDE9002100211023202208468D
:10E7100002F0A3FA0C2100220091234611461A2090
:10E7200002F0A4F81CBD1CB5044610210022009183
:10E7300047A31146402002F099F848490022403191
:10E74000CDE90021102320220021402002F085FA8B
:10E750000C2100220091234611465A2002F086F82F
:10E760001CBD10B5102003F0D1FE04463C4B3DA269
:10E770001021204609F090F82046FFF7D4FF102121
:10E78000204609F074FC364B38A25B1D1021204650
:10E7900009F082F82046FFF7A9FF2046BDE81040A7
:10E7A00003F0EEBE08B500230090012210211846A8
:10E7B00002F087F8BDE80840022002F077B80000B8
:10E7C000D20A00204654502049503A00465450C2C4
:10E7D000B7BEB63A000000005443502049503A00FA
:10E7E000544350B6CBBFDA3A00000000B5B1C7B011
:10E7F000D4CBD0D0415050BAC53A000052756E41CA
:10E8000070704E756D3A5B25635DA1A3000000003A
:10E8100000880108C9FDBCB6C9E8B1B8A3ACBCB456
:10E82000BDABD6D8C6F400004D414349443A000080
:10E8300041505020B0E6B1BEBAC53A00424F4F54E5
:10E84000B0E6B1BEBAC53A00900100203A0000001F
:10E85000202020202020202000000000A6B4020854
:10E86000ED1B002025736D56000000004353512519
:10E870007300000008B5002300900222102101203F
:10E8800002F01FF808BD38B50C46002300900122A5
:10E890001021184602F015F8002302221021184614
:10E8A000009402F00EF838BD70B505460C46002302
:10E8B0000F220A21032005F05AFF2946032005F004
:10E8C0003BFF00230E220A21022005F050FF2146C3
:10E8D000BDE87040022005F02FBF10B5032005F001
:10E8E000A6FFBDE81040022005F0A1BF10B503202F
:10E8F00005F0ACFFBDE81040022005F0A7BF1348AB
:10E900000168491C01600168491C00D10160704721
:10E9100010B500230C226421052005F028FFAFF27A
:10E920002101BDE81040052005F006BF10B5052007
:10E9300005F07DFF05490020086010BD10B50520D9
:10E9400005F084FF0148006810BD0000940100201C
:10E9500070B504460D461021601C09F088FB29465D
:10E96000601CBDE8704009F05EBA10B50446084668
:10E9700009F004FA608210BD10B5002003F0BCF964
:10E98000BDE81040012002F056BE10B503F0DEF8DD
:10E9900003280CD1434803F0B3F904464149032C42
:10E9A00006D04A8A491C40A003F048FE204610BD0C
:10E9B0004A8A491C43A003F0E7FD204610BD0FB46E
:10E9C000F8B50646032540F2492003F09FFD0446B2
:10E9D00008AB00934FF40077394604F12600079AFC
:10E9E00008F01EFF002801DDB8420BDD82223CA1A9
:10E9F00040A003F023FE204603F0C2FD0220F8BC35
:10EA00005DF814FB282222706670642290FBF2F1FC
:10EA10003031A17090FBF2F102FB11010A2291FB4F
:10EA2000F2F13031E17090FBF2F102FB1100303075
:10EA300020711C49891E08786071401CC0B20870A2
:10EA4000392801D930200870042231A1A01D09F015
:10EA500057FB012104F10A0005F0F9F93B2184F884
:10EA600022103022022104F1230009F0F8FA2621B5
:10EA700084F82510032228A1204609F096F92046A3
:10EA800009F000FA82B22146244803F05AFE20B170
:10EA9000A12213A122A003F0D1FD204603F070FDB6
:10EAA0002846ACE79A010020544350205365727603
:10EAB0006572C1ACBDD3CAA7B0DC3A25733A2564F0
:10EAC00020A3A10054435020536572766572C1ACF7
:10EAD000BDD3B3C9B9A63A25733A256420A3A100D2
:10EAE000555345525F5443505C757365725F746350
:10EAF000702E630025732C25643A7570446174612F
:10EB0000427566207370696C6C6F766572A3A100A4
:10EB10004D41433A0000000024582900AA0B002070
:10EB200025732C25643A735463703051756575658F
:10EB3000207370696C6C6F766572A3A10000000091
:10EB4000F0B585B00121374805F081F901F0E0FA10
:10EB50000746344801F0C6FA024633A1384601F0B0
:10EB6000ADF9384601F04AF9044621462FA003F0DA
:10EB700039FD2146324803F037FB0446032C0DD003
:10EB80003048017821F0080101702FA002F05BF9F4
:10EB9000384600F0D7F805B02046F0BD03F071FB11
:10EBA0000446032CF4D17B212B4809F060F900F0D6
:10EBB000E2FD064630000FD028A101F04AF90546D3
:10EBC00015B1E86804280FD0022427A003F036FD11
:10EBD000304600F0B7F8DBE700F068F8014627A000
:10EBE00003F0D2FC0224F3E713222848296909F034
:10EBF00087FA264805F0DEFB13222449684609F00F
:10EC0000B7F99DF80900401C8DF8090020A0008884
:10EC1000ADF80B00684605F06DFC1EA0296903F0F5
:10EC2000E1FCD5E76F0600206D616300D3B2BCFE46
:10EC3000D7A2B2E14A534F4EA3BA25730000000099
:10EC4000B0010020310000204874747020706F7390
:10EC500074206572722E0000501D00207379735469
:10EC6000696D6532000000004E6F20226A736F6E7E
:10EC70005F74696D6522202E00000000636A736F67
:10EC80006E206572723A257300000000445B00201C
:10EC9000303100002573CEAABBF1C8A1B5BDB5C403
:10ECA000B7FECEF1C6F7CAB1BCE42E00FE4800683C
:10ECB000704770B504460D46002C01D02DB10AE016
:10ECC0000DB1012070BD002070BD012070BD207805
:10ECD00098B1641C6D1C207808F095FD06462878D4
:10ECE00008F091FD8642F2D0207808F08CFD0446B1
:10ECF000287808F088FD201A70BD002070BD70B51E
:10ED00000646304609F0BEF8451C284603F0FEFBD7
:10ED1000041E06D02A463146204609F029F920462D
:10ED200070BD204603F02CFC002070BD10B52820DB
:10ED300003F0ECFB04461CB12821204609F0B9F988
:10ED4000204610BD70B5044619E02568A089C005AD
:10ED500003D4A06808B1FFF7F5FFA089C00503D46C
:10ED6000206908B103F00CFCA089800503D4206A57
:10ED700008B103F005FC204603F002FC2C46002CF1
:10ED8000E3D170BD2DE9F34F85B08A4600242546B6
:10ED9000C6490020CDE902010026374683460120FE
:10EDA00001909AF800002D2805D1C1490020CDE935
:10EDB00002010AF1010A9AF80000302801D10AF193
:10EDC000010A9AF800003138082817D89AF800008C
:10EDD00030380BF0F0FE804689460022B54B2046C5
:10EDE00029460BF04FFF42464B460BF037FC0446DA
:10EDF0000D461AF8010F30380928E7D99AF80000B3
:10EE00002E2827D19AF80100302823D3392821D879
:10EE10000AF1010A9AF8000030380BF0CCFE804667
:10EE200089460022A34B204629460BF02BFF424681
:10EE30004B460BF013FC04460D4600229B4B30461C
:10EE400039460CF045F906460F461AF8010F3038DE
:10EE50000928DFD99AF80000652801D045281DD17E
:10EE60001AF8010F2B2802D02D2803D010E00AF148
:10EE7000010A0DE04FF0FF3001900AF1010A07E0AE
:10EE80000BEB8B0100EB410B0AF1010AABF1300BEC
:10EE90009AF80000A0F130010929F1D901980BFB83
:10EEA00000F00BF088FE32463B460BF0D7FB0246E3
:10EEB0000B4600207F490AF093FE06460F46DDE927
:10EEC000020122462B460BF0DDFE32463B460BF09C
:10EED000D9FE04460D460598C0E906452046294658
:10EEE0000BF00CFE0599486105980321C16007B03D
:10EEF0005046BDE8F08F401E40EA600040EAA000A6
:10EF000040EA201040EA202040EA2040401C7047A0
:10EF100070B50446002C08D0236833B1A26850189D
:10EF20006168814203DB981870BD002070BDFFF757
:10EF3000E2FF0646304603F0E9FA054665B1D4E93A
:10EF40000012284609F014F8206803F019FB6660E7
:10EF50002560A068284470BD206803F011FB0020E4
:10EF60006060206070BD10B50446002C08D0206899
:10EF700030B1A168084408F085FFA168084410BDBD
:10EF8000002010BD2DE9F04707460E46DFF8288126
:10EF9000D7E9064500221346204629460BF072FDAC
:10EFA00012D12EB102213046FFF7B2FF814603E0B5
:10EFB000022003F0ABFA8146B9F1000F03D03FA065
:10EFC0000088A9F800009CE078690BF0F4FD224667
:10EFD0002B460CF07DF821F00041002243460BF057
:10EFE00015FE21D8364A374B204629460BF00EFE37
:10EFF0001AD80022344B204629460BF041FF13D883
:10F000002EB115213046FFF783FF814603E015201E
:10F0100003F07CFA8146B9F1000F72D02BA148466B
:10F020007A6908F023FC6CE02EB140213046FFF7EE
:10F030006FFF814603E0402003F068FA8146B9F192
:10F04000000F5ED0204629460AF0AEFB22462B4632
:10F050000CF03EF821F00041002243460BF0D6FDB3
:10F060000ED825F000412046194A1A4B0BF0CEFD70
:10F0700006D222462B4618A1484608F0F7FB40E08E
:10F08000204625F0004106460F46154A154B0BF069
:10F09000BDFD06D3304639460022134B0BF0F0FE7F
:10F0A00029D222462B4621E0C00100200000F03F7B
:10F0B0000000F0BF000024400000B03C3000000021
:10F0C0000000C0FFFFFFDF410000E0C12564000039
:10F0D00044F3C2E4E4E9634C252E306600000000EE
:10F0E0008DEDB5A0F7C6B03E65CDCD41F6A1484641
:10F0F00008F0BCFB05E022462B46F4A1484608F088
:10F10000B5FB4846BDE8F0870178A1F13002092A35
:10F1100001D811460AE0A1F14102052A01D8373988
:10F1200004E0A1F16102052A0AD857390A01401CFE
:10F130000178A1F13003092B04D8303A11440EE0D4
:10F1400000207047A1F14103052B02D8373A114442
:10F1500005E0A1F16103052B0BD8573A11440A01D0
:10F16000401C0178A1F13003092B04D8303A114436
:10F170000EE000207047A1F14103052B02D8373A79
:10F18000114405E0A1F16103052B0AD8573A114457
:10F1900009014078A0F13002092A04D83039084426
:10F1A000704700207047A0F14102052A02D8373984
:10F1B00008447047A0F16102052A02D85739084473
:10F1C0007047002070472DE9F04780460D466C1CC3
:10F1D00000202978222907D0BD480560002091E74A
:10F1E000641C5C2A00D1641C2278222A02D00AB155
:10F1F000401CF5D1401C03F089F90746380004D0C3
:10F20000681C3C464FF480691AE000207AE75C29CC
:10F2100003D004F8011B401C12E0461C3078722811
:10F2200025D006DC622816D0662818D06E2804D1B6
:10F2300019E074281FD0752821D004F8010B701C28
:10F240000178222901D00029E1D100212170017823
:10F2500022296AD06AE0082004F8010BEFE70C20AD
:10F2600004F8010BEBE70A2004F8010BE7E70D2097
:10F2700004F8010BE3E7092004F8010BDFE7701C39
:10F28000FFF742FF0546361DA5F55C404845D6D33D
:10F29000002DD4D0A5F55840484513D270785C288D
:10F2A000CDD1B0787528CAD1F01CFFF72DFFB61D5F
:10F2B000A0F55C414945C2D2C5F3090161F39F2025
:10F2C00000F580350421802D01D2012108E0B5F53B
:10F2D000006F01D2022103E0B5F5803F00D2032187
:10F2E000601801291AD0022911D0032908D0042955
:10F2F00019D105F0BF0242F0800200F8012DAD09DE
:10F3000005F0BF0242F0800200F8012DAD0905F0C2
:10F31000BF0242F0800200F8012DAD096D4A525C37
:10F320002A4300F8012D441889E7401CC8F81070E2
:10F330000421C8F80C10E5E62DE9F04705468A4699
:10F3400000240021A9460AE0421E1F2A11D32228C8
:10F350000FD05C280DD00020014309F1010999F874
:10F3600000000028F0D18046222721B125B32E4687
:10F3700044E00120F0E7A9EB0506BAF1000F05D043
:10F38000F11C5046FFF7C4FD044603E0F01C03F0F7
:10F39000BDF8044674B1277004F1010929464846B6
:10F3A00008F041FD09F8067009EB060080F80180BD
:10F3B0002046A7E60020A5E6BAF1000F05D00321FC
:10F3C0005046FFF7A5FD044603E0032003F09EF836
:10F3D00004462CB140A1204608F025FD204691E6C8
:10F3E00000208FE649463DA008F0D5FC08B1641C1A
:10F3F00003E0B9F1200F00D2641D761C96F800904E
:10F40000B9F1000F01D0641CECD1BAF1000F05D0A6
:10F41000E11C5046FFF77CFD064603E0E01C03F0CC
:10F4200075F806462EB1304600F8017B4FF05C09B6
:10F4300025E0002066E61F2907D9222905D05C298E
:10F4400003D000F8011B6D1C19E000F8019B044675
:10F4500015F8012B0C2A25D006DC082A1ED0092A13
:10F460002CD00A2A06D121E00D2A23D0222A12D03C
:10F470005C2A0CD01BA1204608F0F8F9601D297801
:10F480000029D8D1077080F8018030463AE684F828
:10F490000090601CF3E72770601CF0E7622020708A
:10F4A000601CECE766202070601CE8E76E2020708E
:10F4B000601CE4E772202070601CE0E7742020707C
:10F4C000601CDCE7006937E7256500002566000061
:10F4D000C001002026B5020822220000225C080C90
:10F4E0000A0D0900752530347800000000E0401C4A
:10F4F000002804D00178002901D02029F7D97047CD
:10F500002DE9F04107460878FE4E7B2803D0316094
:10F510000020BDE8F0810620F860481CFFF7E6FFF8
:10F52000054628787D2818D0FFF700FC0446B8600F
:10F53000A8B12846FFF7DAFF01462046FFF743FE51
:10F54000FFF7D4FF68B121692162002727610178A4
:10F550003A2908D030600020DBE7681CD9E700209A
:10F56000D7E70020D5E7401CFFF7C0FF0146204643
:10F5700000F086F8FFF7BAFF0546280028D1C8E753
:10F58000FFF7D4FBA8B1206044600446681CFFF775
:10F59000ADFF01462046FFF716FEFFF7A7FF50B16B
:10F5A00021692162276101783A2906D03060002064
:10F5B000AFE70020ADE70020ABE7401CFFF796FF68
:10F5C0000146204600F05CF8FFF790FF054645B184
:10F5D00028782C28D4D028787D2804D035600020C5
:10F5E00097E7002095E7681C93E72DE9F04107466F
:10F5F0000878C44E5B2802D03160002089E70520DE
:10F60000F860481CFFF772FF044620785D2811D08F
:10F61000FFF78CFB0546B86070B12046FFF766FF28
:10F620000146284600F02CF8FFF760FF0446200052
:10F6300004D016E0601C6CE700206AE7002068E751
:10F64000FFF774FBB0B1286045600546601CFFF70A
:10F650004DFF0146284600F013F8FFF747FF044628
:10F6600054B120782C28EBD020785D2806D0346067
:10F6700000204EE700204CE700204AE7601C48E7E6
:10F6800070B505460C46002C20D004229EA12046D1
:10F6900008F017FCE0B105229DA1204608F011FCFE
:10F6A000D0B104229CA1204608F00BFCC0B1207808
:10F6B00022281AD02D2803D0A0F13001092919D809
:10F6C00021462846BDE87040FFF75CBB002070BDB6
:10F6D0000220E860201D70BD0020E860601D70BD44
:10F6E0000120E8606861201D70BD21462846BDE804
:10F6F000704068E55B2805D07B2808D0814804600D
:10F70000002070BD21462846BDE870406DE72146C7
:10F710002846BDE87040F3E62DE9F04104460D4669
:10F720009046FFF703FB0646764F00203860BEB1D7
:10F730002046FFF7DBFE01463046FFF7A1FF0446F7
:10F7400084B1B8F1000F12D02046FFF7CFFE044677
:10F75000207860B13046FFF7F5FA3C600020D8E62B
:10F760000020D6E63046FFF7EDFA0020D1E605B1DD
:10F770002C603046CDE600221146CDE72DE9F04F52
:10F7800085B00646894615461C4600200490072091
:10F7900002904FF0000BB06800270021019101E0BA
:10F7A0007F1C00680028FBD137B1002C70D0A768FF
:10F7B00095B34FF0020A32E04CB115B109F10401E2
:10F7C00000E003212046FFF7A3FB024607E015B146
:10F7D00009F1040000E0032002F098FE024662B145
:10F7E00010467B2100F8011B85B10A2100F8011B9E
:10F7F00000210923A9F1010906E0002005B0BDE8B8
:10F80000F08F00F8013B491C4945FADB7D2101706E
:10F81000002141701046F1E7FFE74FF0010A0AF1BD
:10F8200001012046FFF774FB88B17B2100F8011B22
:10F8300015B10A2100F8011B4FF0000880F8008084
:10F84000A0685044A060B66809F101096CE000208E
:10F85000D4E78DB149462046FFF75AFB10B100218D
:10F86000092204E00020C9E700F8012B491C4945A2
:10F87000FADBA0684844A0602146306AFFF75CFDCF
:10F880002046FFF770FBA0601DB14FF0020A02E0B6
:10F890006CE04FF0010A51462046FFF739FBA8B152
:10F8A0003A2100F8011B0DB109210170A0685044F4
:10F8B000A06023462A464946304600F026FA2046F4
:10F8C000FFF751FBA0601DB1012002E0002095E789
:10F8D0000020316809B1012100E0002100EB010A9C
:10F8E0000AF101012046FFF713FB18B3316811B18B
:10F8F0002C2100F8011B15B10A2100F8011B80F82A
:10F9000000800DE0C00100206E756C6C00000000EE
:10F9100066616C736500000074727565000000001C
:10F92000A0685044A0603668002E92D125B109F13C
:10F93000010102E0002061E702212046FFF7E8FA1A
:10F9400028B15DB100270921A9F1010904E00020D7
:10F9500054E700F8011B7F1C4F45FADB7D21017045
:10F9600080F80180206838440490D7E0BC0020462D
:10F9700002F0CCFD80465FEA080016D0204602F077
:10F98000C5FD82465FEA0A0011D02146404608F0D4
:10F9900090FB2146504608F08CFBB46809F1010940
:10F9A0008DB302984844029031E0002026E740469B
:10F9B00002F0E6FD002021E70021206AFFF7BCFCF1
:10F9C00003904AF82B0000232A464946204600F0BF
:10F9D0009CF959460BF1010B48F82100039999B1A4
:10F9E00090B108F04FFA0646039808F04BFA311828
:10F9F00015B109F1020000E000200144029808441A
:10FA0000801C029002E002E0012001902468002C9A
:10FA1000D2D1019818B9029802F078FD04900498A8
:10FA200008B9012001900198B0B100240AE05AF809
:10FA3000240008B102F0A4FD58F8240008B102F037
:10FA40009FFD641CBC42F2DB504602F099FD40462B
:10FA500002F096FD0020D1E604997B200870049CFA
:10FA6000641C15B10A2004F8010B4FF0000B84F858
:10FA700000B000263BE03DB10020092102E004F87F
:10FA8000011B401C4845FADB5AF8260008F0FAF939
:10FA900000905AF826102046009A08F069FA00985B
:10FAA00004443A2004F8010B15B1092004F8010BB5
:10FAB00058F82610204608F0B6F958F8260008F045
:10FAC000E1F90444781E864202D02C2004F8010B90
:10FAD00015B10A2004F8010B84F800B05AF826008A
:10FAE00002F04EFD58F8260002F04AFD761CBE4298
:10FAF000C1DB504602F044FD404602F041FD4DB1ED
:10FB000000200921A9F1010902E004F8011B401CB1
:10FB10004845FADB7D20207084F801B004986DE63A
:10FB20002DE9FF4F81B0834690461F464FF00009F4
:10FB30004FF0050ADBF8080000260025002401E04C
:10FB4000761C00680028FBD17EB1002F5FD0BE6814
:10FB500001213846FFF7DCF9C8B15B210170B868B4
:10FB6000401CB860DBF808503DE02FB10321384657
:10FB7000FFF7CEF9044603E0032002F0C7FC044679
:10FB80001CB1FCA1204608F04EF9204636E60020C4
:10FB900034E602993B464246491C284600F0B5F837
:10FBA0003846FFF7E0F9B8602868D8B1B8F1000F1F
:10FBB00002D04FF0020901E04FF0010909F1010103
:10FBC0003846FFF7A5F9F0B12C2100F8011BB8F178
:10FBD000000F02D0202100F8011B00210170B8683D
:10FBE0004844B8602D680DB1002CD2D002213846AF
:10FBF000FFF78EF948B15D2101700021417038682E
:10FC000000EB06097FE00020F8E50020F6E5B000F3
:10FC1000009002F07BFC0746380005D0009908F000
:10FC200048FADBF808B01EE00020E7E5029900235F
:10FC30004246491C584600F068F829466D1C47F8B2
:10FC4000210068B108F01EF90146B8F1000F01D09B
:10FC5000012000E00020084482440AF1020A00E08A
:10FC60000124DBF800B0BBF1000F01D0002CDDD087
:10FC70001CB9504602F04AFC8146B9F1000F00D190
:10FC8000012474B1002405E057F8240008B102F003
:10FC900077FC641CB442F7DB384602F071FC0020AC
:10FCA000ACE55B2089F800004C464FF0000A04F8F0
:10FCB00001AF00251EE057F8250008F0E3F8834661
:10FCC00057F825105A46204608F052F95C44701E39
:10FCD00085420AD02C2004F8010BB8F1000F02D0A5
:10FCE000202004F8010B84F800A057F8250002F04A
:10FCF00047FC6D1CB542DEDB384602F041FC5D205E
:10FD0000207084F801A0484678E570B500240028EA
:10FD100009D083B3057B072D6ED2DFE805F01320F1
:10FD2000062D32373B00002070BD05211846FFF735
:10FD3000EFF80446002C5FD0AFF23441204608F0C3
:10FD400072F859E006211846FFF7E2F80446002C45
:10FD500052D0AFF24441204608F065F84CE005214E
:10FD60001846FFF7D5F8044634B3AFF254412046A5
:10FD700008F059F840E011E01946FFF703F904468E
:10FD80003AE01946FFF79EFB044635E0FFF7C8FE50
:10FD9000044631E0FFF7F2FC04462DE0037B072B1D
:10FDA0002AD2DFE803F00A1004161B202500AFF268
:10FDB000A840FEF7A4FF04461EE0AFF2AC40FEF7F9
:10FDC0009EFF044618E0AFF2B040FEF798FF0446ED
:10FDD00012E00021FFF7D6F804460DE00021FFF7FE
:10FDE00071FB044608E00023FFF79AFE044603E097
:10FDF0000023FFF7C3FC0446204670BD0023012208
:10FE0000194682E700231A4619467EE7FEB50546E5
:10FE10000C461646204602F079FB00900194002023
:10FE200002906B46324600212846FFF76EFFFEBD6A
:10FE30008168002001E0401C09680029FBD170475F
:10FE4000806801E0491E0068002801D00029F9DC23
:10FE5000704770B50D46846800E024682CB12946CF
:10FE6000206AFEF726FF0028F7D1204670BD01600A
:10FE70004860704770B50546FEF758FF044674B1F8
:10FE800028222946204608F0B8F800202062E168C0
:10FE900041F48071E16060602060204670BD002008
:10FEA00070BD02469068002901D010B9916070477A
:10FEB000104610B10268002AFAD1D8E770B505469D
:10FEC0000E461446002C0CD0206A08B102F058FBF4
:10FED0003046FEF714FF206221462846BDE87040F8
:10FEE000DFE770BD70B506460D461446002C10D0F5
:10FEF000A089800503D4206A08B102F041FB256285
:10FF0000E06840F40070E06021463046BDE8704093
:10FF1000C7E770BD10B504460846FFF7ABFF0146C2
:10FF20002046BDE81040BCE770B504460D461046BB
:10FF3000FFF7A0FF024629462046BDE87040BDE716
:10FF40000246906801E00068491E08B10029FADC09
:10FF500090B1416809B103680B60016809B1436859
:10FF60004B609168814201D101689160002101607C
:10FF7000416070475B5D00000020FAE710B5FFF7B5
:10FF8000DFFFBDE81040FEF7DDBE2DE9F04106467B
:10FF90000F460025B46801E06D1C24682CB1394679
:10FFA000206AFEF786FE0028F6D124B129463046A5
:10FFB000BDE8F041C4E70020BDE8F08110B5FFF7CF
:10FFC000E4FFBDE81040FEF7BDBE30B40C4611465C
:10FFD000836801E01B68641E0BB1002CFADC4BB196
:10FFE0000B605A684A60596082689A4204D1816005
:10FFF00030BC704730BC54E748680160F8E730B463
:020000040802F0
:100000000346986801E00068491E08B10029FADC3F
:100010000028EDD0016811604468546001B14A6065
:100020009968814201D19A6001E051680A6000211B
:100030004160016030BCFEF785BED9E72DE9F04193
:100040000646884617460025B46801E06D1C246802
:100050002CB14146206AFEF72CFE0028F6D1002C78
:10006000AAD04046FEF74BFE38623A462946304653
:10007000BDE8F041C3E79FE710B5FEF757FE002843
:1000800001D00221C16010BD10B5FEF74FFE00285F
:1000900001D00121C16010BD10B5FEF747FE002858
:1000A00001D00021C16010BD10B50446FEF73EFE30
:1000B000002804D00CB1012100E00021C16010BD76
:1000C00070B504460D46FEF731FE064646B10320E4
:1000D000F060C6E90645204629460AF00FFD70612A
:1000E000304670BD70B50546FEF720FE04462CB1C3
:1000F0000420E0602846FEF702FE2061204670BD25
:1001000010B5FEF713FE002801D00521C16010BD17
:1001100010B5FEF70BFE002801D00621C16010BD0E
:100120002DE9F047804689460027FFF7E9FF06469C
:1001300000240DE058F824000AF03DFDFFF7C0FF51
:1001400005465CB129463846FFF791FE2F46641CF0
:100150000EB14C45EEDB3046BDE8F087B560F5E703
:100160002DE9F047804689460027FFF7C9FF06467C
:1001700000240DE058F824000BF094F8FFF7A0FFDE
:10018000054654B129463846FFF771FE2F46641CD8
:100190000EB14C45EEDB3046DEE7B560F6E72DE903
:1001A000F047804689460027FFF7AAFF064600244D
:1001B0000CE008EBC40103C9FFF782FF054654B108
:1001C00029463846FFF753FE2F46641C0EB14C45B6
:1001D000EFDB3046C0E7B560F6E72DE9F0470746AC
:1001E00088464FF00009FFF78BFF064600240BE01E
:1001F00057F82400FFF776FF054654B129464846D4
:10020000FFF735FEA946641C0EB14445F0DB3046CD
:10021000A2E7B560F6E72DE9F04106460F46002457
:10022000002E1DD0FEF782FD054628001AD0F0688A
:1002300020F48070E86070696861D6E90601C5E95C
:100240000601306918B1FEF75AFD286160B1306AC5
:1002500018B1FEF754FD286258B17FB1B66821E0AD
:100260000020A9E60020A7E62846FEF76BFD002047
:10027000A2E62846FEF766FD00209DE628469BE69E
:1002800001213046FFF7C7FF20B144B12060446030
:10029000044606E02846FEF755FD00208CE6A860DF
:1002A00004463668002EEBD1284685E6014626E056
:1002B000202A08D0092A08D00D2A08D00A2A08D0F6
:1002C0002F2A08D00AE0401C19E0401C17E0401C0F
:1002D00015E0401C13E043782F2B03D02F2A06D0C3
:1002E00008E0401C027852B10A2A08D0F9E74378A6
:1002F0002A2B0BD0222A12D001F8012B401C0278A5
:10030000002AD5D10020087033E6401C027822B1C3
:100310002A2AFAD142782F2AF7D1801CEFE701F878
:10032000012B401C08E05C2A02D101F8012B401C83
:1003300010F8012B01F8012B02780AB1222AF2D120
:1003400010F8012B01F8012BD9E710220921042014
:1003500003F014BC0921042003F076BC10B5FFF7AC
:10036000F9FF4FF4C87004F0B8F9BDE81040F1E7A8
:1003700038B506240C23482219460020009403F0C7
:1003800019FC082348220B210020009403F012FCE2
:100390000823482209210220009403F00BFC0823C3
:1003A000482207210220009403F004FC082348227D
:1003B00006210220009403F0FDFB082348220F21B0
:1003C0000320009403F0F6FB082348220D210320AC
:1003D000009403F0EFFB48220B21032003F0CEFB37
:1003E00048220821002003F0C9FB482209210220ED
:1003F00003F0C4FB48220821022003F0BFFB48227F
:100400000E21032003F0BAFBBDE8384048220C213E
:10041000032003F0B3BB10220A21042003F0AEBB7B
:100420000A21042003F010BC10B5FFF7F9FF4FF4C8
:10043000C87004F052F9BDE81040F1E710B50A4663
:100440000146114802F07DF9002804D0BDE81040B3
:100450000EA002F0F3B810BD10B504460A4802F031
:1004600067F901230C222146002002F061FCAFF263
:100470003301BDE81040002002F02EBC0A460146C0
:10048000002002F08ABD0000B00F00207355736297
:100490005175657565D2E7B3F6A3A10010B50A469C
:1004A0000146114802F04DF9002804D0BDE8104083
:1004B0000EA002F0C3B810BD10B504460A4802F001
:1004C00037F905230C222146042002F031FCAFF25B
:1004D0003301BDE81040042002F0FEBB0A4601468D
:1004E000042002F05ABD0000B613002073525332AC
:1004F00033325175657565D2E7B3F6A3A1000000EC
:1005000010B50A460146184802F01BF9002804D02D
:10051000BDE8104015A002F091B810BD10B504461A
:1005200010220021032003F029FB154B00221A6042
:100530000D4802F0FDF805230C222146032002F0AD
:10054000F7FBAFF24301BDE81040032002F0C4BB4B
:1005500010B50A460A4C012121600146032002F031
:100560001CFD0020206010BDBC17002073525334C6
:1005700038355175657565D2E7B3F6A3A100000063
:100580008081224270B5002400250126F84B012904
:100590000CD00022C3F89851C3F89051C3F894517D
:1005A0003AB101060DD5C3F89C510CE0C3F898612F
:1005B000F2E7010602D5C3F89C6104E0C3F89C5140
:1005C00001E0C3F89C61C3F894614006000E641C0E
:1005D000E4B2082CE2D3C3F89061C3F8986170BD0F
:1005E00010B50446B031C8B200221146FFF7CAFF69
:1005F000A41CC4F30310002240F010001146FFF7C2
:10060000C1FF04F00F000022BDE810401146B9E719
:1006100030B5002505F1B0000022C0B21146FFF749
:10062000B1FF002211460220FFF7ACFF0022114665
:100630001020FFF7A7FF0024002201211046FFF73A
:10064000A1FF641CE4B2802CF6D36D1CEDB2082D22
:10065000E0D330BD70B510220421002003F08EFAE3
:1006600010220521002003F089FA10220621002023
:1006700003F084FA10220721002003F07FFA1022F1
:100680000521022003F07AFABA4C01252560642086
:1006900004F023F800202060642004F01EF8256098
:1006A00000221146AE20FFF76DFF00221146022006
:1006B000FFF768FF002211461020FFF763FF0022BA
:1006C00011464020FFF75EFF002211468120FFF710
:1006D00059FF00221146FF20FFF754FF0022114668
:1006E000A120FFF74FFF00221146C820FFF74AFF65
:1006F00000221146A620FFF745FF00221146A82040
:10070000FFF740FF002211463F20FFF73BFF00228A
:100710001146D320FFF736FF002211461046FFF79F
:1007200031FF00221146D520FFF72CFF0022114691
:100730008020FFF727FF00221146D920FFF722FF74
:1007400000221146F120FFF71DFF00221146DA209A
:10075000FFF718FF002211461220FFF713FF0022B7
:100760001146DB20FFF70EFF002211464020FFF765
:1007700009FF002211462020FFF704FF0022114646
:100780000220FFF7FFFE002211468D20FFF7FAFE40
:10079000002211461420FFF7F5FE00221146A42086
:1007A000FFF7F0FE00221146A620FFF7EBFE002225
:1007B0001146AF20FFF7E6FE00221146AF20FFF7FB
:1007C000E1FEFFF725FFBDE870400021084607E77E
:1007D0002DE9F041804606980E461F460024203839
:1007E000C5B2B8F17F0F02D9A046B61CF6B20C2AEA
:1007F00006D0102A19D0BDE8F0415FA001F01EBF5D
:10080000761CF1B24046FFF7EBFE604905EB450070
:1008100001EB40053A46285D0121FFF7B3FE641C59
:10082000E4B2062CF6D3BDE8F08131464046FFF72E
:10083000D7FE574800EB05153A46285D0121FFF722
:10084000A1FE641CE4B2082CF6D3761CF1B240463B
:10085000FFF7C6FE002428193A46007A0121FFF767
:1008600091FE641CE4B2082CF5D3DCE72DE9F843D3
:100870000446DDF820800E4691461F46002510E014
:1008800000904B46424631462046FFF7A1FF04EB5D
:100890005800C4B2782C02D90024761CF6B26D1C24
:1008A000EDB2785D0028EBD1BDE8F88308B51021E2
:1008B00040060091010E002236A31046FFF7D6FF36
:1008C00008BD0FB42DE9FE4F0C46934600254FEAB4
:1008D00054088020B0FBF8F64FEA4B07102C1BD0D1
:1008E000042002900DF14409CDF80490701C01F031
:1008F0000DFE82464B46711C5046109A06F090FF42
:100900008146B1450BD90AEB060010F8010C7F288F
:1009100005D9A6F1010905E041200290E2E7B145C1
:1009200000D9B1460C98012802D002280AD105E06E
:10093000A6EB0900400808FB00F503E0A6EB090060
:1009400008FB00F5B9F1000F7DDD5846FFF7AEFF5B
:100950000026A8E01AF806107F2925D80091F9B2E0
:10096000E8B222460F9BFFF733FF05EB540599E0F1
:1009700000002142940122424E6F20204348415200
:10098000484947485F65202E000000007CBE0208F1
:10099000A4C0020820202020202020202020202069
:1009A0002020202000000000002078E0102C02D041
:1009B0000C2C38D072E0C0EBC00202EB8203DA4AA2
:1009C00003EB020898F82020914267D10AEB060257
:1009D00098F8213052789A4260D1F9B2E8B2FFF724
:1009E000FFFD4FF0000B07E018F80B0001210F9AF4
:1009F000FFF7C8FD0BF1010BA345F5D3781CC1B27D
:100A0000E8B2FFF7EDFDA34607E018F80B0001215F
:100A10000F9AFFF7B7FD0BF1010BBBEB440FF4D3BB
:100A20002544761C3EE000EBC00202EB4203BE4AC6
:100A30006C3A03EB020898F8182091422ED10AEB89
:100A40000602527800E032E098F819309A4225D137
:100A5000F9B2E8B2FFF7C4FD4FF0000B07E018F859
:100A60000B0001210F9AFFF78DFD0BF1010BA34540
:100A7000F5D3781CC1B2E8B2FFF7B2FDA34607E098
:100A800018F80B0001210F9AFFF77CFD0BF1010B09
:100A9000BBEB440FF4D32544761C03E0401C029AC0
:100AA000904283D3761C4E45FFF454AF09E008D042
:100AB000B1229EA1A3A006F0CDFEAFF2341006F045
:100AC000C9FE5046BDE8FE0F5DF814EB01F058BDBD
:100AD00000B5002211468D20FFF754FD002211467B
:100AE0001420FFF74FFD00221146AF205DF804EB04
:100AF00048E500B5002211468D20FFF743FD002296
:100B000011461020FFF73EFD00221146AE205DF891
:100B100004EB37E52DE9FF5F80460E9D8B461F46AF
:100B2000002459464046FFF75BFD0BF101090C2DEF
:100B300008D0102D4FD0AFF2C01004B0BDE8F05F68
:100B400001F07CBDDFF8E0A1AAF16C0A3CE06C2268
:100B50001B2300203D1932E000EBC00606EB4606E1
:100B60005644395D96F818C0614527D1697896F8E2
:100B700019C0614522D159464046FFF731FD002595
:100B80000121705D029AFFF7FDFC6D1CEDB20C2D8A
:100B9000F6D309F0FF014046FFF722FD0C250121A5
:100BA000705D029AFFF7EEFC6D1CEDB2182DF6D3C6
:100BB00008F10C0808F0FF08641C04E0401C92FBDC
:100BC000F3F18142C8D8641C384607F05BF9A042B3
:100BD000BDD8BDE8FF9FDFF850A138E000203A5DA6
:100BE0003B19C0EBC00101EB810101EB0A0696F84D
:100BF00020108A4227D1597896F82150A94222D153
:100C000059464046FFF7ECFC00250121705D029A31
:100C1000FFF7B8FC6D1CEDB2102DF6D309F0FF0103
:100C20004046FFF7DDFC10250121705D029AFFF7B9
:100C3000A9FC6D1CEDB2202DF6D308F1100808F0C8
:100C4000FF08641C02E0401C4128CAD3641C3846DB
:100C500007F018F9A042C1D8BBE72DE9F04F814653
:100C6000DDE909BA0E460025580705D0012000EB42
:100C7000D30702EB090815E0DF08FAE731464846DA
:100C8000FFF7AEFC4C4609E028466D1C1AF8000040
:100C90005A460121FFF776FC641CE4B2A045F3D864
:100CA000761CF6B2BE42E9D3BDE8F08F10B586B02F
:100CB0000121080304F0EFFB04220621002002F0CA
:100CC0005DFF18220521002002F058FF182207219D
:100CD000002002F053FF10220421002002F04EFFFA
:100CE0000020ADF804004FF48271ADF80610ADF8A5
:100CF0000800ADF80A00ADF80C004FF40071ADF833
:100D00000E100821ADF81010ADF812000720ADF854
:100D10001400104C01A9204606F0DEFB01212046FC
:100D200006F05FFC06B010BD99B502082E2E5C4897
:100D3000415244574152455C4F4C45445C6F6C6591
:100D4000642E63004C6F674572723A2025732C2520
:100D5000640000000030014010B57E4C204605F0D4
:100D60009BFF2046BDE8104014227B4903F0BDBE26
:100D700070B505F058FF0024784D05EBC42005F050
:100D80008BFF641CE4B2002CF7D073480021416053
:100D9000C160FFF7E1FFBDE8704005F050BF2DE9ED
:100DA000F04105460E464FF40067384601F0AEFBB1
:100DB0008046C6F3CF240BE03A464146284603F06E
:100DC000F1FD3A464146002002F0E7F805F50065DE
:100DD000641EA4B2F0D23946404607F048F9C6F383
:100DE0000A0422464146284603F0DCFD22464146DD
:100DF000002002F0D2F84046BDE8F04101F0C0BB4F
:100E000070B514225449534803F0CCFD524C4FF0B6
:100E1000503000252268011182420ED122698A4297
:100E20000BD121894EA001F0AFFB4C486168FFF760
:100E3000B6FF2581BDE870408EE7206021612581E5
:100E4000BDE8704094E72DE9F84F0546284607F0C5
:100E500019F800287BD0284607F014F814301FFA40
:100E600080F8404601F052FB074600260024464B1E
:100E700046A241463846009506F00EFD80B200F0CD
:100E8000010101EB500505F0CEFE352006F0EFF82C
:100E900010E00A2003F021FC0A2C09D93EA001F041
:100EA000CDFB05F0C0FE3846BDE8F84F01F068BB49
:100EB000641CA4B2012006F0CBF80128E9D0DFF8C9
:100EC0009890DFF898A031E0202006F0D0F8701C50
:100ED00081B2B85D08B940F02D004A1C795C96B229
:100EE00040EA0124200A01D144F43454D9F8040022
:100EF000C8F50061884207D30020C9F80400B9F89A
:100F00000800401CA9F80800D9F804005044410525
:100F100001D105F0C1FED9F804002146504405F086
:100F20008BFFD9F80400801CC9F804006D1EADB217
:100F3000CAD2FFF711FF05F082FE1CA0D9F80410F9
:100F400001F022FB3846BDE8F84F01F019BBBDE8BF
:100F5000F88F000000F00708C41B002000F8070805
:100F6000B1BEB5D8C8D5D6BEB4E6B4A2D2E7B3F602
:100F7000A3BA2564B4CE202E0D0AB1BEB5D8C8D50B
:100F8000D6BE3A20000000004F5B00202A257320C7
:100F900025732A2000000000D0B4466C617368C33A
:100FA000A6B5C8B4FDB3ACCAB1A3A100466C6173C9
:100FB00068C6ABD2C6B3A4B6C83A252378000000F1
:100FC000072813D2DFE800F00406080A0C0E100010
:100FD000E3A07047E4A07047E6A07047E8A0704720
:100FE000EAA07047ECA07047EEA07047F1A07047F0
:100FF0004FF4A071F24807F03AB84FF4A071F148ED
:1010000007F035B870B505460C46EF480078002863
:1010100006D022462946BDE87040EA4806F0C5BE23
:10102000EAA1284601F01AFD002821DBE9A12846A3
:1010300001F014FD00280DDB22462946E94801F0A5
:1010400080FB002830D0BDE870407122E6A1EFA0FF
:1010500001F0F4BA22462946F34801F072FB002859
:1010600022D0BDE870407822DFA1F0A001F0E6BAFE
:10107000D34806F007FFC0F5A070A04205D9294665
:10108000BDE87040CE4806F067BF8422D6A1EEA02E
:1010900001F0D4FAFFF7ACFF2946BDE870404FF4E9
:1010A000A072C74807F02CB870BD0FB42DE9F84FF7
:1010B00082464FF00408C448CAEBCA01001D00EB89
:1010C0008104667E60680B904FF4A165284601F0AC
:1010D0001DFA83460CAB0093294658460B9A06F03E
:1010E0009FFB07464FF00009002F01DDAF423EDDB8
:1010F000B622BDA1DBA001F0A1FA584601F040FAEA
:101100000220BDE8F80F5DF814FBFFF771FF002522
:10111000BAB25946022001F040FF16E0642003F005
:10112000DCFAE168A64801F099FC206120690028FA
:1011300002DB4FF003081DE06169A14801F08EFC5D
:10114000002802DB4FF0020814E028466D1C2189BC
:10115000EDB28842E2D3607E801B00EBC00101EB60
:1011600000104FF4FA7101EB800003F0B6FA761E1E
:10117000F6B2CAD2584601F003FACDF80090B8F1A1
:10118000050F0ED2DFE808F0030507090B00BCA429
:1011900008E0BEA406E0C0A404E0C1A402E0C2A42A
:1011A00000E0C3A45046FFF70BFF01462246C3A050
:1011B00001F018FA4046A4E770B50446002020600C
:1011C000207100210620FFF770FF0546032D05D092
:1011D000BCA1204606F027FE284670BD2C21784889
:1011E00006F045FE411C04230D22204601F059FB68
:1011F000F2E770B505461521284606F038FF0021B4
:101200000520FFF752FF0446032C09D10D216C483D
:1012100006F0C1FD811C14230D22284601F041FB7C
:10122000204670BD10B500210220FFF73EFF0328C5
:1012300008D000210320FFF738FF0021BDE810404F
:10124000022032E710BD002101202EE79F49012036
:101250000860704770B500240425FFF7F7FFFFF71B
:10126000C7FE4FF47A7610E0641CE4B2304603F017
:1012700034FA97A1524801F0F1FB002805DB214622
:1012800094A001F0AFF9032501E0142CECD328461B
:1012900070BD8E490020086040F6B83003F01DBADA
:1012A00010B510220F21042002F068FCFFF7F1FFB7
:1012B00010220B21042002F061FC84490020103927
:1012C000086010BD10B501230C224FF4E13102205B
:1012D00001F02EFDFFF78CFEFFF78FFE414801F075
:1012E00027FA514801F024FAAFF2E721BDE8104097
:1012F000022001F0F1BC70B5FFF7E4FFFFF7D0FF6B
:10130000FFF7A8FFFFF79FFFFFF78CFF04462C486D
:101310003838FFF76EFF2A4A1421383A73A001F0DB
:1013200033F9274823380546FFF746FF294674A0BE
:1013300001F02AF9204670BD10B500210846FFF7DC
:10134000B4FE0446032C02D073A001F077F94FF4E9
:101350007A7003F0C2F9FFF79CFF204610BD000031
:101360005455524E4F46460048414E445348414B17
:10137000450000005155455259434F4E46494700DC
:10138000434C4F534545434F0000000053415645E1
:10139000434F4E4649470000515545525952454C1E
:1013A000455345005155455259564F4C54414745B8
:1013B00000000000CEDEB4CBC3FCC1EE0000000094
:1013C000101C0020501D0020C40100202B51495545
:1013D00052433A002B51495552433A2022726563D9
:1013E00076220000901E00202E2E5C484152445769
:1013F0004152455C4C54455C454332305C65633238
:10140000306D6F64756C652E6300000025732C25AC
:10141000643A735463705175657565207370696CB7
:101420006C6F766572A3A1009622002025732C258F
:10143000643A735572635175657565207370696C94
:101440006C6F766572A3A10025732C25643A6563E1
:1014500032304174427566207370696C6C6F7665CA
:10146000722E200025732C25643A636D64506163ED
:101470006B207370696C6C6F766572A3A1000000BD
:10148000496E506172616D45727200004F75745003
:101490006172616D4572720052554E4552520000A4
:1014A00052554E4F4B00000054494D454F55540086
:1014B000CEB4D6AAB4EDCEF30000000025732025EB
:1014C000730000003335303000000000BC012342BF
:1014D000524459004543323020537461727420578E
:1014E00061697465643A25642053000045433230D5
:1014F00020C8EDBCFEB0E6B1BEA3BA252E2A73000B
:101500004543323020B9A9B5E7B5E7D1B9A3BA252B
:1015100073206D56000000004543323020C8EDB9FD
:10152000D8BBFACAA7B0DCA3ACBCB4BDABB6CFB5D0
:10153000E7B9D8BBFAA3A1000FB42DE9F84F814653
:101540000427F348C9EBC90100EB8104667E60689B
:101550000B90802000F0DAFF82460CAB00938021D4
:1015600050460B9A06F05CF98046B8F1000F02DD98
:10157000B8F1800F2FDD6522E6A1EEA001F05EF844
:1015800002272BE0FFF734FD00251FFA88F25146B1
:10159000022001F002FD14E0642003F09EF8E168EF
:1015A000EB4801F05BFA20612069002801DB03278A
:1015B00014E06169E64801F051FA002801DB0227D6
:1015C0000CE028466D1C2189EDB28842E4D34FF42B
:1015D0007A7003F082F8761EF6B2D3D2504600F04D
:1015E000CFFF00200090052F0ED2DFE807F00305A3
:1015F00007090B00D7A408E0D9A406E0DBA404E0A7
:10160000DCA402E0DDA400E0DEA4484600F05AF9C4
:1016100001462246DEA000F0E5FF3846BDE8F80F9F
:101620005DF814FB02460021DBA3072084E7024695
:101630000021082080E70246002109207CE72DE9EF
:10164000F04104460F46224600210A20FFF774FFAE
:101650000646032E20D1AE4D012C20D0022C25D0E1
:10166000032C2AD0CEA1BA4801F0F8F9C5F8280118
:10167000D5F8280100280EDBD5F82811B4483034FD
:101680000830085CA04206D1D5F82811B0480A30CD
:10169000085C312818D002263046BDE8F081C0A190
:1016A000AB4801F0DBF9C5F82801E1E7BFA1A84884
:1016B00001F0D4F9C5F82801DAE7BFA1A44801F088
:1016C000CDF9C5F82801D3E7D5F82811A048102393
:1016D0000F3001442222384601F0E3F8DCE72DE91F
:1016E000F04104252D2400210120FFF725FF984E0D
:1016F000874F09364FF4FA6815E0404602F0EDFFD7
:1017000000210220FFF718FF0546032D0BD1B86C0E
:10171000002807DDB86C805D312807D0B86C805D8B
:10172000352803D00225641E601CE6D12846B4E7A4
:101730002DE9F04104251E2400210320FFF7FCFEC3
:10174000834E734F0A364FF4FA6818E0404602F0B1
:10175000C4FF00210420FFF7EFFE0546032D0ED144
:10176000D7F88000002809DDD7F88000805D312897
:1017700008D0D7F88000805D352803D00225641E8C
:10178000601CE3D1284688E770B505461921284634
:1017900006F06DFC00210846FFF7CEFE0446032C40
:1017A00009D15B4801696A481923083001440D22B8
:1017B000284601F076F8204670BD10B500210520BE
:1017C000FFF7BAFE032801D07EA010BD504C9C3418
:1017D00020685F4908440D2106F0DDFA0021017000
:1017E00021685B480A30084410BD70B505460020EA
:1017F000286000210620FFF79FFE0446032C0AD133
:101800004348D0F8B81052481923801D01442C22B7
:10181000284601F046F8204670BD2DE9F041054606
:101820000E466D480446FFF7AFFF032809D06BA2B0
:101830003146284606F030F86BA000F0FFFE02208B
:101840002BE7224619216CA000F09EFEFFF747FF10
:101850000446032C09D06DA23146284606F01CF838
:101860006DA000F0EBFE022017E7FFF761FFFFF726
:10187000A4FF01466EA000F087FE5748001F0746F0
:10188000FFF7B3FF3B466EA23146284606F004F848
:101890003A4603216DA000F077FE2046FDE670B5C4
:1018A00005460E462846FFF7BDFE2846FFF7BFFE59
:1018B0000446032C03D131462846FFF7C0FE2046DC
:1018C00070BDB8E610B50B281DD2DFE800F00608A1
:1018D0000A0C0E10121416181A0060A010BD62A097
:1018E00010BD63A010BD64A010BD65A010BD66A0B2
:1018F00010BD69A010BD6BA010BD6DA010BD6FA084
:1019000010BD72A010BD75A000F098FE79A010BDAA
:101910008C0200202E2E5C48415244574152455CB7
:101920004C54455C454332305C656332306E6574BF
:101930002E63000025732C25643A636D6450616347
:101940006B207370696C6C6F766572A3A1000000E8
:10195000101C0020496E506172616D45727200006A
:101960004F7574506172616D4572720052554E45EB
:101970005252000052554E4F4B00000054494D4505
:101980004F555400CEB4D6AAB4EDCEF300000000FB
:101990002573202573000000434D494F540000007B
:1019A0002B51494143543A20310000002B51494109
:1019B00043543A20320000002B51494143543A200D
:1019C00033000000BBF1C8A1CDF8C2E7D0C5CFA25B
:1019D000CAA7B0DC21000000F61B0020C7EBB2E56F
:1019E000C8EB53494DBFA800CEB4BCECB2E2B5BDC4
:1019F00053494DBFA800000053696DBFA849434338
:101A00004944A3BA252E2A730000000053494DBF54
:101A1000A8C7B7B7D100000053494DC7B7B7D1CE5B
:101A2000DEB7A8D7A2B2E1C9CFCDF8C2E700000067
:101A3000CDF8C2E7D0C5CFA2A3BA2573000000003D
:101A4000D0C5BAC5D6CAC1BF3A2573004C5445208B
:101A5000435351A3BA252E2A730000005155455215
:101A6000594943434944000053455443530000003F
:101A700051554552594353005345545053000000AB
:101A8000515545525950530051554552594E4554A0
:101A9000494E464F0000000051554552594353519D
:101AA00000000000434F46434F4E54455854000039
:101AB000414354434F4E544558540000444541431C
:101AC00054434F4E54455854000000005155455260
:101AD00059434F4E5445585400000000454332309E
:101AE00020CEDED0A7654E6574436D644E756D21C2
:101AF00000000000CEDEB4CBC3FCC1EE000000004D
:101B000005280ED2DFE800F0030507090B00D7A077
:101B10007047D9A07047DBA07047DCA07047DDA0FC
:101B20007047DEA0704705280ED2DFE800F00305FD
:101B300007090B00DCA07047DEA07047E0A07047EB
:101B4000E2A07047E4A07047E6A0704770B510208F
:101B500000F0DCFC054629460120FFF770FD032854
:101B600007D029460120FFF79AFE0446032C02D035
:101B700005E0032070BD2946DDA000F005FD2846E4
:101B800000F0FEFC204670BD0FB42DE9F84F8146F1
:101B90004FF00408DA48C9EBC90100EB8104667E06
:101BA00060680B90802000F0B1FC82460CAB009383
:101BB000802150460B9A05F033FE0746002F01DDC9
:101BC000802F2FDDCFA000F039FD4FF002082CE070
:101BD000FFF70EFA0025BAB25146022001F0DDF9F6
:101BE00016E0642002F079FDE168D24800F036FF8B
:101BF00020612069002802DB4FF0030815E06169CD
:101C0000CC4800F02BFF002802DB4FF002080CE06C
:101C100028466D1C2189EDB28842E2D34FF47A70D8
:101C200002F05BFD761EF6B2D2D2504600F0A8FC60
:101C30004046FFF765FF04464846FFF774FF01463C
:101C40002246BDA000F0CEFC4046BDE8F80F5DF88E
:101C500014FB7CB5024600210220FFF795FF0646E3
:101C6000032E2BD1002000900190162000F04EFC96
:101C70000446A34DA96CAF480A30085C2070A96CDB
:101C8000AC481023133001442C22601C00F009FEE4
:101C9000601C06F0F7F8A96C1430A64A052311441D
:101CA00001442C22684600F0FCFD21786B46621C42
:101CB000A3A000F097FC204600F062FC30467CBDFB
:101CC0001CB50446CDE900230B46002122460846F8
:101CD000FFF75AFF03280ED189490B69954A303422
:101CE00009329A5CA24205D10A6992490B31515CD2
:101CF000302900D002201CBD02460021012043E70C
:101D000070B504462078FFF7F7FF03280CD1A38AAB
:101D1000628A2078611CFFF7D3FF0546032D02D1AC
:101D20002078FFF796FF284670BD2DE9F84F06464C
:101D30008A469146B9F1000F0DD00025A84600242F
:101D40000427FFF755F932786D4EB16D4B460220EE
:101D500001F06CF90DE00320BDE8F88F142002F0CB
:101D6000BCFC3E21734806F016F810B14FF0010894
:101D700004E028466D1CEDB24628EFD3B8F1010F00
:101D800010D03846FFF7BCFE04460320FFF7CBFE19
:101D900001466848009077A3224679A000F04EFCE7
:101DA0003846D9E74A465146022001F0F6F830E0BD
:101DB000642002F092FCF16F5E4800F04FFEC6F81E
:101DC0008000D6F8800000280DDB03273846FFF797
:101DD00097FE04460420FFF7A6FE0146224656A0C1
:101DE00000F000FCDCE7D6F88410524800F036FE24
:101DF00000280EDB02273846FFF782FE0446042047
:101E0000FFF791FE01464B4B224660A000F016FC06
:101E1000C6E72046641CB6F87810A4B28842C7D33F
:101E2000BEE770B5054605245BA1284600F016FE06
:101E3000002801DD002416E05CA1284600F00EFE1B
:101E4000002801DD04240EE05DA1284600F006FE16
:101E5000002801DD022406E05EA1284600F0FEFD18
:101E6000002800DD0324204670BD0000496E50614B
:101E700072616D45727200004F7574506172616DD0
:101E80004572720052554E455252000052554E4F07
:101E90004B00000054494D454F555400CEB4D6AACE
:101EA000B4EDCEF3000000004F50454E534F434B6E
:101EB00045540000434C4F5345534F434B4554004A
:101EC0005155455259534F434B4554005443505379
:101ED000454E44434D44000054435053454E444204
:101EE00055460000CEDEB4CBC3FCC1EE00000000BE
:101EF000544350B1BEB5D84950A3BA257300000071
:101F0000C003002054637020636D645061636B20D4
:101F1000D2E7B3F6A3A12D2DD4F6BCD35443505F22
:101F2000434D445041434B5F4C454ECAFDD6B5A18D
:101F3000A3000000101C0020257320257300000062
:101F4000544350204368616E6E616CA3BA256320D0
:101F5000A1A320B7FECEF1C6F74950A3BA2573A1BD
:101F6000A320B7FECEF1C6F7B6CBBFDAA3BA25736E
:101F700000000000CEB4CAD5B5BD223E220000004C
:101F800025732025732025732025730025732025B4
:101F900073202573000000002B51495552433A200D
:101FA00022636C6F73656422000000002B51495559
:101FB00052433A20227064706465616374220000A9
:101FC0002B51495552433A2022696E636F6D696EF9
:101FD000672200002B51495552433A2022696E6313
:101FE0006F6D696E672066756C6C220005280ED2D5
:101FF000DFE800F0030507090B00D5A07047D7A064
:102000007047D9A07047DAA07047DBA07047DCA00A
:102010007047092818D2DFE800F00507090B0D0FFB
:1020200011131500D9A07047DBA07047DDA07047E1
:10203000DFA07047E1A07047E3A07047E4A07047BD
:10204000E6A07047E8A07047EAA070470FB42DE9FA
:10205000F84F81464FF00408E948C9EBC90100EB8D
:102060008104667E60680B904FF49675284600F0F8
:102070004DFA82460CAB0093294650460B9A05F068
:10208000CFFB0746002F01DDAF422EDDDDA000F0C3
:10209000D5FA2DE0FEF7ACFF0025BAB2514602207A
:1020A00000F07BFF16E0322002F017FBE168E14808
:1020B00000F0D4FC20612069002802DB4FF0030807
:1020C00016E06169DB4800F0C9FC002802DB4FF034
:1020D00002080DE028466D1C2189EDB2B0EB410FDE
:1020E000E1D34FF47A7002F0F8FA761EF6B2D1D24C
:1020F000504600F045FA4046FFF778FF0446484650
:10210000FFF787FF01462246CBA000F06BFA40465E
:10211000BDE8F80F5DF814FB10B500210846FFF785
:1021200095FF032809D100210120FFF78FFF032825
:1021300003D1BDE81040002188E710BD70B5102024
:1021400000F0E4F9054629460220FFF778FA032853
:1021500007D029460220FFF7A2FB0446032C02D039
:1021600005E0032070BD2946B5A000F00DFA284611
:1021700000F006FA204670BDF8B50446204605F08A
:1021800081FE0A30064600F0C1F90546B0A3B2A2AE
:1021900031462846009405F07FFB284605F072FE84
:1021A000024600210420FFF751FF0446032C0BD107
:1021B0002A4600210520FFF749FF0446032C03D1DE
:1021C0002946A7A000F0E0F9284600F0D9F92046FA
:1021D000F8BD10B50424FFF79FFF032801D0204667
:1021E00010BDBDE81040A9E72DE9FF4104460F46A8
:1021F0006068FFF7C1FF4FF49676304600F086F92D
:102200000546384605F03EFED4E90131CDE9020726
:10221000CDE9001331462846226805F03DFB024611
:10222000002A01DDB24204DD022491A000F006FA8A
:102230000CE000210620FFF709FF0446032C05D11E
:102240002A4600210720FFF701FF0446284600F038
:1022500097F904B02046BDE8F081002808D0A0F529
:102260000070BD3807D0012808D08EA000F08CB9CE
:1022700092A000F089B998A000F086B99CA000F067
:1022800083B92DE9F04100240426FEF7B6FE9D4FE8
:10229000012038705A4DD5F8E40005F0F3FDD5F86B
:1022A000E41082B2022000F078FE39E0642002F0EF
:1022B00014FA55F8EC1F944800F0D0FB6860686889
:1022C000EC3D002823DBD5F8F0108F480C30085C7B
:1022D000302819D055F8F01F8B482A68401C095C3B
:1022E0006420303941438848801C105C2A683038AB
:1022F00000EB800001EB40018348C01C105C0844E7
:102300000226FFF7AAFF12E000200326F9E7D5F81E
:10231000F410484800F0A2FB002801DB022606E08A
:102320002046641CB5F8E810E4B28842BED3002011
:1023300038703046FFF75AFE04460820FFF769FE62
:10234000014622463CA000F04DF9304683E70000EC
:10235000496E506172616D45727200004F75745024
:102360006172616D4572720052554E4552520000C5
:1023700052554E4F4B00000054494D454F555400A7
:10238000CEB4D6AAB4EDCEF30000000048545450A9
:10239000434F4E5445535400454E524551484541D4
:1023A00044455200434C4F534554494D45000000AD
:1023B000424F44595459504500000000534554556C
:1023C000524C434D440000004854545055524C0068
:1023D000504F5354524551434D440000504F5354B5
:1023E00052455142554600004854545052454144CC
:1023F00000000000CEDEB4CBC3FCC1EE0000000044
:102400004C0400204874747020636D645061636BE9
:1024100020D2E7B3F6A3A12D2DD4F6BCD348545453
:10242000505F434D445041434B5F4C454ECAFDD62F
:10243000B5A1A300101C0020257320257300000007
:1024400048545450B1BEB5D84950A3BA25730000C2
:10245000687474703A2F2F002573257300000000F4
:10246000504F53542055524C3A25732E0000000013
:10247000686561646572426F647942756620D2E76F
:10248000B3F6A3A12D2DD4F6BCD3485454505F43CA
:102490004D445041434B5F4C454ECAFDD6B5A1A3B8
:1024A0000000000048545450285329206F74686578
:1024B00072206572726F722E000000004874747092
:1024C000204F7065726174696F6E20737563636508
:1024D000737366756C2E000048545450285329209D
:1024E000756E6B6E6F776E206572726F722E000064
:1024F000485454502853292074696D656F75742EA3
:1025000000000000C4010020501D002070B50646E8
:102510003146002000F0AEFB0446002000F017FB1F
:1025200005464B2D08D918225AA161A005F092F951
:10253000294663A005F08EF924B13146204605F006
:1025400096FD1BE0202253A159A005F083F92946EE
:1025500063A005F07FF9002000F0E0FA314600208A
:1025600000F088FB04464CB925224AA150A005F092
:1025700071F968A005F06EF904F0BAFE204670BD4E
:102580000146002000F06DBB0FB4F8B507AD009513
:102590004FF400742046FFF7B9FF06465EA22146BD
:1025A000304605F079F90446C4F5007130192B4620
:1025B000069A05F035F9002806DD204482B231463E
:1025C000002000F0EAFC07E0502232A138A005F01C
:1025D00041F950A005F03EF93046FFF7D1FFF8BCB5
:1025E0005DF814FB0FB4F8B507AD00954FF4007417
:1025F0002046FFF78BFF064649A22146304605F0EC
:102600004BF90446C4F5007130192B46069A05F0C3
:1026100007F9002806DD204482B23146002000F090
:10262000BCFC07E06E221BA121A005F013F939A024
:1026300005F010F93046FFF7A3FFD0E70FB4F8B567
:1026400007AD00954FF400742046FFF75FFF064684
:1026500035A22146304605F01FF90446C4F5007145
:1026600030192B46069A05F0DBF8002806DD2044D9
:1026700082B23146002000F090FC07E08B2205A1D9
:102680000BA005F0E7F823A005F0E4F83046FFF7CB
:1026900077FFA4E72E2E5C53595354454D5C535994
:1026A00053504F52545C737973706F72742E630081
:1026B0004C6F674572723A2025732C256400000028
:1026C0000D0AB6AFCCACC4DAB4E6D5BCD3C3D2D114
:1026D000B3ACB9FDA3BA25642525A3A10D0A00005A
:1026E0000D0AC4DAB4E6D5BCD3C3A3BA2564252544
:1026F0002D2DB6AFCCACC4DAB4E6D2E7B3F6A3A1C5
:10270000B3F5CABCBBAFB6AFCCACC4DAB4E6BFD588
:10271000BCE4A3A1000000004C6F674170703A0058
:102720004C6F674465623A004C6F674572723A00BD
:1027300000210180418081804FF48061801D05F07F
:1027400096BC2DE9F0418388161D33444FF4806711
:10275000BB4202D30120BDE8F08145881223841DCD
:102760002B5543885B1CC3F30903438045883423FE
:102770002B5543885B1CC3F30903438000230BE004
:1027800011F8015BB0F802C00CF8045045886D1CCC
:10279000C5F3090545805B1C9342F1DB4288562155
:1027A00011554188491CC1F30901418042887821B3
:1027B00011554188491CC1F3090141808188314488
:1027C00081808188B94209D3FFF7B2FF4322BFA1BC
:1027D000C5A005F03FF8C8A005F03CF80020BAE716
:1027E00070B58388002B08D003889B1CC3F30903B2
:1027F000038000231380831D21E0022070BD148814
:10280000641C14800488E45C01F8014B0488641C97
:10281000C4F30904048014888588AC4203D2048878
:10282000B4F5806F0BD3FFF783FF6622A7A1AEA09C
:1028300005F010F8B0A005F00DF8022070BD048876
:10284000E45C562CDBD10488641CC4F30904044402
:10285000A479782CD3D10188891CC1F309010180A6
:1028600081881288891A091F8180002070BD2DE996
:10287000F04105460C461746284605F003FB064680
:10288000384605F0FFFA3118A14204DB00212A196D
:10289000101A00F8011C39462846BDE8F04105F041
:1028A0005BBB30B5054600205B1E04E02C5498420B
:1028B00004DA401C80B20C5C9442F7D130BD70B594
:1028C0000446084611461D46049E05F064FA024679
:1028D000012006E0231803F8011CB04204D8401C74
:1028E00080B2115CA942F5D170BD30B5002311440E
:1028F000491E18E00C7824090A2C01D2302500E08A
:1029000037252C4400F813400C7804F00F040A2CEF
:1029100001D2302500E037252C4400EB43056C70D4
:102920005B1C9BB2491E9342E4D330BD30B50023FB
:102930001AE0CD5C2C0905F00F053034392C03D991
:10294000E41D00F8134001E000F813403035ECB20C
:10295000392C04D900EB4305E41D6C7002E000EB58
:1029600043056C705B1C9BB29342E2D330BDF0B563
:1029700003460025084600260A2A01D00670F0BD4D
:10298000002B1DD005DA4FF02D0200F8012BC3F10A
:10299000000342F210724FF00A0793FBF2F454EA7C
:1029A000050C06D004F1300500F8015B04FB12337E
:1029B000012592FBF7F2002AEFDC06700846F0BD15
:1029C0003022027046700846F0BDF0B5054600237F
:1029D000002042F210720A26B5FBF2F4E4B254EA87
:1029E000000704D030340746401CC0B2CC55B5FBBC
:1029F000F2F402FB1455B2FBF6F25B1CDBB2052BC2
:102A0000EAD308B9302008700846F0BD2DE9F0413E
:102A100005460C46284605F035FA80B2002100B183
:102A200021700122002312E0AE5CEF5CBE420CD1AB
:102A3000521C92B25B1C9BB2AE5CEF5CBE4201D0FA
:102A4000A35404E0E65CA65401E01BB1E35C8242BF
:102A5000EAD380E6521C92B2A154F8E72DE9F04780
:102A600082468946504605F00DFA87B2484605F081
:102A700009FA86B2002500243046FFF747FD80465C
:102A800041464846FFF7C2FF0DE01AF8050019F865
:102A90000410884204D16D1CADB2641CA4B202E0E3
:102AA0006CB118F80440BD4201D2B442EDD34046A7
:102AB000FFF766FDB44205D3A81BBDE8F0876D1C87
:102AC000ADB2F0E74FF0FF30F7E700002E2E5C5379
:102AD000595354454D5C5359534C49425C73797377
:102AE0006C69622E630000004C6F674572723A2079
:102AF00025732C25640000000000000003E011F89D
:102B0000013B00F8013B521E531CF8D1704701E015
:102B100000F8011B521E531CFAD1704770B50446D1
:102B20006B486C4E002150F8240006EB84054200EF
:102B30002869FFF7ECFF66480021103050F8242088
:102B4000A868FFF7E4FF01203119087670BD10B5C1
:102B5000002200215E4B5F4C53F8203004EB8000D4
:102B600005E0046934F8114004B1521C491C8B4241
:102B7000F7D864204243B2FBF3F0C0B210BD2DE998
:102B8000F04105460F460024DFF8488108EB0500B8
:102B9000007E002803D1D8F80010284688474FF05F
:102BA000FF32FFB14A4E083656F82500B7FBF0F366
:102BB000B7FBF0F100FB117000B15B1C444850F80A
:102BC0002510491E002921DB08EB8507386930F8FC
:102BD00011C0BCF1000F08D000249C4213D1002288
:102BE00098B20AE01046BDE8F081641CF5E73C6944
:102BF00001EB020C24F81C00521C9A42F7D356F841
:102C000025004843EFE7491E0029E0DA1046EAE7CD
:102C100070B5304A13181B7E002B13D02C4B103389
:102C200053F820308B421AD9294B083353F82030FF
:102C3000B1FBF3F102EB8002106930F81130002093
:102C4000002408E011688847012070BD15690E183E
:102C500025F81640401C9842F8DB002070BD022089
:102C600070BD002905D01B4A02EB80029268891AC8
:102C7000CEE7704710B504462046FFF780FF411CA1
:102C800005D0144901EB84018968084410BD002077
:102C900010BD2DE9F04106468846174639463046B4
:102CA000FFF76DFF0446601C0FD00A483A4600EB60
:102CB00086054146A8682044FFF720FF414630467C
:102CC000FFF7CFFFA86820448DE700208BE70000C6
:102CD00094C602084805002010B50C46F24A52F886
:102CE0002030002B09D05222F0A1F6A004F0B2FD52
:102CF000F8A004F0AFFD204610BD42F82040FAE7EE
:102D000030B40C46E84951F82030002B03D020465F
:102D100030BC1146184730BC704770477047F449C3
:102D2000C2B20B689A8009680A885206FCD57047BF
:102D30002DE9F04387B004460D461646984601211A
:102D4000084602F0A8FBEA4818220F38015D401F30
:102D5000005D00F013FFE6480422401F015D401FA4
:102D6000005D00F00BFFE348002C7CD050F82400FD
:102D7000012102F09BFB02950025ADF80C50ADF847
:102D80000E50ADF81050ADF81450ADF81260D84E9A
:102D900002A956F8240002F01DFC56F824004FF456
:102DA000587102F067FDBDF8120006F11409000722
:102DB00022D5042C20D056F824000122802102F0D4
:102DC000ABFCCC4F00950195183F59F82410385DA5
:102DD0001023002200F02BFC06F12400002150F803
:102DE0002420385D00F01CFBAF480121303850F83A
:102DF0002420385D00F014FBBDF81200400759D5BF
:102E0000BC481038005D8DF818008DF819808DF8D9
:102E10001A5001208DF81B0006A802F076F856F82B
:102E20002400012240F2244102F05BFC042C3BD040
:102E300056F824000122402102F06EFCCDE9005832
:102E4000AC4859F824101430A0F1280550F824207B
:102E5000285D002300F0EBFB05F10A00A64F30F8D7
:102E60001410285D00E01AE057F8200004F0D0F9B3
:102E70008D480021203850F82420285D00F0D0FA39
:102E800089480121103850F82420285D00F0C8FA44
:102E9000285D012157F8200004F0A3F90AE000683A
:102EA000012102F0F8FA66E7012240F2255130696B
:102EB00002F017FC56F82400012102F006FC07B0CE
:102EC000BDE8F0831CB5044689480122802150F8F2
:102ED000240002F021FC06200021CDE900108448E6
:102EE00010231430002250F8241082481838005D56
:102EF00000F09DFB1CBD7CB504467D4801224021AD
:102F000050F8240002F008FC06200021CDE9001052
:102F10007848784D1430143D50F82420744800232C
:102F2000143050F82410285D00F081FB05F10A00F0
:102F3000714E30F81410285D56F8200004F068F93E
:102F4000285D012156F82000BDE87C4004F049B915
:102F50002DE9F0410446674D674E143D0021285D80
:102F600056F8200004F03DF905F10A0705F12800A4
:102F700037F8141050F8240005F079F8285D37F878
:102F8000141056F8200004F043F9285D012156F88A
:102F90002000BDE8F04104F024B92DE9F0470446D3
:102FA00088461646B8F1000F25D0002E23D0042CF9
:102FB00023D0504FDFF84091183F0021385D59F879
:102FC000200004F00EF94A4D0020183D2855385DC8
:102FD00059F82000C0F80C80385D314659F82000BF
:102FE00004F016F9385D012159F8200004F0F9F8D1
:102FF000285D0028FCD0BDE8F08700253C4F40212B
:10300000386902F030FC0EE018F8051057F824007B
:1030100002F0BCFB57F82400402102F024FC0028F9
:10302000F8D06D1CADB2B542EED3E4E70FB470B585
:1030300086B004460CA801902D4E10E05C2916D0F5
:1030400025295BD0401C0B9056F8240002F09EFB13
:1030500056F82400402102F006FC0028F8D00B9816
:1030600001780029EAD106B070BC5DF814FB401C61
:103070000B9001786E290DD0722902D0401C0B9064
:10308000E6E756F824000D2102F080FB0B98401C67
:103090000B90DDE756F824000A2102F077FB0B982D
:1030A000401C0B90D4E70000905500202E2E5C535E
:1030B000595354454D5C55534152545C757361727C
:1030C000742E63004C6F674572723A2025732C256D
:1030D00064000000556172742043616C6C6261632E
:1030E0006B20726570656174207265672100000055
:1030F00080050020C4C60208B8050020401C0B90C3
:10310000017864291BD0732902D0401C0B909FE7E3
:10311000019820C801900BE056F8240002F036FB1D
:1031200056F82400402102F09EFB0028F8D06D1CC8
:1031300029780029F0D10B98401C0B9088E7019862
:1031400001990068091D01910A2202A9FFF70FFCED
:1031500002AD0BE056F8240002F018FB56F82400EC
:10316000402102F080FB0028F8D06D1C297800294E
:10317000F0D10B98401C0B906AE770B59C4C40F264
:103180002441204602F07AFBA0B19A4D0021286923
:1031900004F027F82088201D0088286904F03AF8F8
:1031A000C0F5807082B294490020FFF7A9FD00208D
:1031B000FFF7CEFE40F225552946204602F05EFB81
:1031C00018B12946204602F079FB40F227752946BE
:1031D000204602F053FB002806D029462046BDE8D1
:1031E0007040002202F07DBA70BD70B5834C40F291
:1031F0002441204602F042FBA0B17E4D00216869C7
:1032000003F0EFFF2088201D0088686904F002F8B1
:10321000C0F5807082B27A490120FFF771FD01206C
:10322000FFF796FE40F225552946204602F026FB80
:1032300018B12946204602F041FB40F22775294685
:10324000204602F01BFB002806D029462046BDE898
:103250007040002202F045BA70BD70B5694C40F272
:103260002441204602F00AFBA0B1624D0021A8686B
:1032700003F0B7FF2088201D0088A86803F0CAFF6C
:10328000C0F5807082B260490220FFF739FD02204C
:10329000FFF75EFE40F225552946204602F0EEFA81
:1032A00018B12946204602F009FB40F2277529464D
:1032B000204602F0E3FA002806D029462046BDE861
:1032C0007040002202F00DBA70BD70B54F4C40F254
:1032D0002441204602F0D2FAA0B1464D0021686A8E
:1032E00003F07FFF2088201D0088686A03F092FFAA
:1032F000C0F5807082B246490320FFF701FD03202C
:10330000FFF726FE40F225552946204602F0B6FA80
:1033100018B12946204602F0D1FA40F22775294615
:10332000204602F0ABFA20B100222946204602F0E6
:10333000D8F92046BDE87040402102F09BBA2DE943
:10334000F041344D40F22551284602F097FA324CB4
:10335000002658B1AA882168481C20602F48425492
:10336000216846542068FF2800DB266040F224478D
:103370003946284602F082FA88B12888A888206851
:10338000264982B20420FFF7BBFC4FF4807123482A
:1033900004F08FFE26603946284602F08FFA40F28C
:1033A00027742146284602F069FA002806D02146F3
:1033B0002846BDE8F041002202F093B9BDE8F08153
:1033C00015490120091D0870704713490120091D86
:1033D0004870704710490120091D887070470E49D8
:1033E0000120091DC87070477047704770477047CB
:1033F00000380140B8050020A455002000440040DA
:10340000A456002000480040A4570020004C004073
:10341000A45800200050004064050020A45900205A
:1034200010B5144600290BD0012919D04E22E9A16C
:10343000EDA004F00FFAF0A004F00CFA204610BD45
:10344000F64951F8202042B14322E2A1E6A004F05F
:1034500001FAF3A004F0FEF9F0E741F82040EDE7AF
:10346000EE49303151F8202042B14A22D9A1DEA0E4
:1034700004F0F0F9F1A004F0EDF9DFE741F82040A5
:10348000DCE730B4E549B0F1007F01F1300271D0E2
:1034900036DCB0F5005F6ED018DC80287AD00ADC0C
:1034A00002286DD0082870D0202868D148680028EC
:1034B00065D030BC0047B0F5007F71D0B0F5006F2B
:1034C0005DD1906800285AD030BC0047B0F5002F7D
:1034D00077D00ADCB0F5004F6ED0B0F5003F4ED18A
:1034E000086900284BD030BC0047B0F5001F6DD0F4
:1034F000B0F5000F43D15069002840D030BC0047E0
:10350000D54C031BA0427CD01ADCD44CA0EB0403A6
:10351000A0426CD00BDCB0F1006F61D0A0F1805004
:10352000801E2CD1C86900287FD030BC0047182BE2
:1035300062D0782B79D1106A002876D030BC004751
:10354000B3F5FC4F67D00ADCB3F5C06F5ED0B3F5BE
:10355000F05F6AD1886A002867D030BC0047B3F5B5
:10356000FF3F5DD0BE48C3425FD1D06A00285CD027
:1035700030BC00472FE018E00CE001E005E054E02B
:103580000868002851D030BC0047106800284CD093
:1035900030BC00475068002847D030BC0047FFE7E8
:1035A0008868002841D030BC0047C86800283CD05B
:1035B00030BC004705E0FFE7D068002835D030BCBC
:1035C00000471069002830D030BC00474869002807
:1035D0002BD030BC00478869002826D030BC00477B
:1035E0009069002821D030BC00470AE0FFE7D0698D
:1035F00000281AD030BC0047086A002815D030BC1B
:103600000047486A002810D030BC0047506A0028A4
:103610000BD030BC0047906A002806D030BC004771
:10362000C86A002801D030BC004730BC70472DE983
:10363000F0478CB00446DDE914980D4617469A46CB
:10364000072C04D20121084601F01AFF03E00121F2
:10365000022001F015FF834E56F8240003F020FDF0
:1036600001950297CDF80CA00025049505958020C2
:10367000069007950895CDF8249040010A900B9587
:1036800056F8240001A903F082FD774810F82400C1
:103690008DF800008DF801808DF8025001208DF822
:1036A0000300684601F031FC56F824000122022193
:1036B00003F0A4FD0CB0BDE8F08710B5022003F0C4
:1036C000ACFD012805D1022003F0CFFD0220FFF759
:1036D000D8FE082003F0A1FD01280ED1082003F038
:1036E000C4FDD5223BA140A004F0B4F85FA004F0D3
:1036F000B1F8BDE810400820C3E610BD10B5202089
:1037000003F08BFD012805D1202003F0AEFD202021
:10371000FFF7B7FE802003F080FD01280ED1802046
:1037200003F0A3FDEB222BA12FA004F093F852A0ED
:1037300004F090F8BDE810408020A2E610BD10B55E
:103740004FF40074204603F068FD012805D120469F
:1037500003F08BFD2046FFF794FE4FF400642046F3
:1037600003F05BFD01280FD1204603F07EFD40F2FF
:10377000011218A11CA004F06DF842A004F06AF830
:103780002046BDE810407CE610BD10B54FF4005453
:10379000204603F042FD012805D1204603F065FDD7
:1037A0002046FFF76EFE4FF40044204603F035FD3F
:1037B000012874D1204603F058FD40F2171205A1EC
:1037C00009A004F047F832A004F044F82046BDE810
:1037D000104056E62E2E5C53595354454D5C444DD3
:1037E000415C646D612E63004C6F674572723A20D4
:1037F00025732C2564000000446D615465204361ED
:103800006C6C6261636B20226549727154797065DA
:1038100022206572726F722100000000A45A0020FD
:10382000446D6154632043616C6C6261636B207210
:10383000657065617420726567210000446D615494
:10384000652043616C6C6261636B207265706561B9
:10385000742072656721000000020010080000104B
:103860000002F8FFB8050020E8C60208444D4131C7
:103870005F54453121000000444D41315F544532D1
:1038800021000000444D41315F54453321000000C8
:10389000444D41315F54453421000000FFE710BD25
:1038A00010B54FF40034204603F0B7FC012805D1D1
:1038B000204603F0DAFC2046FFF7E3FD4FF4002436
:1038C000204603F0AAFC012811D1204603F0CDFCCC
:1038D00040F22D12AFF20411AFF2F40003F0BAFF80
:1038E0008AA003F0B7FF2046BDE81040C9E510BD2F
:1038F00010B54FF40014204603F08FFC012805D1C9
:10390000204603F0B2FC2046FFF7BBFD4FF4000455
:10391000204603F082FC012811D1204603F0A5FCCB
:1039200040F24312AFF25411AFF2441003F092FF91
:1039300079A003F08FFF2046BDE81040A1E510BD3F
:1039400010B54FF00074204603F067FC012805D144
:10395000204603F08AFC2046FFF793FD4FF00064F9
:10396000204603F05AFC012811D1204603F07DFCCB
:1039700040F25912AFF2A411AFF2941003F06AFFB3
:1039800068A003F067FF2046BDE8104079E510BD50
:1039900010B5674C204603F040FC012805D12046B5
:1039A00003F063FC2046FFF76CFD614CA41D20462C
:1039B00003F033FC012811D1204603F056FC40F2FD
:1039C0006F12AFF2F011AFF2E01003F043FF59A015
:1039D00003F040FF2046BDE8104052E510BD10B591
:1039E000534C1E34204603F018FC012805D1204614
:1039F00003F03BFC2046FFF744FD4D4C7E3420464F
:103A000003F00BFC012811D1204603F02EFC40F2FC
:103A10008512AFF24021AFF2302003F01BFF45A02A
:103A200003F018FF2046BDE810402AE510BD10B590
:103A3000434C204603F0F1FB012805D1204603F05A
:103A400014FC2046FFF71DFD3E4C204603F0E5FB2D
:103A5000012811D1204603F008FC40F29B12AFF27E
:103A60008C21AFF27C2003F0F5FE37A003F0F2FECC
:103A70002046BDE8104004E510BD10B5354C204689
:103A800003F0CBFB012805D1204603F0EEFB2046D6
:103A9000FFF7F7FC304C204603F0BFFB012810D1A4
:103AA000204603F0E2FB40F2B112AFF2D821AFF2B0
:103AB000C82003F0CFFE29A003F0CCFE2046FFF77C
:103AC000E0FC294C204603F0A8FB012805D1204644
:103AD00003F0CBFB2046FFF7D4FC244C204603F038
:103AE0009CFB012811D1204603F0BFFB4FF4DF728D
:103AF000AFF22031AFF2103003F0ACFE1CA003F0A7
:103B0000A9FE2046BDE81040BBE410BD444D413144
:103B10005F54453521000000444D41315F54453626
:103B200021000000444D41315F5445372100000021
:103B300002000010444D41325F5445322100000024
:103B40000002001000080010444D41325F5445331C
:103B5000210000000020001000800010444D413280
:103B60005F544534210000000000021000000810DE
:103B7000444D41325F54453521000000F8B50446FC
:103B80000D4616469848012150F8240001F083FCA8
:103B900095481C3030F81500ADF800008DF8036032
:103BA00003208DF802009148694650F8240001F086
:103BB0006CFAF8BD2DE9FE430646DDF828900C4668
:103BC000154698462A4621463046FFF7D7FF282D4E
:103BD00001D0482D36D10121084601F05CFC824F0E
:103BE0008C37385D8DF800008DF8019000258DF838
:103BF00002508DF80350684601F087F9A7F1500094
:103C0000015D4438805D01F0FCFAA7F1400656F8EA
:103C1000240001908DF808508DF8098001258DF859
:103C20000A5001A802F09AF856F8240002F0F5F8BC
:103C3000385700F01F018D404009800000F1E0205E
:103C4000C0F80051BDE8FE83684A52F82000C268FF
:103C5000654B1C3333F811104A40C260704710B5F1
:103C60000C46634A52F82030002B09D0952261A1FE
:103C700065A003F0EFFD68A003F0ECFD204610BD49
:103C800042F82040FAE770B5064600204FF0804128
:103C900005F0F8FD04460D46304606F0A3FF05F09A
:103CA000F1FD22462B4606F095FD06F027FF504910
:103CB00051F82000002802D0BDE87040004770BDD8
:103CC00010B5012002F08EF828B1012002F093F81F
:103CD0000120FFF7D8FFBDE81040012002F09DB899
:103CE00010B5022002F07EF8012805D1022002F072
:103CF00082F80220FFF7C7FFBDE81040022002F063
:103D00008CB810B5042002F06DF828B1042002F040
:103D100072F80420FFF7B7FFBDE81040042002F05E
:103D20007CB810B5082002F05DF8012805D1082004
:103D300002F061F80820FFF7A6FFBDE81040082058
:103D400002F06BB810B5102002F04CF828B110202A
:103D500002F051F81020FFF796FFBDE81040102048
:103D600002F05BB830B591B005241F4D4C3555F8C5
:103D7000240002F044F888B155F8240002F03BF822
:103D8000402101A804F095F9234629A2402101A869
:103D900003F082FD55F82400FFF775FF641C092C21
:103DA000E5DD11B030BD30B591B00A240E4D4C3573
:103DB00055F8240002F023F888B155F8240002F0E9
:103DC0001AF8402101A804F074F9234618A24021F2
:103DD00001A803F061FD55F82400FFF754FF641CAF
:103DE0000F2CE5DDDDE7000020C70208E805002014
:103DF000045B00202E2E5C53595354454D5C494FB3
:103E00005C696F2E630000004C6F674572723A2048
:103E100025732C2564000000494F2043616C6C62BF
:103E200061636B2072657065617420726567210043
:103E30004558544925642049525121000021016010
:103E40004160018181720B2210A104F059B90EB5B5
:103E5000114A12680092104A121D126801920E4A0D
:103E600008321268029200290BD0012904D00C22DA
:103E70006946FEF75BFD0EBD0C226946FEF756FD56
:103E80000EBD0C22694604F03BF90EBD4E6F762044
:103E90003237203230323000E8F7FF1F10B50C46C1
:103EA000F54901280BD0022816D03D22F3A1F8A035
:103EB00003F0D0FCFAA003F0CDFC204610BD48680A
:103EC00040B13222EDA1F2A003F0C4FCFBA003F04C
:103ED000C1FCF2E74C60F0E7886840B13922E7A105
:103EE000EBA003F0B7FCFDA003F0B4FCE5E78C60A9
:103EF000E3E7E149012805D0022807D188680028B6
:103F000004D000474868002800D00047704710B52B
:103F1000012002F042F838B1012002F04CF802F022
:103F20001DF80120FFF7E5FF022002F036F8002817
:103F300008D0022002F03FF802F010F8BDE810406F
:103F40000220D6E710BD10B5022002F026F80028A6
:103F50000CD04FF4003001F060FF022002F02BF88B
:103F600001F0FCFFBDE810400220C2E710BD30B5F3
:103F70006423B0FBF3F4E4B2B0FBF3F503FB1500EC
:103F8000132C01D96430C0B200EB90030724B3FBBB
:103F9000F4F504FB1533D94D1A440D4415F8015CB2
:103FA0002A4492B2800703D1032901D2521E92B251
:103FB000B2FBF4F004FB102030BD810701D00020DB
:103FC00070476421B0FBF1F201FB120109B101203D
:103FD00070474FF4C871B0FBF1F201FB120008B159
:103FE00000207047012070472DE9F04788B0044653
:103FF00001F0BAFF01F089FF0646DFF80483B6FB43
:10400000F8F39D480A270188994279D0038040F24D
:10401000B2754FF4B7794FF4B67A0FE02846FFF740
:10402000CCFF38B14B4502D3A3F5B77304E06D1C48
:10403000ADB205E0A3F26D136D1CADB25345EDD8E2
:104040000195BDF804104FF47A70B1FBF0F13031F6
:104050002170BDF80410B1FBF0F200FB12126421D4
:10406000B2FBF1F230326270BDF80420B2FBF0F521
:1040700000FB1520B0FBF1F201FB1200B0FBF7F0E2
:104080003030A070BDF80400B0FBF7F107FB110061
:104090003030E0700025DFF8649209F10C090DE082
:1040A000BDF80400FFF789FF08B1012D7AD019F897
:1040B0000500984204D81B1A6D1CADB21C2BEFD220
:1040C0006D1C04955B1C03939DF81000B0FBF7F08A
:1040D000303060719DF81000B0FBF7F107FB110064
:1040E0003030A0719DF80C00B0FBF7F0303020723A
:1040F0009DF80C00B0FBF7F107FB11003030607247
:10410000B6FBF8F008FB10604FF46161B0FBF1F210
:104110000792B0FBF1F201FB12033C22B3FBF2F376
:104120000693B0FBF1F301FB1300B0FBF2F102FBCD
:10413000110005909DF81C00B0FBF7F03030E072E4
:104140009DF81C00B0FBF7F107FB11003030207325
:104150009DF81800B0FBF7F03030A0739DF8180000
:10416000B0FBF7F107FB11003030E0739DF814004D
:10417000B0FBF7F0303060749DF81400B0FBF7F13D
:1041800007FB11003030A0749DF80C209DF8101032
:10419000BDF80400FFF7EBFE029008B00320BDE875
:1041A000F087FFE71D2B8BD31D3B85E755481BE7A9
:1041B00008B503218DF800108DF8010000208DF85E
:1041C000020001208DF80300684600F09EFE08BD45
:1041D0002DE9F041074600244A48202181722D2113
:1041E000C17101713A210174417301214FF0C05036
:1041F00001F05CF90121084601F04DF9012001F0C0
:1042000021FE042001F078FD45F25006B04232D084
:1042100001F048FD012001F0C8F801F068FE01F04E
:104220009DFE6FF07F4500E0641C412001F042F8E4
:1042300008B9AC42F8D3DFF8D080444505D24FF43A
:10424000807001F0C7F8012466E00024012001F02D
:10425000BEF800E0641C612001F02CF808B9AC4203
:10426000F8D3444570D24FF4007001F0B3F8CA227D
:1042700002A107A04AE079E0040600202E2E5C533C
:10428000595354454D5C5254435C7274632E630021
:104290004C6F674572723A2025732C25640000002C
:1042A0005274635F526567486F6F6B43616C6C62F9
:1042B00061636B204661696C656421005274632000
:1042C00053656354692043616C6C6261636B207257
:1042D0006570656174207265672100005274632007
:1042E000416C7254692043616C6C6261636B207233
:1042F000657065617420726567210000BCC70208A3
:1043000080510100445B0020F0FFFF0003F0A2FA9F
:10431000C9A003F09FFA0024012001F060F801F029
:104320001DFEF4B147F6FF7001F0FFFD01F016FE2F
:1043300001F014FE01F0E2FD01F010FE3146042010
:1043400001F0D2FC18E0FFE7CF22AFF2D001AFF2CC
:10435000C00003F07FFAB8A003F07CFA0220BDE8A9
:10436000F08149F6404001F0E0FDDFE701F0F6FDA5
:104370000121084601F0B0FD01F0F0FD01210846E1
:1043800001F0AAFD01F0EAFD0121022001F0A4FDE7
:1043900001F0E4FD002001F055FD3846FFF708FF6D
:1043A000A648FFF721FEAFF2FB110120FFF776FDD3
:1043B0000320D4E72DE9F05F00230178C27830397B
:1043C00001EB4104C4EBC11102EBC104427864214A
:1043D000303A4A438178303901EB810102EB4101E7
:1043E000214430398DB241798279303901EB810431
:1043F0006FF02F0101EB44042244D7B2027A447AD1
:10440000303A02EB820201EB42022244D6B2C27A77
:10441000047B303A02EB820201EB4202224402F0BA
:10442000FF08827BC47B303A02EB820201EB42023E
:10443000224402F0FF09827C407C303800EB80008F
:1044400001EB4000104400F0FF0AA5F2B270822890
:1044500002D30220BDE8F09F40F2B274DFF8E0B171
:1044600009E02046FFF7A9FD08B15B4401E075486B
:104470000344641CA4B2AC42F3D37F1EFFB20024F9
:10448000DFF8C4B110E01BF8040040F2A321484358
:1044900003EBC0132846FFF790FD18B1012C01D1A2
:1044A0006A480344641CA4B2BC42ECD3761E40F2BA
:1044B000A320464303EBC610C8EB4811C1EB08210B
:1044C00000EB0110C9EB091100EB810000EB0A04BD
:1044D000012001F0B7FC01F00AFD01F03FFD20468C
:1044E00001F01CFD01F03AFD01F008FD01F036FD80
:1044F0000320AFE72DE9F05F00230178C27830395F
:1045000001EB4104C4EBC11102EBC1044278642108
:10451000303A4A438178303901EB810102EB4101A5
:10452000214430398DB241798279303901EB8104EF
:104530006FF02F0101EB44042244D7B2027A447A8F
:10454000303A02EB820201EB42022244D6B2C27A36
:10455000047B303A02EB820201EB4202224402F079
:10456000FF08827BC47B303A02EB820201EB4202FD
:10457000224402F0FF09827C407C303800EB80004E
:1045800001EB4000104400F0FF0AA5F2B27082284F
:1045900001D302205EE740F2B274DFF8A4B009E074
:1045A0002046FFF70AFD08B15B4401E025480344BB
:1045B000641CA4B2AC42F3D37F1EFFB20024DFF828
:1045C00088B010E01BF8040040F2A321484303EB3D
:1045D000C0132846FFF7F1FC18B1012C01D11B488C
:1045E0000344641CA4B2BC42ECD3761E40F2A32068
:1045F000464303EBC610C8EB4811C1EB082100EBA2
:104600000110C9EB091100EB810000EB0A04012045
:1046100001F018FC01F06BFC01F0A0FC204601F059
:104620008CFC01F09BFC01F069FC01F097FC002080
:1046300001F008FC03200DE700000000445B0020AF
:104640000085E2018033E101C8C702088051010002
:10465000704710B5042000F09BFC27482749284AE2
:104660000068B0FBF1F31370B0FBF1F142F210708F
:1046700041430A2050804FF0E020026942F00202DC
:1046800002614161016941F00101016110BD70B534
:1046900005461C48854208D905464A221AA121A090
:1046A00003F0D8F823A003F0D5F800214FF0E0265E
:1046B0007469134800784543B369B2699A42FCD0E3
:1046C00003D2A3EB0200014403E0A4EB0200184470
:1046D00001441346A942F0D370BD70B505460024CD
:1046E0004FF47A7605E000F05BF93046FFF7CFFF34
:1046F000641CAC42F7D370BD4006002040420F005E
:1047000010060020E3388E032E2E5C535953544577
:104710004D5C5359535449434B5C737973746963CB
:104720006B2E63004C6F674572723A2025732C25FF
:10473000640000000000000010B50C46794A52F8F1
:104740002030002B09D0342277A17DA003F082F81D
:104750007FA003F07FF8204610BD42F82040FAE722
:10476000704951F82000002800D0004770472DE91B
:10477000FF4104460F4615461E4641F699108742F2
:1047800008D907465E2268A16DA003F063F870A007
:1047900003F060F86F48012150F8240000F086FE15
:1047A0006C480838005D8DF80C008DF80D50002520
:1047B0008DF80E5001208DF80F0003A800F0A5FB26
:1047C00041F61F40ADF80000ADF80650ADF80250BC
:1047D000384606F007FA604A604B05F0FBFF0022FE
:1047E0005F4B06F075FC06F0B9F9ADF804008DF8E2
:1047F00008505C4D694655F8240001F0CDFC0122BB
:1048000055F82400114601F0B2FF55F82400314656
:1048100001F093FF55F82400012102F0E7F9BDE80B
:10482000FF81504951F82000002102F0A7B970B56E
:1048300004464C4D002155F8240002F09FF955F82C
:104840002400BDE87040012101F077BF454951F8CF
:104850002000002101F071BF10B501218C07204616
:1048600002F0B8F9012807D10121204602F0BEF973
:10487000BDE81040002073E710BD10B53A4C01218F
:10488000204602F0A7F9012807D10121204602F0B5
:10489000ADF9BDE81040012062E710BD10B5334C02
:1048A0000121204602F096F9012807D10121204676
:1048B00002F09CF9BDE81040022051E710BD10B590
:1048C0002B4C0121204602F085F9012807D1012156
:1048D000204602F08BF9BDE81040032040E710BDF0
:1048E00010B5244C0121204602F074F9012807D1AB
:1048F0000121204602F07AF9BDE8104004202FE79C
:1049000010BD10B51C4C0121204602F063F90128AE
:1049100007D10121204602F069F9BDE810400520C9
:104920001EE710BD585B00202E2E5C535953544592
:104930004D5C54494D45525C74696D65722E63003F
:104940004C6F674572723A2025732C256400000075
:1049500000000000DCC702089A9999999999B93F1B
:104960000000F03F14060020000400400008004052
:10497000000C0040001000400014004010B545F24B
:10498000555001F071F9062001F071F940F20D3037
:1049900001F070F901F071F9BDE8104001F072B951
:1049A00001F06BB903E010F8013B01F8013B521E26
:1049B00092B2F8D270472DE9F04105460E461746EF
:1049C000002407E0284602F035FA26F81400AD1C52
:1049D000641CA4B2BC42F5D3BDE8F0812DE9F041DE
:1049E0000E4617460546002409E036F814102846FE
:1049F00002F022FA0428EFD1AD1C641CA4B2BC4220
:104A0000F3D3E9E72DE9F04FADF6040D82460F46EA
:104A10001546AAF10064B4F1005F04D300200DF63E
:104A2000040DBDE8F08F212000F044FC012809D0DE
:104A30006B22A3A1A8A002F00DFFABA002F00AFF19
:104A40000220ECE702F0EFF84FEAD428C4F349065D
:104A5000C6F58064A54200D82C460DF1040B37E062
:104A600032183BF812208A4203D1401C80B2A04287
:104A7000F6D3A04214D2484602F00EF9002006E018
:104A8000821937F810102BF81210401C80B2A04287
:104A9000F6D348464FF4806201A9FFF79FFF04E078
:104AA000224639465046FFF799FFA54203D102F04E
:104AB000C6F80320B3E708F10108002607EB440716
:104AC000A244281B85B24FF48064A54200D82C462E
:104AD0004FF0006000EBC829421401A94846FFF7D7
:104AE0006AFF00204FF6FF71C1E72DE9F04107464C
:104AF0000E46002402F0010000EB5205212000F0D8
:104B0000D9FB012809D0A8226DA173A002F0A2FE52
:104B100075A002F09FFE02205EE702F084F8A7F184
:104B20000060B0F5002F01D278050BD0AE2264A151
:104B300069A002F08FFE6CA002F08CFE02F07FF8FC
:104B4000022049E7B5F5006F0BD9B4225CA162A041
:104B500002F080FE64A002F07DFE02F070F80220F8
:104B60003AE7352002F083FA384602F095F8042837
:104B70001BD0BB2252A158A002F06CFE5AA002F03A
:104B800069FE12E00A20FFF7A8FD0A2C0BD9C22209
:104B90004BA151A002F05EFE53A002F05BFE02F0BA
:104BA00042F8022018E7641CA4B2012002F050FA77
:104BB0000128E7D023E0202002F059FA30787178FC
:104BC000B61C40EA0121384602F036F9002410E014
:104BD0000A20FFF782FD1E2C09D9D32238A13EA05E
:104BE00002F038FE40A002F035FE0220F4E6641C1C
:104BF000A4B2202002F02CFA0128E9D1BF1C6D1EBE
:104C0000ADB2D8D202F01BF80320E5E62DE9F0475B
:104C10008146884600260024002702F0010000EBB0
:104C20005205212000F046FB01280AD0F12224A1E0
:104C300029A002F00FFE2CA002F00CFE0220BDE81D
:104C4000F08701F0F0FF352002F011FA12E00A209F
:104C5000FFF743FD0A2C0BD9FB2219A11EA002F07D
:104C6000F9FD21A002F0F6FD01F0DDFF0220E6E7EC
:104C7000641CA4B2012002F0EBF90128E7D018E08F
:104C8000202002F0F4F9701C18F8061080B2421CC3
:104C900018F8000096B241EA002A09EB0704600503
:104CA00002D1204601F0F8FF2046514602F0C4F838
:104CB000BF1C6D1EADB2E3D201F0C1FF0320BEE701
:104CC0002E2E5C53595354454D5C464C4153485C21
:104CD000666C6173682E63004C6F674572723A2090
:104CE00025732C25640000000000000010B586B07C
:104CF00001214FF4017000F0CEFB4FF4004000F0B2
:104D00004DFB494C204600F0EBFD002101918DF850
:104D100008108DF809104FF46022039204910121CC
:104D20008DF8141001A9204600F006FE012000F0C5
:104D300065FF0121204600F027FE204600F047FED7
:104D4000204600F049FE0028FAD1204600F04BFE34
:104D5000204600F04DFE0028FAD106B010BD10B577
:104D6000314C014607230122204600F06FFE01214D
:104D7000204600F044FE0221204600F04DFF0028AE
:104D8000F9D02046BDE8104000F0A6BE70B5002561
:104D900000241020FFF7E3FF284485B20A20FFF724
:104DA0009CFC641CE4B2052CF3D30520B5FBF0F0A9
:104DB00070BD2DE9F04107460E460025002408E0AD
:104DC0003846FFF7CCFF05440A20FFF786FC641C39
:104DD000E4B2B442F4D3B5FBF6F080B2BDE8F081A2
:104DE00010B50A211020FFF7E4FF06F087FA06F05D
:104DF00059FA4FF066320D4B05F044FF02460B4660
:104E00000B480C4906F064F90B4A0C4B05F0E2FC28
:104E100000220B4B05F022FC00220A4B05F032FF6A
:104E200005F06CFE00B210BD0024014066664A3FEA
:104E3000E17A14AE47E1F63F22FDF675E09C713F42
:104E40000000394000005940FEB505460E460121DC
:104E5000084600F020FB4FF48037019700248DF8BE
:104E600008408DF8095001258DF80A5001A800F07E
:104E700075FF384600F0D1FF8DF800508DF80160C5
:104E80008DF802408DF80340684600F03EF81B495B
:104E900002200860C02000F0DBFF012000F0D5FFF9
:104EA000FEBD3EB50121080700F000FB01248DF88E
:104EB00008408DF8094000258DF80A508DF80B4008
:104EC00002A800F022F8684600F07FFF200400905E
:104ED0008DF8045008208DF805008DF806406846CE
:104EE00000F03CFFC02000F0B3FF012000F0ADFF58
:104EF0003EBD4FF4803000F090BF000000E100E0C4
:104F00002A4908432A490860704770B50F23C278C0
:104F100001260178002A1ED0254A126802F4E062B8
:104F2000C2F5E062120AC2F10404D3404578A540FC
:104F300082781A402A43120101F1E02181F800240D
:104F4000007800F01F018E404009800000F1E02051
:104F5000C0F8006170BD01F01F0086404809800064
:104F600000F1E020C0F8806170BD124A1140014399
:104F70000F48001F016070470D4A121D002903D021
:104F800011680143116070471168814311607047D7
:104F90004FF0E021042804D0086920F004000861E3
:104FA0007047086940F00400086170470000FA0586
:104FB0000CED00E080FFFF1F10B59C49884209D12D
:104FC0000121042000F07DFA0021BDE810400420FA
:104FD00000F077BA9649884209D10121082000F0F3
:104FE00070FA0021BDE81040082000F06ABA91492B
:104FF000884209D10121102000F063FA0021BDE8A8
:105000001040102000F05DBA8B49884209D101217F
:10501000202000F056FA0021BDE81040202000F0CA
:1050200050BA8649884209D10121402000F049FA4E
:105030000021BDE81040402000F043BA804988427A
:1050400009D10121802000F03CFA0021BDE8104088
:10505000802000F036BA7B4988420AD184150121AC
:10506000204600F02EFA2046BDE81040002100F056
:1050700028BA10BD10B50121084600F022FA00211F
:10508000BDE81040012000F01CBA2DE9F0410022DB
:10509000CC7804F00F03E40601D58C7823430C7818
:1050A0004FF00F0714F0FF0F4FF0010C1CD00568F4
:1050B0000CFA02F40E882640A64211D1960007FA97
:1050C00006F825EA080503FA06F848EA0505CE7849
:1050D000282E02D0482E02D002E0446100E0046194
:1050E000521C082AE4D305600A88FF2A1ED94568A5
:1050F000002202F108060CFA06F40E882640A642A9
:1051000010D1960007FA06F825EA080503FA06F812
:1051100048EA0505CE78282E00D14461CE78482E85
:1051200000D10461521C082AE3D34560BDE8F08138
:105130004FF6FF710180022181700421C170704718
:105140000246002092680A4200D001207047806821
:1051500080B2704702460020D2680A4200D0012087
:105160007047C06880B27047016170474161704705
:10517000002A01D00161704741617047C1607047EA
:1051800041F4803282618161826181698069704706
:1051900010B52D4B1A684FF68074224042EA001079
:1051A0000843186010BD2949C8617047F0B5264C06
:1051B000002801DAE36900E06368C0F30346420DAA
:1051C000120185B2C0F301579540032F07D0C202E8
:1051D0000CD50322B240934343F0706209E023F000
:1051E0007062636823F07063636002E0AB4343F076
:1051F000706201B12A43002801DAE261F0BD626009
:10520000F0BD10B58A07120F0F23934021F003045D
:105210000D4921448C689C438C608B68904003430B
:105220008B6010BD0949DC310860704700080140FF
:10523000000C014000100140001401400018014022
:10524000001C0140002001400000014000002042FD
:10525000B448016841F0010101604168B24A11405F
:1052600041600168B14A11400160016821F4802168
:105270000160416821F4FE0141604FF41F0181602B
:105280007047A8490A6822F480320A600A6822F44A
:1052900080220A60B0F5803F07D0B0F5802F03D19F
:1052A000086840F4A02008607047086840F4803027
:1052B000086070470346002059099A4A01290AD01C
:1052C00002290AD0516A03F01F02012393400B42C6
:1052D00000D0012070471168F5E7116AF3E718B5AF
:1052E000002000904FF4A0643120FFF7E3FF009905
:1052F000491C00910099A14201D00028F4D031202E
:10530000FFF7D8FF08B1012018BD002018BD854A5D
:10531000116821F0F80141EAC0001060704784492B
:10532000086070477F4B5A6822F47C120843104390
:10533000586070477E49086670477A4A516821F084
:1053400003010143516070477648406800F00C004B
:105350007047744A516821F0F00101435160704771
:10536000704A516821F4E0610143516070476D4A11
:10537000516821F4605141EAC00050607047694AA9
:10538000002903D0517A014351727047517A814309
:10539000517270476649D83108607047614A516858
:1053A00021F440410143516070475E4900222031A1
:1053B0000A7001F82029012805D0042802D105200F
:1053C00081F820007047012081F82000704759497A
:1053D0000860704753490A6A02430A627047554998
:1053E00044390860704710B54E4A516801F00C010D
:1053F000514B002927D0042927D0082927D0036042
:10540000516801F0F00109094C4B5C5C0168E14016
:105410004160546804F4E064240A1C5D21FA04F439
:105420008460546804F46054E40A1B5DD940C16090
:10543000526802F44042920B404B1B1F9A5CB1FB36
:10544000F2F1016110BD0360DAE70360D8E751684B
:1054500001F47011536803F48033022404EB91418A
:1054600033B153689B0307D5354B59430160C7E7F8
:10547000334B59430160C3E72F4B59430160BFE7EA
:10548000284A002903D0516901435161704751698D
:10549000814351617047234A002903D09169014338
:1054A0009161704791698143916170471D4A00295C
:1054B00003D0D1690143D1617047D1698143D16182
:1054C0007047184A002903D0D1680143D160704762
:1054D000D1688143D1607047124A002903D0116915
:1054E000014311617047116981431161704711498E
:1054F0004039086070470E49C86470470949C8714F
:1055000070470848416A41F0807141627047014626
:105510000020044A92680A4200D0012070470149E5
:1055200088727047001002400000FFF8FFFFF6FE8F
:10553000000042428004424200127A0030060020FD
:1055400000093D0010B5E14988420AD101218C03D0
:105550002046FFF7B6FF2046BDE810400021FFF7C8
:10556000B0BFDB4988420AD101214C042046FFF735
:10557000B3FF2046BDE810400021FFF7ADBFD5497D
:1055800088420AD101218C042046FFF7A5FF20465E
:10559000BDE810400021FFF79FBFCF4988420AD1E4
:1055A0000121CC042046FFF797FF2046BDE81040BC
:1055B0000021FFF791BFC94988420AD101210C059A
:1055C0002046FFF789FF2046BDE810400021FFF785
:1055D00083BF10BD30B585B004460D46208A4CF619
:1055E000FF710840E98801432182A0894EF6F3113A
:1055F0000840A9882A8911436A8902431143A1817D
:10560000A08A4FF6FF410840A9890143A18268465C
:10561000FFF7E9FEAD48844201D1039800E002980B
:10562000A189090408D500EBC00101EB001029682D
:105630004900B0FBF1F007E000EBC00101EB001006
:1056400029688900B0FBF1F06422B0FBF2F1090196
:105650000B096FF018056B4300EB8300A3891D0451
:105660004FF0320307D503EBC000B0FBF2F000F0BF
:105670000700084306E003EB0010B0FBF2F000F077
:105680000F000843208105B030BD4FF41651016072
:1056900000218180C18001810C224281818170477B
:1056A00010B5038A4FF2FF0213400A884C88224348
:1056B0008C88C9880C4322431A43028210BD002102
:1056C000018041808180C1807047002904D0818998
:1056D00041F4005181817047818921F40051818119
:1056E000704710B540F66A13C1F3421301F01F046E
:1056F0000121A140012B07D0022B07D014303AB171
:1057000002680A43026010BD0C30F8E71030F6E77B
:1057100002688A43026010BD002A03D0828A0A43CD
:1057200082827047828A8A4382827047028A22F08C
:105730000F020282028A0A4302827047828922F49F
:105740000062828182890A4382817047002904D0E5
:10575000818941F0020181817047818921F0020134
:1057600081817047028A22F020020282028A0A4363
:1057700002827047002904D0018A41F480410182ED
:105780007047018A21F4804101827047C1F308010A
:10579000818070478088C0F308007047818941F09C
:1057A000010181817047028BD2B20283028B42EAEF
:1057B000012101837047028B02F47F420283028B36
:1057C0000A4302837047002904D0818A41F02001F6
:1057D00081827047818A21F02001818270470029EF
:1057E00004D0818A41F0100181827047818A21F0C2
:1057F000100181827047002904D0818A41F008019C
:1058000081827047818A21F00801818270470029D6
:1058100004D0818941F40041818170478189C1F3BD
:105820000E0181817047002904D0818A41F4006112
:1058300081827047818A21F4006181827047828A67
:1058400022F004028282828A0A43828270470029FF
:1058500004D0818A41F0020181827047818A21F05F
:105860000201818270470246002012880A4200D05D
:10587000012070478A05C9430180704770B5002434
:1058800040F66A12C1F3421301F01F05012606FA21
:1058900005F2012B0CD0022B0DD0838A1340090A8C
:1058A0008E40008830400BB100B10124204670BD0D
:1058B00083891340F3E7038A1340F0E740F66A1246
:1058C0000A0A01219140C943018070470038014014
:1058D0000044004000480040004C004000500040A0
:1058E00010B5DB4988420AD1441501212046FFF753
:1058F000E8FD2046BDE810400021FFF7E2BDD54994
:1059000088420AD1041501212046FFF7DAFD20461E
:10591000BDE810400021FFF7D4BDCF4988420AD12D
:105920000121CC032046FFF7CCFD2046BDE8104006
:105930000021FFF7C6BD10BD10B54268C74B1A4025
:105940000C790B6842EA0422134343608268C44B1B
:105950001A40D1E9024323434C7942EA44021343FB
:105960008360C26A22F47002097C491EC9B242EA0D
:105970000151C16210BD002101600171417181605E
:10598000C160012101747047002904D0816841F091
:10599000010181607047816821F0010181607047D9
:1059A000002904D0816841F480718160704781686A
:1059B00021F4807181607047C9B2002A03D0426827
:1059C0000A434260704742688A4342607047816878
:1059D00041F008018160704701460020896809078D
:1059E00000D501207047816841F004018160704753
:1059F000014600208968490700D501207047002929
:105A000004D0816841F4A00181607047816821F46D
:105A1000A00181607047014600208968490200D5D5
:105A200001207047426822F46042491E42EA413137
:105A300041607047002904D0416841F40061416031
:105A40007047416821F400614160704770B50726D6
:105A500009290AD9C568A1F10A0404EB4404A64047
:105A6000B543A3401D43C56007E0056901EB410450
:105A7000A640B543A3401D4305611F23072A09D251
:105A8000446B521E02EB820293409C4391400C43B4
:105A9000446370BD0D2A09D2046BD21F02EB82024F
:105AA00093409C4391400C43046370BDC46A0D3A1B
:105AB00002EB820293409C4391400C43C46270BD50
:105AC000002904D0816841F48011816070478168A9
:105AD00021F4801181607047C06C80B270475C48CF
:105AE0004C3000687047002904D0416841F480615F
:105AF00041607047416821F480614160704700292E
:105B000004D0416841F4805141607047416821F4FC
:105B1000805141607047826822F4E0420A4382600B
:105B20007047002904D0816841F4004181607047CA
:105B3000816821F4004181607047002904D08168A8
:105B400041F4021181607047816821F40211816083
:105B50007047014600208968890200D501207047FE
:105B600070B5072609290AD9C568A1F10A0404EB12
:105B70004404A640B543A3401D43C56007E0056942
:105B800001EB4104A640B543A3401D430561836B6F
:105B9000C3F30154121B921C02EB82021F24944097
:105BA000A34391400B43836370BD826B22F4401288
:105BB000491E42EA01518163704708B50090009880
:105BC000084400900098026008BD08B50090009855
:105BD0000844283000900098006880B208BD4268F0
:105BE000204B1A400A43426070474162826270470C
:105BF000426822F01F020A4342607047144908318C
:105C0000002804D0086840F4000008607047086865
:105C100020F40000086070470246002012680A4223
:105C200000D001207047C9430160704710B502469B
:105C300000200B0A5468C9B20C401168194202D006
:105C4000002C00D0012010BD090AC9430160704733
:105C50000024014000280140003C0140FFFEF0FF0D
:105C6000FDF7F1FFFFFD3FFF0D49086070470C494C
:105C7000486070470A498860704709494AF6AA2077
:105C80000860704706494CF6CC40086070470146F2
:105C90000020034AD2680A4200D001207047000069
:105CA0000030004010B50120FFF721FCBDE8104096
:105CB0000020FFF71CBC2049086070471E49091FDF
:105CC000086070471C498431086070471B4A11887E
:105CD00021F46071014311807047184A118821F046
:105CE0007F0101431180704708B5144A2C3A1044D3
:105CF00000900098016008BD08B510492C3908448F
:105D000000900098008808BD0B489C300068C0B225
:105D100070470A480830018841F00101018070474E
:105D20000548A0300068C0B27047044808300188B8
:105D300041F002010180704704860D422C6C004046
:105D4000384900200860091D0860091D0860091D08
:105D500008603449344814310860704730B5314A1E
:105D600083790168002B2AD013688B431360111DBF
:105D70000B680468A3430B60017911440B68046845
:105D800023430B60274C0834216803689943216042
:105D9000231D19680568A94319604179102905D0A8
:105DA00011440A68006802430A6030BD2168026835
:105DB00011432160196800680143196030BD007902
:105DC000104402688A43026030BD00210160017105
:105DD0000C22427181717047124910310A680243E6
:105DE0000A607047014600200E4A143212680A42C7
:105DF00000D0012070470B491431086070470146FC
:105E00000020084A12680A40064B14331B680B42F4
:105E100002D0002A00D001207047024914310860E6
:105E20007047000000040140FFFF0F0010B5012182
:105E30000C072046FFF750FB2046BDE8104000212C
:105E4000FFF74ABB21490862704720490861704743
:105E50001F4A116821F0E0010143116070471B499E
:105E6000A031086070471A4B1A6822F003020243FF
:105E70001A601848026842F004020260012905D045
:105E800020BF016821F004010160704730BFF8E7CE
:105E90000F48016841F004010160016841F002010E
:105EA00001600C48016841F00401016030BF704797
:105EB00001460020064A52680A4200D0012070477D
:105EC00003490A6842EA80000860704700000E42F9
:105ED0000070004010ED00E03A4A002903D011881C
:105EE0000143118070471188814311807047354804
:105EF000001D018841F01001018070473148001DEC
:105F0000018821F01001018070472E481C30008864
:105F10002C491831098840EA01407047294A010C90
:105F200018321180111D08807047264AC0F30341C2
:105F300008321180111D0880E0E7224A010C20324E
:105F40001180111D088070471E481030008800071E
:105F5000010B1C4814300088084370471948001D85
:105F600001888906FCD570471648001D018821F07C
:105F70000801018001880907FCD57047014600200F
:105F8000104A121D12880A4200D0012070470D49A4
:105F9000091D0A8882430A8070470A49091D098839
:105FA000C2B21140074A1288024202D009B1012050
:105FB0007047002070470349091D0A8882430A8000
:105FC000704700000028004010B5FE4988420AD101
:105FD000C41401212046FFF774FA2046BDE81040A2
:105FE0000021FFF76EBAB0F1804F0CD0F64988421D
:105FF00013D101210220FFF76FFA0021BDE8104004
:106000000220FFF769BA01210846FFF765FA00216F
:10601000BDE810400120FFF75FBAEC49884209D182
:1060200001210420FFF758FA0021BDE810400420A8
:10603000FFF752BAE649884209D101210820FFF74B
:106040004BFA0021BDE810400820FFF745BAE149AE
:10605000884209D101211020FFF73EFA0021BDE856
:1060600010401020FFF738BADB49884209D10121DE
:106070002020FFF731FA0021BDE810402020FFF773
:106080002BBAD64988420AD1441401212046FFF791
:1060900018FA2046BDE810400021FFF712BAD04997
:1060A00088420AD10121CC042046FFF70AFA204693
:1060B000BDE810400021FFF704BACA4988420AD15E
:1060C00001210C052046FFF7FCF92046BDE81040F1
:1060D0000021FFF7F6B9C44988420AD101214C05D5
:1060E0002046FFF7EEF92046BDE810400021FFF7FB
:1060F000E8B9BE49884209D101214020FFF7ECF9F7
:106100000021BDE810404020FFF7E6B9B8498842B9
:1061100009D101218020FFF7DFF90021BDE81040FF
:106120008020FFF7D9B9B34988420AD184150121EB
:106130002046FFF7D1F92046BDE810400021FFF7C7
:10614000CBB9AD4988420AD101210C042046FFF7A2
:10615000B8F92046BDE810400021FFF7B2B9A749C1
:1061600088420AD101214C042046FFF7AAF92046B3
:10617000BDE810400021FFF7A4B9A14988420AD127
:1061800001218C042046FFF79CF92046BDE8104011
:106190000021FFF796B910BD30B50288894C8F4DAC
:1061A000A0420DD0A8420BD0B0F1804F08D0864B52
:1061B000984205D0854B984202D0854B984203D136
:1061C00022F070034A881A43824B984206D0824BD1
:1061D000984203D022F44073CA881A4302808A8806
:1061E00082850A880285A0420AD0A84208D0824A45
:1061F000904205D0814A904202D0814A904201D11A
:10620000097A01860121818230BD30B5028C22F0ED
:1062100001020284028C8388048B24F0700424F031
:1062200003050C882C4322F002020D8915434A888D
:106230002A43644DA8420BD0684DA84208D06E4D49
:10624000A84205D06D4DA84202D06D4DA8420FD195
:1062500022F008054A892A4322F004058A882A4345
:1062600023F4807323F400738D891D43CB892B4362
:1062700083800483C9888186028430BD70B5028C16
:1062800022F010020284028C8388048B24F4E04400
:1062900024F440760D884FF6FF7404EA0525354353
:1062A00022F020020E8904EA061616434A8804EA00
:1062B00002123243434EB04202D0484EB04217D190
:1062C00022F080024E8904EA0616164326F04006A4
:1062D0008A8804EA0212324323F4806323F40063C1
:1062E0008E8904EA86061E43CB8904EA830333437E
:1062F00083800583C9880187028470BD70B5028CD4
:1063000022F480720284028C8388848B24F07004CF
:1063100024F003040D88254322F400720E894FF601
:10632000FF7404EA062616434A8804EA022232432E
:10633000244EB04202D0294EB04217D122F400665A
:106340004A8904EA0222324322F480668A8804EAF7
:106350000222324323F4805323F400538E8904EA4B
:1063600006161E43CB8904EA0313334383808583D7
:10637000C9888187028470BD70B5028C22F4805276
:106380000284058C8288838B23F4E04323F44076D7
:106390000C884FF6FF7303EA0424344325F40055B8
:1063A0000E8903EA06362E434D8803EA0535354348
:1063B000044EB04202D0094EB04226D122F48046AB
:1063C0008A891FE0002C01400004004000080040C2
:1063D000000C004000100040001400400034014058
:1063E000004C0140005001400054014000180040A2
:1063F000001C0040002000400040014000440140DB
:106400000048014003EA8212324382808483C988B3
:10641000A0F84010058470BD828B22F44062828314
:10642000828B4FF6FF7303EA01210A438283704790
:10643000F0B5048C24F480540484868B048C4FF6CD
:10644000FF7505EA013726F4734605EA0222324356
:1064500005EA03331343F74A90420ED0F64A9042BE
:106460000BD0B0F1804F08D0F44A904205D0F44AE6
:10647000904202D0F34A904205D124F400513943AE
:1064800041F4805104E024F402420A4342F4805172
:1064900083830184F0BD828B22F00C028283828B85
:1064A0000A4382837047F0B5048C24F4807404841A
:1064B000858B048C4FF6FF7707EA012625F0F3055C
:1064C00007EA031313432B43DA4A90420ED0DA4A09
:1064D00090420BD0B0F1804F08D0D84A904205D0FE
:1064E000D74A904202D0D74A904205D124F4007195
:1064F000314341F4807104E024F420620A4342F401
:10650000807183830184F0BD028B22F44062028398
:10651000028B4FF6FF7303EA01210A43028370479F
:10652000F0B5048C24F010040484068B048C4FF620
:10653000FF7505EA011726F4734605EA0333334372
:1065400005EA02221A43BB4B98420ED0BA4B98423E
:106550000BD0B0F1804F08D0B84B984205D0B84B63
:10656000984202D0B74B984205D124F0200139431C
:1065700041F0100104E024F0A0030B4343F01001AC
:1065800002830184F0BD028B22F00C020283028B95
:106590000A430283704770B5048C24F0010404841C
:1065A000058B048C25F0F3054FF6FF7606EA0313FE
:1065B00013432B439F4A90420ED09F4A90420BD0E8
:1065C000B0F1804F08D09D4A904205D09C4A90423D
:1065D00002D09C4A904205D124F002020A4342F0C4
:1065E000010104E024F00A020A4342F0010103839E
:1065F000018470BD70B505460C468E48854209D0B1
:106600008D48854206D0B5F1804F03D08B48854236
:1066100000D08B4820886188A288238958B104283B
:1066200011D0082817D02846FFF702FFE188284636
:10663000BDE87040F0E62846FFF7ADFFE188284648
:10664000BDE870409FE72846FFF76AFFE1882846CB
:10665000BDE8704058E72846FFF725FFE188284647
:10666000BDE8704017E72DE9F04107460C460025CC
:1066700001266188002900D10225A288012A00D1C3
:1066800002262088238988B13846FFF749FFE18830
:106690003846FFF739FF2389324629463846FFF747
:1066A0007AFFE1883846BDE8F0416CE73846FFF7ED
:1066B00072FFE1883846FFF766FF23893246294694
:1066C0003846FFF72DFFE1883846BDE8F0411BE76B
:1066D00010B50A884B88CC881A438B8823431A4309
:1066E0000B891A434B8989891A430A43A0F844202D
:1066F00010BD4FF6FF71818000210180C180418073
:10670000017270470021018041808180C180018138
:1067100041818181C1817047002101804180012236
:106720008280C18001817047002101804180818089
:10673000C1800181418181817047002904D0018895
:1067400041F0010101807047018821F001010180C1
:106750007047002905D030F8441F41F40041018002
:10676000704730F8441FC1F30E0101807047002AC2
:1067700003D082890A438281704782898A43828159
:106780007047818270471143A0F848107047002A73
:1067900003D082890A438281704782898A43828139
:1067A0007047018921F0070101817047028922F0B9
:1067B00070020A430281704700B503461846FFF78E
:1067C000F5FF188940F00700188100BD70B50D462F
:1067D00004461146602D0CD001222046FFF7DBFE57
:1067E00029462046FFF7E2FF208940F0070020817C
:1067F00070BD01222046FFF793FEF1E730B5048912
:10680000E4B24FF6FF7505EA032313430B4323431A
:10681000038130BD10B504462046FFF7EFFF208905
:1068200020F0070040F0070020F0700040F07000FA
:10683000208110BD002C01400034014000040040C4
:1068400000080040000C004010B504462046FFF749
:10685000D5FF208940F480402081EAE701858282CB
:106860007047028822F070020A430280704770B5B8
:106870000589048B068C25F007050D434FF6FC4176
:106880000C4040F201110C4326F022064FF6FF7136
:1068900001EA03111143314305810483018470BD72
:1068A000028B22F070020A4302837047028B22F4AB
:1068B000E0424FF6FF7303EA012111430183704761
:1068C000828B22F070020A4382837047828B22F40B
:1068D000E0424FF6FF7303EA0121114381837047C1
:1068E000002904D0018841F08001018070470188AF
:1068F00021F0800101807047002904D0818841F097
:10690000040181807047818821F0040181807047F3
:10691000002904D0818841F0080181807047818876
:1069200021F0080181807047002904D0818841F05E
:10693000010181807047818821F0010181807047C9
:10694000028B22F008020A4302837047028B22F472
:1069500000624FF6FF7303EA012111430183704780
:10696000828B22F008020A4382837047828B22F4D2
:1069700000624FF6FF7303EA0121114381837047E0
:10698000028B22F004020A4302837047028B22F436
:1069900080624FF6FF7303EA0121114301837047C0
:1069A000828B22F004020A4382837047828B22F496
:1069B00080624FF6FF7303EA012111438183704720
:1069C000028B22F080020A4302837047028BC2F3DB
:1069D0000E024FF6FF7303EA012111430183704752
:1069E000828B22F080020A4382837047828BC2F33B
:1069F0000E024FF6FF7303EA0121114381837047B2
:106A0000028C22F002020A4302847047028C22F0B8
:106A100008020A4302847047028C22F020024FF6DB
:106A2000FF7303EA0111114301847047028C22F0C5
:106A300080024FF6FF7303EA01111143018470478E
:106A4000028C22F400724FF6FF7303EA0121114316
:106A500001847047028C22F400624FF6FF7303EA50
:106A60000121114301847047028C22F400524FF639
:106A7000FF7303EA013111430184704710B501230C
:106A80008B40048C9C430484038C8A40134303840E
:106A9000CFE610B504238B40048C9C430484038C04
:106AA0008A4013430384C4E630B500F1180301247F
:106AB0008C40058CA5430584002911D008290FD0EE
:106AC000091FC1F34E001844016821F4E041016040
:106AD00001684FF6FF7303EA02221143016030BDE3
:106AE00003EB5100016821F070010160016811435E
:106AF000016030BD002904D0018841F0020101800D
:106B00007047018821F0020101807047002904D0FC
:106B1000018841F0040101807047018821F00401DF
:106B200001807047002904D0818841F08001818074
:106B30007047818821F0800181807047028822F0AF
:106B40000802028002880A4302807047828822F08D
:106B50007002828082880A4382807047028922F014
:106B60000702028102890A4302817047028922F0EA
:106B70008002028102890A43028170478184704742
:106B8000818570478186704701877047818770478C
:106B9000A0F840107047028822F4407202800288F8
:106BA0000A4302807047808E7047008F7047808F45
:106BB0007047B0F840007047808C7047008D704778
:106BC00002460020128A0A4200D001207047C943C1
:106BD0000182704702460020138A0B4092890A40C6
:106BE000002B02D0002A00D001207047C943018247
:106BF00070470000FE4A116801F03801014311603E
:106C00007047FB490A6822F008020A600A680243DA
:106C10000A607047F6490A6822F010020A600A68A2
:106C200002430A607047F248F2494160F24941600C
:106C30007047EF48EF494160EF4941607047EC48C9
:106C4000016941F0800101617047E948016941F043
:106C50008001016170470420E549CA68D20701D06C
:106C600001207047CA68520701D502207047C968E1
:106C7000C906FBD50320704700B50346FFF7EBFFBD
:106C800002E0FFF7E8FF5B1E012801D1002BF8D1DD
:106C9000002B00D1052000BD70B505464FF430260D
:106CA0003046FFF7E9FF042811D1D14C206940F0AC
:106CB000020020616561206940F04000206130469B
:106CC000FFF7DAFF216941F6FD721140216170BDC5
:106CD00030B54FF430252846FFF7CEFF042810D1F9
:106CE000C34C206940F004002061206940F040005E
:106CF00020612846FFF7C0FF216941F6FB72114071
:106D0000216130BD00B50346FFF7A5FF02E0FFF7A4
:106D1000A2FF5B1E012801D1002BF8D1002B00D16E
:106D2000052000BD30B54FF430252846FFF7EAFFB7
:106D3000042810D1AE4C206940F004002061206985
:106D400040F0400020612846FFF7DCFF216941F652
:106D5000FB721140216130BD0020A549C969890736
:106D600000D50120704770B5A525FFF7F5FF00B1EC
:106D700000254FF430263046FFF77EFF042818D157
:106D80009B4C9C48A0609C48A060206940F020007B
:106D90002061206940F0400020613046FFF76CFF21
:106DA00041F6EF76042805D0052802D0216931404C
:106DB000216170BD206941F6DF71084020612069C2
:106DC00040F0100020618D4805804FF40050FFF71F
:106DD00053FF0528EDD021693140216170BD2DE9B7
:106DE000F84105460E46002000904FF40057384603
:106DF000FFF742FF04280FD17D4C206940F00100CD
:106E000020612E80B8464046FFF736FFBF1E04289B
:106E100004D0216939402161BDE8F881AD1C00959D
:106E20000099300C08804046FFF726FF2169394061
:106E30002161F1E700887047F0B506460D464FF432
:106E400000573846FFF718FF04280CD1684C20691A
:106E500040F00100206135803846FFF70DFF2169C1
:106E6000BA1E11402161F0BDF0B505460E464FF443
:106E700000573846FFF700FF042813D15C4C5D48EB
:106E8000A0605D48A060206940F0100020612E8065
:106E90003846FFF7F1FE052804D0216941F6EF726C
:106EA00011402161F0BD2DE9F043C043C4B2C0F3ED
:106EB0000725C0F30746070E4FF400594846FFF771
:106EC000DBFE04283CD1DFF828814A49C8F80810C5
:106ED0004949C8F80810D8F8101041F01001C8F856
:106EE0001010FF2C05D04548083004804846FFF7B5
:106EF000C3FE042807D1FF2D05D040480A30058085
:106F00004846FFF7B9FE042807D1FF2E05D03B48BD
:106F10000C3006804846FFF7AFFE042807D1FF2F4C
:106F200005D036480E3007804846FFF7A5FE0528F5
:106F300006D0D8F8101041F6EF721140C8F81010C2
:106F4000BDE8F08370B505464FF430263046FFF7B4
:106F500093FE042818D1264C2648A0602648A0603D
:106F6000206940F020002061206940F0400020614D
:106F70003046FFF781FE41F6DF71042805D0052871
:106F800002D022690A40226170BD20690840206158
:106F9000206940F010002061184815B100210180DF
:106FA00001E0A52101803046FFF766FE0528EBD001
:106FB000216941F6EF721140216170BD2DE9F04168
:106FC00006460D4617460A4C0A48A0600A48A060CB
:106FD0004FF400584046FFF74FFE04281DD12069AA
:106FE00040F0100020613D43354345F0F80007E0D4
:106FF0000020024023016745AB89EFCD00F8FF1F59
:107000002549891C08804046FFF736FE052804D034
:10701000216941F6EF7211402161BDE8F0811F48FE
:10702000C069800870471D48006A704700201B49EE
:107030000968890600D501207047184A002903D045
:1070400011690143116170471169814311617047F2
:1070500001460020114A012904D0D2680A4200D01A
:1070600001207047D169C907FBD0012070470B4947
:10707000C860704704200949CA68D20701D00120BE
:107080007047CA68520701D502207047C968C9060F
:10709000FBD503207047000000F8FF1F00200240CE
:1070A00001684FF6FE7211400160002101604160ED
:1070B0008160C1607249724A0839904204D14868BF
:1070C00040F00F00486070476D4A1432904204D17E
:1070D000486840F0F00048607047694A28329042A2
:1070E00004D1486840F4706048607047644A3C329C
:1070F000904204D1486840F4704048607047604A4C
:107100005032904204D1486840F470204860704783
:107110005B4A6432904204D1486840F47000486091
:107120007047574A7832904204D1486840F0706006
:1071300048607047534A111F904204D1086840F0DC
:107140000F00086070474F4A1432904204D108681B
:1071500040F0F000086070474A4A2832904204D15B
:10716000086840F4706008607047464A3C329042BC
:1071700004D1086840F4704008607047414A5032BA
:107180009042FAD1086840F470200860704730B52A
:10719000026847F6F0739A430C6A8B682343D1E97F
:1071A00004452C4323438C692343CC6923434C6A15
:1071B00023438C6A234313430360CA6842600A680E
:1071C00082604968C16030BD00210160416081601A
:1071D000C160016141618161C1610162416281629D
:1071E0007047002904D0016841F001010160704737
:1071F00001684FF6FE72114001607047002A03D00B
:1072000002680A430260704702688A43026070475E
:1072100041607047406880B2704702460020D1004C
:1072200003D518490839096802E015490839096881
:10723000114200D001207047C10003D51149091F38
:10724000086070470E4908394860704702460020C0
:10725000D10003D50B490839096802E0084908390B
:107260000968114200D001207047C10003D50549CB
:10727000091F0860704702490839486070470000DC
:1072800008000240080402407047162205A10FA022
:1072900000F0E0FA11A000F0DDFAFEE7FEE7FEE7FD
:1072A000FEE770472E2E5C53544D33324631307812
:1072B0005F46574C69625C7372635C73746D333202
:1072C000663130785F69742E630000004C6F67454B
:1072D00072723A2025732C256400000048617264A4
:1072E0004661756C745F48616E646C657221000064
:1072F00071B65A4801685A4A01F4E06111430160CD
:10730000BFF34F8FFEE70CB5002201920092554863
:10731000016841F4803101604FF4A063016801F419
:10732000003100910199491C0191009911B901990D
:107330009942F3D10168890302D50121009100E04F
:1073400000920099012930D147490A6842F01002A1
:107350000A600A6822F003020A600A6842F0020228
:107360000A604168416041684160416841F4806160
:107370004160416821F47C114160416841F4E811A9
:107380004160016841F08071016001688901FCD5AC
:10739000416821F003014160416841F00201416010
:1073A0004168C1F381010229FAD10CBDABE710B5E8
:1073B0002C48016841F00101016041682B4A1140ED
:1073C000416001682A4A11400160016821F480216E
:1073D0000160416821F4FE0141604FF41F018160AA
:1073E000FFF7E4FF1D494FF00060091F086010BD62
:1073F00010B51C4A506800F00C011E4B1E480029B5
:107400000ED004290ED008290ED0036051681A4A04
:10741000C1F30311121D515C0268CA40026010BD25
:107420000360F3E70360F1E7516801F470115368FA
:1074300003F48033022404EB914133B153689B037E
:1074400007D50E4B59430160E0E70C4B59430160EF
:10745000DCE7084B59430160D8E700000CED00E081
:107460000400FA0500100240002002400000FFF86E
:10747000FFFFF6FE00127A004006002000093D00E2
:1074800010B5A94988420AD1841401212046FEF78B
:1074900018F82046BDE810400021FEF712B8A349B5
:1074A00088420AD1041401212046FEF715F820462F
:1074B000BDE810400021FEF70FB89D4988420AD16F
:1074C000C41301212046FEF707F82046BDE810400E
:1074D0000021FEF701B810BD30B5028802F4415317
:1074E0000A884C88CD8822438C882C4322430C89FF
:1074F00022434C8922438C892243CC8922431A435C
:107500000280828B22F400628283098A018230BD6C
:10751000F0B585B005460C46022000210126AA8B55
:107520004FF240031A40AA8302222A84AF8BA2683A
:10753000022A21D0A08800B102266846FDF753FF39
:107540000098E188B1F5007F2CD07101B0FBF1F01B
:1075500000EB8000A1684000B0FBF1F0401D80B25C
:107560000A21B0FBF1F000F00101401AC0F34F0016
:107570004FF6FF7202EA0121821EFE2A01D3022089
:107580000021E288084302432A8420886188A28976
:107590000843A18811430843384340F40060A8839E
:1075A00005B0F0BD000A00EB8000A1684000B0FB10
:1075B000F1F0401D80B2D3E700210180418081803D
:1075C000C180018141818181C18107210182704790
:1075D0000021018041808180C180022282608181FE
:1075E0007047002904D0018841F0400101807047B4
:1075F000018821F0400101807047002904D0818B6F
:1076000041F4806181837047818B21F480618183A3
:107610007047090901238B4099B2002A03D0828860
:107620000A438280704782888A4382807047002A9A
:1076300003D082880A438280704782888A4382808E
:1076400070478181704780897047A1F57E42FF3A7B
:1076500004D0018841F4807101807047018821F4D1
:10766000807101807047002904D0818841F00401B5
:1076700081807047818821F00401818070470288F1
:1076800022F40062028002880A4302807047018867
:1076900041F4805101807047002904D0018841F4F1
:1076A000005101807047018821F40051018070472A
:1076B000012901D0008B7047808A7047008A70478B
:1076C000B1F5804F04D0018821F4804101807047DA
:1076D000018841F4804101807047024600201289F0
:1076E0000A4200D001207047C9430181704730B57C
:1076F0000246002001F00F03012505FA03F4A3B2AE
:10770000090905FA01F4A4B29188214012891A42AC
:1077100002D0002900D0012030BD01F00F0201216C
:107720009140C9430181704700300140003800405A
:10773000003C004030B50446039D2F4800EB031089
:1077400004600024047141718260C560102B00DB6D
:10775000002030BD29A10160002101714A1E826014
:10776000C1607047012101717047002101717047AC
:1077700070B5234D2868401C2860286810F1100F50
:1077800001D30020286000241B4E06EB0410017971
:1077900001290BD14179022908D181682A68B2FBFD
:1077A000F1F301FB132109B9C0688047641C102C58
:1077B000EBDB70BD70B5124D6868401C686068688E
:1077C00010F1100F01D30020686000240A4E06EB70
:1077D0000410017901290BD14179012908D181686F
:1077E0006A68B2FBF1F301FB132109B9C068804755
:1077F000641C102CEBDB70BD705B002020000000CF
:1078000054060020704710B5044600F0A9FC00683B
:10781000005DC00602D504F1200010BD204610BD59
:107820007CB51D4616460C00009001D02044401E39
:10783000074B7B442A4669460190304600F015FF0D
:1078400005461CB10020694600F022FF28467CBD99
:10785000650E00000FB4044910B503AA029800F0A9
:107860003BFF10BC5DF814FBB40500200FB41CB541
:10787000084B06AA7B4469460090059800F0F5FE87
:1078800004460020694600F003FF20461CBC5DF85A
:1078900014FB0000190E00000FB47CB50C0009AAFF
:1078A000009001D02044401E084B7B446946019063
:1078B000089800F0DAFE05461CB10020694600F089
:1078C000E7FE28467CBC5DF814FB0000ED0D0000CF
:1078D00070B5044685690068C10601D5302600E010
:1078E0002026C00707D070BDD4E90121304690475B
:1078F000206A401C20626D1EF6D570BD70B504462E
:1079000085690078C00707D170BDD4E90121202026
:107910009047206A401C20626D1EF6D570BD096834
:107920004A0501D540B27047C905FCD500B2704781
:1079300009684A0501D5C0B27047C905FCD580B2B7
:10794000704770B50C460546012A05D02878800698
:1079500000D5EA69002302E0012305E05B1C9342A5
:1079600002D2E05C0028F9D1A869E618C01AA86123
:10797000286A184428622846FFF7AAFF04E0D5E9E0
:10798000012114F8010B9047B442F8D32846FFF7C1
:10799000B5FF70BD2DE9F041064600241068752939
:1079A000314616A510D0FFF7BAFF002802DA404290
:1079B00013A507E031688A0701D512A502E049073F
:1079C00004D511A5012401E0FFF7B2FF00210A222E
:1079D00006F1240709E0B0FBF2FCB0FBF2F302FB76
:1079E0001C00303078541846491C0028F3D1234637
:1079F0002A463046BDE8F04100F0C9BB0000000057
:107A00002D0000002B00000020000000116802681B
:107A1000006A530501D508700AE0D30501D5088036
:107A200006E0130603D5C217C1E9000200E00860B2
:107A3000012070472DE9FF5F15468A460446DFF8AE
:107A4000AC80F8440027D8E900103E46CDE900108C
:107A500010E03AF816106A4602A800F0DBFE411C5E
:107A600007D02178890603D5E269391891420DD8EB
:107A70000744761C2078800602D5E069B84205DD0F
:107A8000AE42E6DB3AF816000028E2D1A069C01B3E
:107A9000A0612046FFF71CFFD8E90010CDE90010D7
:107AA000002017E03AF818106A4602A800F0B2FE6B
:107AB000B0F1FF3F81460BD000250DF1080B05E02A
:107AC000D4E901211BF8050090476D1C4D45F7D303
:107AD00008F10100B0428046E4DB206A38442062AD
:107AE0002046FFF70BFFBDE8FF9F0000AE4D0000F2
:107AF00030B4002100F1240408E002F00705D208A8
:107B0000303542EA4372DB086554491C52EA0305EA
:107B1000F3D10468002310A2250707D5A40600D4DA
:107B200021B1C46901230DA2641EC46130BC00F000
:107B30002EBB10B5044621461068FFF7F9FE024639
:107B40002046BDE810400023D2E7D21D22F00701F5
:107B5000D1E90023CCE70000000000003000000065
:107B6000F0B40D460188090502D5214C7C4402E0A1
:107B70001F4C7C440E34002100F1240608E002F082
:107B80000F071209E75D42EA03721B097754491C8B
:107B900052EA0307F3D102780023120704D5702DAF
:107BA00006D009B1022311342246F0BC00F0EFBA2E
:107BB00001231034F8E770B504460D4621461068DD
:107BC000FFF7B6FE024629462046BDE87040002376
:107BD000C6E7D21D22F00703D3E90023C0E70368FC
:107BE000126843F0200303600823C3610023B7E752
:107BF0008C4C00002DE9F05F894604464FF0000AE6
:107C0000DFF874B1FB44C0F820A02046E168884743
:107C1000002874D0252806D0D4E901219047206A95
:107C2000401C2062F1E700265F462046E168884755
:107C30002028054607DB312D05D2781910F8200CD5
:107C400008B10643F1E7B00701D526F00406C4F8F1
:107C50001CA00027C4F818A02A2D09D0284601F03E
:107C60009BFD38B304EB8708303DC8F8185019E085
:107C700059F8041B204604EB87029161E1688847AC
:107C8000012F054618D1E069002820DA26F02006E9
:107C90001DE0D8F8180000EB800005EB40003038FC
:107CA000C8F818002046E1688847054601F074FDD1
:107CB0000028EED1012F0AD02E2D08D12046E168F0
:107CC00088477F1C0546022F46F02006C4DBA069CA
:107CD000002803DA404246F00106A061F00701D017
:107CE00026F010066C2D0BD0682D09D04C2D39D004
:107CF0006A2D35D0742D35D07A2D33D016E038E08A
:107D0000E1682F4620468847B842054609D16C2FC6
:107D100026D04FF48060E168064320468847054638
:107D200004E06C2F1AD04FF4807006430DB3A5F118
:107D30004100192802D8203546F400664A462946F3
:107D4000204626604E46F4F74DFA80B101280BD04C
:107D5000F61D26F0070000F1080956E74020E4E789
:107D60008020D8E70020D6E706F104094DE7284631
:107D700052E7206ABDE8F09F1C4C000070B5064633
:107D800000F0F6F90468054630460A22002100F0AA
:107D900009FD2C6070BD401ECAB210F8011F8A4256
:107DA00002D00029F9D10020704710B5431E13F806
:107DB000014F002CFBD105E011F8014B002C03F81A
:107DC000014B03D0521EF7D20021197010BD40EABA
:107DD000010310B59B070FD1042A0DD310C808C9A1
:107DE000121F9C42F8D020BA19BA884201D901204A
:107DF00010BD4FF0FF3010BD1AB1D30703D0521C95
:107E000007E0002010BD10F8013B11F8014B1B1BCF
:107E100007D110F8013B11F8014B1B1B01D1921E39
:107E2000F1D1184610BD40EA0103024630B59B0768
:107E300010D14FF0013400E008C208C91D1B9D435A
:107E400015EAC41FF8D013F0FF0102F8011B0DD092
:107E50001B0AF8E711F8013B002B02F8013B05D0A3
:107E600011F8013B002B02F8013BF3D130BD002299
:107E7000CBB210F8011B994200D1421E0029F8D163
:107E80001046704710B5431C02E010F8011B71B199
:107E90008107FAD14FF0013202C88C1A8C4314EAE0
:107EA000C211F9D0C01A0A0603D0C01E10BDC01AF4
:107EB00010BD0A0401D0801E10BD0902FCD0401E76
:107EC00010BD40EA010370B59B072ED14FF001367B
:107ED000042A2AD308C810C99D1B9D43121F15EA06
:107EE000C61517D0D8B2E1B2401A50EA056110D1D8
:107EF00098B2A1B2401A50EA05410AD123F07F405E
:107F000024F07F41401A50EA052102D1180EA0EB5F
:107F1000146070BDA342DBD018BA21BA884201D9DF
:107F2000012070BD4FF0FF3070BD0AB9002070BD58
:107F300010F8013B11F8014B63B1A3420AD1521E64
:107F400008D010F8013B11F8014B1BB1A34201D13D
:107F5000521EEDD1181B70BD421E12F8013F002BBE
:107F6000FBD111F8013B002B02F8013BF9D170471E
:107F7000032A40F2308010F0030C00F0158011F855
:107F8000013BBCF1020F624498BF11F801CB00F82D
:107F9000013B38BF11F8013BA2F1040298BF00F881
:107FA00001CB38BF00F8013B11F0030300F025803E
:107FB000083AC0F0088051F8043B083A51F804CB65
:107FC000A0E80810F5E7121D5CBF51F8043B40F82B
:107FD000043BAFF30080D20724BF11F8013B11F836
:107FE00001CB48BF11F8012B24BF00F8013B00F87A
:107FF00001CB48BF00F8012B704710B5203AC0F004
:108000000B80B1E81850203AA0E81850B1E8185099
:10801000A0E81850BFF4F5AF5FEA027C24BFB1E8D6
:108020001850A0E8185044BF18C918C0BDE8104047
:108030005FEA827C24BF51F8043B40F8043B08BF50
:108040007047D20728BF31F8023B48BF11F8012B17
:1080500028BF20F8023B48BF00F8012B704702F010
:10806000FF0343EA032242EA024200F002B84FF063
:1080700000020429C0F0128010F0030C00F01B80F5
:10808000CCF1040CBCF1020F18BF00F8012BA8BF03
:1080900020F8022BA1EB0C0100F00DB85FEAC17CC7
:1080A00024BF00F8012B00F8012B48BF00F8012B7A
:1080B00070474FF0000200B51346944696462039AB
:1080C00022BFA0E80C50A0E80C50B1F12001BFF491
:1080D000F7AF090728BFA0E80C5048BF0CC05DF8F7
:1080E00004EB890028BF40F8042B08BF704748BF45
:1080F00020F8022B11F0804F18BF00F8012B7047B9
:1081000010B5044610F0030F08BF11F0030F40F044
:1081100015804FF0013E121FC0F20E8051F8043B53
:10812000A3EB0E0C2CEA030C1CEACE1C08BF40F893
:10813000043BF0D0A1F1040102F10402521E08DB5D
:1081400011F8013B002B00F8013BF7D11146FFF776
:108150008EFF204610BD7047704770477047000083
:1081600010B500F07BFB001D10BD00BF992400007E
:1081700000487047705C002010B5FFF7F9FF0068F9
:1081800010BD10B50446FFF7F3FF046010BD2DE9E4
:10819000F0470D4699469246044600F124080168CE
:1081A000880604D5E06921F01001216000E001207B
:1081B000A84201DD471B00E00027A1697A1902EB04
:1081C0000900081AA0612078C00602D42046FFF7F3
:1081D0007FFB002608E0D4E901211AF80600904749
:1081E000206A401C761C20624E45F4DB2078C006D5
:1081F0000AD52046FFF76CFB06E0D4E901213020C8
:108200009047206A401C2062381EA7F10107F4DC69
:1082100007E0D4E9012118F805009047206A401CC6
:108220002062281EA5F10105F3DC2046FFF766FB5E
:108230002078000602D50220BDE8F0870120FBE788
:1082400070472DE9FF4F0C461E464FF0FF378BB0AD
:10825000D2E90001DDF860800A908A46C1F30A5530
:1082600005B93D46002108464FF00000BAF1000F65
:1082700000F4400005DA00EB80004FF4400101EA11
:1082800050004FEA9059B9F1010F00DDB9460A9844
:1082900050EA4A000ED044F61050A5F2FF3545438F
:1082A0002F14B8F1000F1ED07542291E1EDDC9F132
:1082B00000021CE0B8F1010F4FF0000001D03021A6
:1082C00003E0F24305E02154401CB042FBDB3046A2
:1082D0000022002121540B99C1F80880C1E9002037
:1082E0000FB0BDE8F08FBD1B6D1CDEE74A4600DA1B
:1082F000694206A800F00AFD06AB93E8070003AB4D
:1083000083E8070050460A9900F0F2FD8DE8070067
:10831000A0F500501F3800900398002D0ADD42F2AE
:108320001F014A460844002303A90390684601F050
:108330005BF809E0A0F500504A461F38002303A966
:108340000390684601F065F88DE807000004000C12
:1083500003D04FF0FF30410800E01046B8F1000FA5
:1083600003D00022009215461EE0751E05D400F0D1
:1083700079FA303262556D1EF9D5B34601220843B1
:1083800002D000227F1C04E02078302801D1002296
:108390007F1E002A099784D01DE0112D07DA00F016
:1083A00061FA303262556D1C50EA0102F5D1084382
:1083B00002D00098C8B10EE00021681E05E0235CE1
:1083C000625C63542254401E491C8142F7DBAB4679
:1083D000A81B401E0990002004F80B000B98099A76
:1083E000C0F80880C0E9002B7AE711264FF000089A
:1083F00057E72DE9F04F88460446D21D22F00701C9
:1084000091B0D1E90001CDE90A0101F039F9024644
:108410000B98C00F01D02D2007E02068810701D5FF
:108420002B2002E0202101EAC000032A099001D09C
:10843000072A05DB03464146204600F0D7FB0BE147
:108440002078800601D5E06900E00620B8F1650FCC
:10845000814606D0B8F1660F18D0B8F1670F70D119
:1084600031E00020B9F1110F009001DB112301E090
:1084700009F101030AAA01A90CA8FFF7E2FEDDE950
:108480000C70002609F10105834647E001204B46A8
:1084900000904FF000470AAA01A90CA8FFF7D1FEEF
:1084A000DDE90DB00C995D46002610B909F1010017
:1084B0000D18B9EB050003D4C0F1FF3609F1010531
:1084C000A5EB09002BE0B9F1010F01DA4FF001092A
:1084D0000020B9F1110F0090484601DD112300E0A2
:1084E00003460AAA01A90CA8FFF7ABFEDDE90C7050
:1084F0004D4600268346207800070AD4AB4500DAB3
:108500005D4601A8012D04DD411911F8011C302937
:1085100007D04F4502DA17F1040F04DA0120824632
:108520000FE06D1EEEE7002F02DCED1B3E4403E082
:10853000781CA84200DD7D1CB81B00F1010A4FF039
:1085400000472078000703D4AA4501DB4FF0FF3A2B
:108550000021B7F1004F0DF143088DF8431024D0EE
:1085600002202B23002F01DA7F422D230A21021E35
:10857000A0F1010000DC5FB197FBF1FC97FBF1F289
:1085800001FB1C7C17460CF1300C08F801CDEEE71E
:10859000A8F1010003702188090501D5452100E0FB
:1085A0006521A0F1010800F8011C09980FA9A1EBB1
:1085B0000807FF1D00B10120411901EBEA70A16914
:1085C0003844081A401EA0612078C00602D4204614
:1085D000FFF77EF9099828B1D4E901219047206A74
:1085E000401C20622078C00622D52046FFF770F993
:1085F0001EE0002E04DBB34502DD01A8805D00E033
:108600003020D4E901219047206A401C2062761C6A
:10861000AAF101005FEA000A0AD100F01FF9C06860
:108620000168405CD4E901219047206A401C206227
:10863000281EA5F10105DCDC07E0D4E9012118F8CA
:10864000010B9047206A401C2062381EA7F10107E9
:10865000F3DC2046FFF752F9032011B041E6000099
:1086600001694A1C02610878704700B58FB0CDE9F6
:1086700001310021059105497944CDE903101146E6
:108680006846FFF7B7FA0FB000BD0000E5FFFFFF37
:108690000A6802F8010B0A607047D1E900239A4288
:1086A00002D2531C0B601070704710B5436913B1B0
:1086B000AFF3008001E0FFF744F9012010BD12780C
:1086C00000F124010A7000224A700122EDE71168CE
:1086D0004FF0FF32E9E70000074B70B50D467B44D1
:1086E000FFF7C3FF0446284600F082FB10B14FF0AD
:1086F000FF3070BD204670BD3DA6FFFF10B5436939
:1087000013B1AFF3008001E0FFF794F9012010BD31
:10871000128800F1240182840022C2840122EDE744
:1087200011684FF0FF32E9E72DE9F0418046D21D94
:1087300022F007020025D2E90002F52915A614D07F
:10874000011E72F1000106DA0023D0EB030063EB97
:10875000020211A608E0D8F800108B0701D50FA679
:1087600002E0490701D50EA601251146002408F1B3
:10877000240704E000F076F830323A55641C50EAE1
:108780000102F7D12B46324621464046BDE8F04172
:10879000FFF7FDBC000000002D0000002B000000D2
:1087A000200000002DE9F04791460F468046044620
:1087B000002614F8015B2DB1FFF7D2FC0068405D84
:1087C000C007F6D12B2D02D02D2D18D0641E4A469D
:1087D0003946204600F04AFA27B13968A14201D152
:1087E000C7F800804FF0020471050BD54042002805
:1087F00003DDFFF7BDFC0460A007BDE8F08746F489
:108800008066E4E70028F8DAFFF7B2FC04606FF056
:108810000040F2E770B516460C460546FFF7A0FC8F
:10882000036893F80101012806D0FF2C0FD8185DCA
:1088300068B101202C7070BDD3F807013246214683
:1088400003F2071303442846BDE8704018474FF071
:10885000FF3070BD00487047705C002000487047D2
:10886000905C002030B5B0F10A024FEA900E71F131
:1088700000034EEA817EB0EB0E0061EB91014FEAFE
:10888000101E4EEA017E10EB0E0041EB11114FEA73
:10889000102E4EEA016E10EB0E0041EB11214FEA53
:1088A000104E4EEA014E10EB0E0041EB1141401804
:1088B00041F100014FEAD00040EA41704FEAD10196
:1088C00010EB80054FEA810444EA907444EB010404
:1088D0006D1944EB0404521BA3414FF0000348BF41
:1088E0000A3200D530BD401C41F1000130BD00000E
:1088F0002DE9F04F04460D46D21D22F0070089B045
:10890000D0E900974846394600F0BAFE0246F80F13
:1089100001D02D2307E02068810701D52B2302E039
:10892000202101EAC0038DF820300BB1012000E0C6
:108930000020032A824601D0072A04DB294620466C
:1089400000F054F93FE12078800601D40D2500E0C5
:10895000E569C7F30A560D2D49DA00214FEA175B86
:1089600008464FF00000002F00F4400007DA00EB4B
:1089700080004FF4400100EBD07001EA60008115E7
:10898000012901DD4FF0FF3100224FEA850CBCF1D7
:10899000180F06D31346ACF118004FF08052C240B6
:1089A00003E04FF4801323FA0CF30CF10C0CBCF130
:1089B000200F04D3ACF1200C09FA0CF001E007FA07
:1089C0000CF000294FF0004801DD18B90FE00ED17E
:1089D00040450CD319EB02095F4121B9404502D152
:1089E0009F4329EA0209BBEB175F00D0761C208861
:1089F000000502D57B48784402E07A48784419386B
:108A000008AA302302F80A30037C0AF10101002E83
:108A10000AF1020A53546A4602DC4FF0300101E0C9
:108A20004FF031014FF001088DF8001002D0A6F28E
:108A3000FF3603E059EA470100D06B4E002D02DCFF
:108A40002178090704D54FF002082E218DF8011076
:108A5000C44600210BE0C7F303433F01C35C491C3C
:108A60006D1E02F80830052908F1010801DA002D11
:108A7000F1DC00210CE000EB1973491C1B786D1E22
:108A8000082902F808304FEA091908F1010801DA4B
:108A9000002DF0DC21688B0602D516E0A8F1010854
:108AA000E04505DD02EB080313F8013C302BF5D05F
:108AB000B8F1000F09DD02EB080313F8013C2E2B7F
:108AC00003D1090701D4A8F10108002D05DD3E21DD
:108AD00002F808106D1E08F10108407C002E02F813
:108AE000080008F1010804DA2D20764202F8080097
:108AF00002E02B2002F808000A214FF47A70864227
:108B000008F101080BDB96FBF0F3303302F8083074
:108B100096FBF0F308F1010800FB136601E0642EF8
:108B20000CDB642096FBF0F3303302F8083096FB40
:108B3000F0F308F1010800FB136601E00A2E06DBE2
:108B400096FBF1F0303002F8080008F1010896FBBE
:108B5000F1F001FB1060303002F80800A16908F163
:108B6000010808EB050202EB0A00081AA061207850
:108B7000C00602D42046FEF7ABFE216A08AE01EB28
:108B80000A00206204E0D4E9012116F8010B9047A5
:108B9000BAF1010AF7D22078C00602D52046FEF7C6
:108BA00097FE6E4609E016F8010B3E280FD0D4E977
:108BB00001219047206A401C2062B8F10108F2D2DE
:108BC0002046FEF79BFE09B00320BDE8F08F206A27
:108BD0002844206203E0D4E90121302090476D1E33
:108BE000EBD3F8E7193F000002FCFFFF2DE9F0414D
:108BF0001F46044603260168072A01F4006004DBCF
:108C000008B116A505E016A503E008B115A500E01A
:108C100015A521F010002060A069C01EA0610FB151
:108C2000401EA0612046FEF753FE4FB1D4E901215A
:108C300038469047206A401C2062C01C206206E033
:108C4000206AFAE7D4E9012115F8010B9047761E56
:108C5000F8D22046FEF752FEBDE8F0814E414E00AC
:108C60006E616E00494E4600696E66002DE9F05F48
:108C7000824615468B4600270AF10104B946007862
:108C8000302801D09DB113E014F8010B012778289A
:108C900003D0582801D045B10AE00DB1102D07D1FD
:108CA000002714F8010B102502E0082500E00A2532
:108CB0000026B0460EE005FB080005FB06F1012783
:108CC0001FFA80F801EB1046B6F5803F00D3B94695
:108CD00014F8010B294600F0B4F80028EBDABBF1D8
:108CE000000F05D00FB1641E00E05446CBF80040E1
:108CF000B9F1000F06D0FFF73BFA02210160C81E50
:108D0000BDE8F09F48EA0640FAE700002DE9F04789
:108D1000814616468AB0354878440DC88DE80D0066
:108D200032487844801C03AC0DC884E80D0041F63D
:108D30009B300844372190FBF1F290FBF1F5A5F14F
:108D4000800501FB12041B3C02D56442012000E0B7
:108D50000020DFF898A080460027FA44AAF1BE0A56
:108D60000EE0E0070AD03246684607EB47010123D0
:108D70000AEB810100F04DFB8DE8070064107F1CB9
:108D8000002CEED1194F7F44AE3F19E0E80715D013
:108D900007EB04100DF1180A90E80E008AE80E00A7
:108DA000C068F04201D1981908903246012306A903
:108DB00003A800F02EFB03AB83E807006D10641CD2
:108DC000002DE3D14FF0010332466946B8F1000FA0
:108DD00003A802D000F008FB01E000F01AFBC9E98B
:108DE0000001C9F808200AB0BDE8F087883C0000FF
:108DF000007B00F0800070477546FFF72BFDAE4604
:108E000005006946534620F00700854618B020B596
:108E1000F3F760FABDE820404FF000064FF000077E
:108E20004FF000084FF0000B21F00701AC46ACE812
:108E3000C009ACE8C009ACE8C009ACE8C0098D467F
:108E400070473A2800D2303820F02002412A01D35E
:108E5000A2F13700884201D34FF0FF30704710B5C0
:108E60000446AFF300802046BDE81040F3F71DBA7A
:108E70004FF0013C50F8042B51F8043B9A4221D1A9
:108E8000A2EB0C03934313EACC1317D150F8042B35
:108E900051F8043B9A4215D1A2EB0C03934313EA19
:108EA000CC130BD150F8042B51F8043B9A4209D152
:108EB000A2EB0C03934313EACC13DBD04FF000007A
:108EC000704700BFD01A01BAB1FA81F101F0180160
:108ED00022FA01F0CB40C1F12001DBB2C0B2C01ACE
:108EE0002CFA01F3D11A914311EAC311E6D170476C
:108EF0005FEA400C08BF91F0000F4FEA8C234FEA65
:108F0000C12243EA51514FEA1C5018BF00F5F0400E
:108F10004FEA300018BF41F000415FEA6C5C00F09E
:108F20002980BCF1FF3F08BF40F080407047130C20
:108F300006BF12044FF0100C4FF0000C130E04BFCC
:108F400012020CF1080C130F04BF12010CF1040CF7
:108F5000930F04BF92000CF1020CD30F04BF520018
:108F60000CF1010C11464FF00002A0F11F00A0EB24
:108F70000C00704711F0004F08BF704731F00041FE
:108F80003FF4D5AF0B0C06BF09044FF0100C4FF0A7
:108F9000000C0B0E04BF09020CF1080C0B0F04BFF0
:108FA00009010CF1040C8B0F04BF89000CF1020CB9
:108FB000CB0F04BF49000CF1010CCCF12003A0EB56
:108FC0000C0022FA03F302FA0CF241EA030100F169
:108FD0000100704720F07F4C80EA030023F07F47B8
:108FE000ACEB070303F57C5300F0004003F1FF03F3
:108FF0002DE980494FEA154B09B44FEA144325EA9D
:109000000B4E24EA03480FF2042606EB1327490807
:109010003E785FEA320203FB0667C7F5000707FBED
:1090200006F64FEA54374FEAD64606F1020607FB2A
:10903000066CCCF1005C4FEA1C472CEA074C07FB9E
:1090400006F40CFB06F504EB15464FEA961634BF02
:1090500000204FF000404FEAD13706FB07FC4FEAF3
:109060001C4C0CFB0BF7D21B03FB0CF761EB07014D
:109070000CFB0EF7B0EB074072EB17420CFB08F746
:1090800034BFA2EB0742B2EB074261EB17414FEA54
:109090000C444FEA910706FB07FC4FEA1C4C0CFB03
:1090A0000BF7B0EBC74072EB573203FB0CF734BF42
:1090B000A2EBC742B2EBC74261EB57310CFB0EF794
:1090C000B0EBC70072EB57720CFB08F734BFA2EB92
:1090D000C702B2EBC70261EB5771039F4FEA816190
:1090E00041EA921104EBCC044FEAD1374FEA826295
:1090F00006FB07FC42EA90124FEA80604FEA1C4CE4
:109100000CFB0BF7D21B03FB0CF761EB07010CFB0D
:109110000EF7B0EB074072EB17420CFB08F734BFB9
:10912000A2EB0742B2EB074261EB17414FEA8C55C5
:109130004FEA910704EB9C2406FB07FC4FEA1C4C0A
:109140000CFB0BF7B0EBC74072EB573203FB0CF78D
:1091500034BFA2EBC742B2EBC74261EB57310CFB05
:109160000EF7B0EBC70072EB57720CFB08F734BF79
:10917000A2EBC702B2EBC70261EB577115EB4C25AE
:109180004FEA816141EA92114FEA82624FEAD13798
:1091900042EA901206FB07FC44F100044FEA8060AB
:1091A0004FEA1C4C0CFB0BF7D21B03FB0CF761EBDB
:1091B00007010CFB0EF7B0EB074072EB17420CFBFC
:1091C00008F734BFA2EB0742B2EB074261EB17414D
:1091D00015EB1C154FEA813141EA92414FEA823288
:1091E00042EA90424FEA80304FEA0C7644F10004A4
:1091F00048EA03434EEA0B484FF0000EB2EB080C6E
:1092000071EB030724BF624639464EEB0E0E4FF05A
:10921000000B0018524149414BEB0B0BB2EB080C11
:1092200071EB03077BF1000B24BF624639464EEB1E
:109230000E0E4FF0000B0018524149414BEB0B0B47
:10924000B2EB080C71EB03077BF1000B24BF624605
:1092500039464EEB0E0E51EA020718BF46F00106E2
:1092600016EB0E7655F1000254F1000103D5BDE86E
:109270008901BDE80088BDE88901BDE80048B6194C
:10928000524141EB0101A3F10103704780807F7ED1
:109290007D7C7B7A7978777676757473727171706C
:1092A0006F6E6E6D6C6C6B6A6A696868676666651E
:1092B0006464636362616160605F5F5E5E5D5D5CAC
:1092C0005C5B5B5A5A59595858575756565555551D
:1092D0005454535352525251515050504F4F4F4E7D
:1092E0004E4D4D4D4C4C4C4B4B4B4A4A4A494949CB
:1092F000484848474747474646464545454444440D
:10930000444343434342424242414141002B9C4635
:1093100030D477002BD01CB54FEA370703B44FF099
:1093200010004FF01001BAF1000F06D0BCF1000F91
:10933000DCBF40F0080040F008014FF000000FBC17
:10934000BDE810400BF1010BBBF1010F08BF5FEA54
:10935000170722BF12F1010211F101014FF0004184
:1093600043F1000300F0004043EA00007047F9D3E6
:109370005708D0E746EA064613F1400F4FEA164673
:109380001FDD13F1200FDFBF16430A4600212033F3
:109390005B42BED0C3F1200746EA064602FA07F751
:1093A0004FEA164646EA0706C3F1200722FA03F2FF
:1093B00001FA07F721FA03F14FF0000342EA07022E
:1093C000A7E746EA020646EA06464FEA164646EA96
:1093D0000106BCBF46EA0646360C4FF000034FF0CC
:1093E00000024FF0000194E72DE9804C9A46934625
:1093F00070B491E8380007C831EA400C48BF34EA3D
:10940000430C03D5FFF7E6FDFFF780FFF0BCBDE896
:10941000008C2DE9804C9A46934670B491E8380050
:1094200007C810F0804F08BF13F0804F03D100F041
:1094300005F8FFF76BFFF0BCBDE8008C20F07F471C
:1094400080EA030023F07F4C07EB0C03A3F57C5369
:1094500000F00040A3F1FE0392F0000F00F0B38093
:1094600095F0000F00F077802DE901494FEA114097
:109470004FEA144621EA004800FB06FC24EA0647AE
:1094800008FB06F607FB08F800FB07F718EB064891
:109490004CEB164C4FEA124B18EB07484FEA1546B7
:1094A0004CEB174022EA0B4E0BFB06FC25EA064765
:1094B0000EFB06F607FB0EFE0BFB07F71EEB064E38
:1094C0004CEB164C4FF000061EEB074E4CEB174BC7
:1094D00018EB0B0840F1000018EB0E0B58EB0008DE
:1094E00040F100008F1A4FF000013CBFC943661BDA
:1094F00014BFB5EB040C00213CBFC943F61B4FEA77
:1095000017444EEA8E0E27EA04454FEA1C4704FB37
:1095100007622CEA074C05FB07F70CFB05F604FB7A
:109520000CFC16EB074642EB174216EB0C4642EBDF
:109530001C421BEB060658EB0202414146EA9E061E
:1095400001D5BDE80189B619524141EB0101A3F1F2
:109550000103BDE801894FEA14454FEA114724EAA7
:10956000054621EA074C05FB07F406FB07F70CFB51
:1095700006F105FB0CFC11EB074144EB17444FEAE5
:10958000124711EB0C4144EB1C4422EA074C05FB4B
:1095900007F206FB07F70CFB06F605FB0CFC16EBC7
:1095A000074642EB174216EB0C4642EB1C456A1885
:1095B00054F1000148BF7047B619524141EB010117
:1095C000A3F10103704795F0000F37D04FEA114225
:1095D0004FEA144721EA024624EA074C02FB07F14E
:1095E00006FB07F70CFB06F402FB0CFC14EB07442C
:1095F00041EB17414FEA154714EB0C4441EB1C417A
:1096000025EA074C02FB07F506FB07F70CFB06F6FD
:1096100002FB0CFC16EB074645EB174516EB0C4618
:1096200045EB1C42121951F1000148BF7047B619B1
:10963000524141EB0101A3F1010370474FEA144588
:109640004FEA114724EA054621EA074C05FB07F1DA
:1096500006FB07F70CFB06F24FF0000605FB0CFCBF
:1096600012EB074241EB174112EB0C4251EB1C414C
:1096700048BF7047921841EB0101A3F10103704705
:10968000490050EAC12018BF04204A0D18BF40F01D
:10969000010040F2FF72B2EB515F08BF40F00200E0
:1096A000012808BF052070472DE9F0414F1E00EB4F
:1096B000C7010446D1E9000115461E4637F00602EF
:1096C0000DD02A46334601F0DDFA7F1E04EBC703B6
:1096D000D3E9002300F0C2FF37F00602F1D1022FD8
:1096E00025D0042F13D0062F18BFBDE8F0812A46DD
:1096F000334601F0C7FAD4E90A2300F0AFFF2A4647
:10970000334601F0BFFAD4E9082300F0A7FF2A4648
:10971000334601F0B7FAD4E9062300F09FFF2A464A
:10972000334601F0AFFAD4E9042300F097FF2A464C
:10973000334601F0A7FAD4E9022300F08FFF2A464E
:10974000334601F09FFAD4E90023BDE8F04100F070
:1097500085BF0000002213461046014901F03AB8C7
:109760000000F03F012201F058BE00F077BF002258
:1097700013461046114601F02DB840F20132002088
:109780004FF0E04101F049BE024A0020110701F00C
:1097900044BE000001FDFFFF30380A2801D201203D
:1097A00070470020704700002DE9F041C1F30A52D4
:1097B000A2F2FF362F4A304B0D460446142E2FDA04
:1097C000002E12DA00F04AFF0022134601F058FB87
:1097D0004CD2002DA4BF0024254647DA25F00040D6
:1097E000204318BF254D41D018E0DFF894C02CFA73
:1097F00006F705EA070C5CEA040C08BFBDE8F08137
:1098000000F02CFF0022134601F03AFB2ED2002D6F
:1098100003DA4FF48010F0400544BD43002425E0F6
:10982000332EC8BFBDE8F081A6F1140C4FF0FF370E
:1098300027FA0CF73C4208BFBDE8F08101F056FB67
:109840000022134601F01CFB10D2002D0DDA142E5D
:1098500008BF6D1C09D0C6F13400012101FA00F0E7
:109860002044A04238BF6D1C0446BC432946204614
:10987000BDE8F0819C7500883CE4377E0000F0BFB5
:10988000FFFF0F002DE9F04DC84A002490B091422F
:1098900005DA21F00043934201D805D120B110B080
:1098A000BDE8F04DFFF75EBFB1F5801F1BDA53EA4C
:1098B000000209D0002911DA0120FEF762FC10B085
:1098C000BDE8F04DFFF753BF0220FEF75AFCFFF74B
:1098D00041FF10B081F00041BDE8F08D6FF035041C
:1098E000362201F09AFD04EB2152C1F31308B0496E
:1098F000A2F2FF33414401F4801282F07F6103EB56
:10990000225281F04051009241EA08010022A94B05
:1099100001F0DEFB044608F10200A74EC0F313007D
:109920000D467E44032867D2D6E90023204601F085
:10993000A9F81ED10098002802BFD6E9000110B096
:10994000BDE8F08D01F037F907460C469B4A9C4B69
:1099500001F098F906460D469A4A9B4B3846214637
:1099600001F090F910B032462B46BDE8F04D00F002
:1099700075BE4FF05532954B2046294601F082F9CD
:109980000022934B01F0B2FA06460F4622462B46C0
:109990001046194601F076F932463B4601F072F95D
:1099A000064600980F46F0B101F005F980468A4658
:1099B000824A834B01F066F932463B4601F096FA43
:1099C00022462B4601F084FB05460C467D4A7E4B21
:1099D0004046514601F056F910B02A462346BDE8EC
:1099E000F04D01F075BB0B4610B0324620462946BB
:1099F000BDE8F04D01F06CBB00224FF080432046E3
:109A000000F02CFE02460B462046294600F0E2FEFE
:109A100006460F46009801F0CEF8CDE90401324623
:109A20003B461046394601F02DF90C9069480C9AD6
:109A30004044019009910B46104601F023F98246FB
:109A4000024665488B46C8F151080B4608F5D728F1
:109A500003217844FFF728FE52465B4601F012F9D5
:109A60000A905E480D9152465B4604217844FFF708
:109A70001BFE099B0C9A01F005F9844601980D9B89
:109A800040EA080860460A9A00F0E8FD834608911B
:109A9000B8F1000F4EDD4FF0FF322046294601F0AD
:109AA000BCFC22462B4601F0EDF8804600988A4621
:109AB00060B3DDE90401414A414B01F0E3F809914B
:109AC00000905A4640465146089B00F0C7FD32467A
:109AD0003B4601F0D7F8099B009A00F0BFFD4246D3
:109AE000534601F003FA22462B4601F0F1FA0446F0
:109AF0000D46DDE90401334A334B01F0C3F810B0E1
:109B000022462B46BDE8F04D01F0E2BA5A464046E7
:109B1000089B00F0A3FD32463B4601F0B3F84246F5
:109B2000534601F0E3F910B022462B46BDE8F04D54
:109B300001F0DCB9009840B3DDE904011F4A204B75
:109B400001F0A0F880468A465A4620462946089BDE
:109B500001F0BEFA32463B4601F094F842465346C5
:109B600001F0B6FA22462B4601F0B2FA04460D4641
:109B7000DDE90401134A144B01F084F810B02246C9
:109B80002B46BDE8F04D01F0A3BA0B465A462046DD
:109B9000294601F09DFA32463B4601F073F810B0B9
:109BA00022462B46BDE8F04D01F0A0B90000F07F41
:109BB000645F09000000F03FD22F0000763C793549
:109BC000EF39EA3D0000E0FE422EE63F5555D53F15
:109BD0000000E03F86EBF9FFE22D0000E02D0000E1
:109BE0002DE9F04D1D460C4698B0174621F0004176
:109BF00023F00043002814BF4FF0010C4FF0000C7D
:109C00000CEB440CFE4A0CEB02064FEA620C664574
:109C10002BD33E0018BF012606EB45061644F94A31
:109C2000964222D3F84A53EA070C02D0944205D157
:109C300048B918B000201146BDE8F08D002808BFD3
:109C40004FF0000C01D04FF0010C0CEB440212F568
:109C5000001F0AD8002F14BF4FF0010C4FF0000C6A
:109C60000CEB450212F5001F07D918B03A462B46F7
:109C70002146BDE8F04DFFF778BD0022DFF88CA348
:109C8000002CB8BF534526DADFF884C36345A8BF6C
:109C9000022220DADFF870C39C451CDCDFF874C3B5
:109CA0000CEB235CBCF1140F08DDCCF1340627FA71
:109CB00006FC0CFA06F6BE420DD108E05FB9CCF105
:109CC000140623FA06FC0CFA06F69E4203D10CF0A9
:109CD0000102C2F1020251EA000C19D1002D17DA7B
:109CE000002C18BF022A01D0012A07D00220FEF75B
:109CF00048FA18B0BDE8F04DFFF72CBD0220FEF782
:109D000040FAFFF727FD18B081F00041BDE8F08D63
:109D1000B7F1000C6CD1534525D104F1804212F506
:109D2000801201BF00280020B74918B008BFBDE865
:109D3000F08DB548884207DC002DA1BF604629465A
:109D400018B0BDE8F08D07E0281E05DA80F000416C
:109D500018B06046BDE8F08DAF497944D1E9000103
:109D600018B0BDE8F08DDFF8A0C2634525D1002D05
:109D70001FDA19B1514512D1D8B909E0002840F0D5
:109D8000EC82A24A214618B062F31E01BDE8F08DB4
:109D90000020214618B060F31E01BDE8F08D08DAFE
:109DA00018B02346BDE8F04D02460020614600F0A1
:109DB00011BD18B02146BDE8F08D514518DAB5F156
:109DC000804F0DD0A5F1005CBCF1FF5C10D1B4F167
:109DD000000C0DDB18B06146BDE8F04D00F0ECBBA7
:109DE000234618B00246BDE8F04D194600F04ABFC0
:109DF000060024F0004C3BD1D9B1514533D1002CA1
:109E000006DD002DA1BF0020514618B0BDE8F08D41
:109E1000002C01DD002D1BDB002C13DA002D11DBE3
:109E2000012A4FF0000014BF78497C4918B0BDE802
:109E3000F08D022A18BF002C0AD0012A08D1002C6C
:109E400006DA0AE0002CB8BF002D11DA012A04D08E
:109E5000002018B00146BDE8F08D18B000204FF08A
:109E60000041BDE8F08DA1F14050B0F17F601AD003
:109E7000012000EBE47050EA020421D0624C521E33
:109E80004FF0000B104304BF4FF0000B644C6548CB
:109E900083427CDD644A654893421FDD884217DBBC
:109EA000002D25DB37E0002C00DA4AB1022A0CBF76
:109EB00001204FF0FF3018B0BDE8F04D00F07BBE40
:109EC0000120FEF75EF918B0BDE8F04DFFF74FBC7A
:109ED0004D4A8A4202DC002D0ADC1CE0814202DA93
:109EE000002D18DA04E0484B994220DD002D12DDE8
:109EF0000220FEF746F9FFF740FC05460E46002219
:109F000053465846214600F0BDFE18B066F31E01C8
:109F10002846BDE8F08D0220FEF733F9FFF734FC48
:109F20000A46214618B062F31E01BDE8F08D0022FA
:109F30003046614601F0CCF880460E466FF00102D3
:109F400001F06BFA4FF05532394B00F0CFFF42462B
:109F5000334600F097FE0022364B00F0C7FF8246E2
:109F60004246334604911046194600F08BFE524695
:109F7000049B00F087FE8A4600904FF0C0422E4BB3
:109F80004046314600F07EFE2C4A2B4B00E027E095
:109F9000CDE906015146009800F074FE8246019119
:109FA000274A284B4046314600F06CFE5246019B42
:109FB00001F08EF882460B4602460591DDE9060166
:109FC00000F04CFBDDE9062300268846304601F010
:109FD0007FF85246059B00F089FF024600F07EB9EB
:109FE0000020B1F5801F07DA35223046614601F0C6
:109FF00014FA06466FF0340000EB215024E0000014
:10A00000FFFF1F00FFFF0F000000F03F0000F07F88
:10A010000000404301FCFFFF9A2B00000000F0FF0E
:10A020000000F0BF0000E0410000F043FFFFEF3F01
:10A030005555D53F0000E03F4715F73FFE822B65A1
:10A0400044DF5DF80BAE543EA0F2FF300190C1F347
:10A05000130040F07F6141F040510291FE49884277
:10A06000D8BF002004DDFD498142C8BF012001DDC9
:10A070000D9008E000200D900198401C019002987E
:10A08000A0F5801002900299F54878440B910D9943
:10A0900000EBC100D0E900230F9330460A920B99E0
:10A0A00001F016F8CDE90601DDE90A2130460F9BE3
:10A0B00000F0D4FA02460B460020EA4900F08AFB81
:10A0C000059102460B460090DDE9060100F0DAFD3D
:10A0D0001490E5488A464FF00008784402990068D9
:10A0E00012904FF0005040EA61010D980F9B01EB78
:10A0F000804000F5002109910A9A129800F0E8FFCB
:10A1000032460B9B00F0F2FE4246534600F0BAFD89
:10A110000646029140465146099B129A00F0B2FD54
:10A12000DDE9062300F0E2FE3246029B00F0D0FF9C
:10A13000059B009A00F0A6FD0091149A04905346E6
:10A140001046194600F09EFD06460246C7480B46DB
:10A15000029106217844FFF7A7FACDE90510029B8A
:10A1600032461046194600F08DFDDDE9053200F05B
:10A1700089FD05910646534640461946149A00F05B
:10A180006DFA009B049A00F07DFD3246059B00F0BD
:10A1900065FACDE90510424653461046194600F0CF
:10A1A00071FD0022B24B02910A9000F057FADDE9EE
:10A1B000053200F053FA0E464246AD4B404600F0E1
:10A1C00087FF029B0A9A00F083FFDDE9053200F069
:10A1D0008DFE424602910A9033461046514600F0E9
:10A1E00051FDCDE906015346149A02990A9800F0F0
:10A1F00049FD8A460290334642460099049800F091
:10A2000041FD5346029A00F029FA82460B46024667
:10A210000591DDE9060100F021FADDE906230020C1
:10A220008846064600F054FF5246059B00F05EFE4D
:10A23000824609914FF060428E4B3046414600F015
:10A2400021FD049006918C4A8A4B5046099900F0F2
:10A2500019FD82460291894A894B3046414600F0F9
:10A2600011FD5246029B00F0F9F9864B7B440D9A92
:10A2700003EBC203D3E9002300F0F0F90E9007913D
:10A28000019800F098FC0591DDE9061382460E9ACC
:10A29000049800F0E3F97C4A7A440D9B02EBC30377
:10A2A000D3E900230093029200F0D8F95246059BAF
:10A2B00000F0D4F90026884652463046059B00F04F
:10A2C00007FF009B029A00F003FF069B049A00F030
:10A2D000FFFE079B0E9A00F009FE024600200B4687
:10A2E00002903846294600F0CDFC824601912B466B
:10A2F00038461946029A00F0EBFE3246434600F01B
:10A30000C1FC5246019B00F0A9F907468A46324635
:10A3100043462946029800F0B5FC05460E463A46EB
:10A32000534600F09BF9594A8846914221DBA8EB3D
:10A33000020353EA000210D12A46334600F0C8FE59
:10A34000CDE90401524A534B3846514600F086F994
:10A35000DDE9042300F094FD21D20220FDF711FF76
:10A36000FFF70BFA0A46214618B062F31E01BDE85A
:10A37000F08D494B28F000429A4210D3474A08EB2F
:10A38000020353EA00027FF4C6AD2A46334600F0CA
:10A390009FFE3A46534600F073FD7FF6BCAD0022A7
:10A3A000019228F000403E493E4A01EB2051824292
:10A3B00023DA481C4FF4801121FA00F040443A4A55
:10A3C000C0F30A517A44394BA1F2FF31CB4020EA65
:10A3D0000303C0F3130040F48010C1F11401C8401E
:10A3E00012680190B8F1000FBCBF404201902846AE
:10A3F000314600F06DFE05460E462A463346384685
:10A40000514600F02BF94FF000084246284B4046D9
:10A41000059100F037FCCDE90601264A264B40465F
:10A42000059900F02FFC009102902A4633464046E1
:10A43000059900F04DFE3A46534600F057FD1F4A7D
:10A440001F4B00F01FFC009B029A00F007F9074623
:10A45000884602460B4635E08E9803007AB60B001C
:10A46000E22700000000F03F1A2800004827000003
:10A470000000084009C7EE3FFD033ADCF5015B141C
:10A48000E02F3EBE20260000E425000000009040A2
:10A49000FE822B654715973C00CC904000346F3FFF
:10A4A00001FCFFFF0000E03F30250000FFFF0F0030
:10A4B000432EE63F396CA80C615C20BEEF39FAFEF2
:10A4C000422EE63FDDE9060100F0C8F8DDE906238B
:10A4D00005460E4600F0FCFD3A46434600F006FDF8
:10A4E0000F462A46334600901046194600F0CAFB34
:10A4F000824602462E4888460B4605217844FFF7DF
:10A50000D3F85246434600F0BDFB2A46334600F0DE
:10A51000EDFC80468A463B4628463146009A00F0CC
:10A52000B1FB3B46009A00F099F80691009000229A
:10A530004FF080434046514600F0CAFD0F460C9054
:10A54000424653462846314600F09CFB3B460C9A57
:10A5500000F040F9069B009A00F0BAFD2A46334607
:10A5600000F0B6FD0022134B00F0C0FC0546019838
:10A570000E4601EB00510815002810DC2846314634
:10A58000019A00F04AFFFFF77BF8042808BFFFF7A5
:10A59000FBF828463146019A00F03FFF05460B467E
:10A5A00018B02A4658462146BDE8F04D00F06ABB77
:10A5B000D02300000000F03F2DE9F04106460F4691
:10A5C00000F0A0FC041E0D4618BF0120284320F017
:10A5D0000040C0F17F6000F1E040C00F0ED0301CA1
:10A5E00018BF0120384320F00040C0F17F6000F127
:10A5F000E040C00F04BF0120FDF7C3FD20462946FF
:10A60000BDE8F08110B500290AD00878002807D0ED
:10A6100005487844FEF72CFC002801D0002010BD2E
:10A620000248784410BD0000CA280000C22800007B
:10A6300010B500290AD00878002807D005487844CA
:10A64000FEF716FC002801D0002010BD0248784417
:10A6500010BD0000AE290000A629000010B591EA47
:10A66000030F48BF83F0004300F13A85841A71EB71
:10A67000030C05D2121943EB0C03001B61EB0C0118
:10A68000DFF824E14FEA1154A4EB135C1EEA430FF8
:10A6900018BF9EEA445F73D023EA0E03DCF1200E5C
:10A6A00021EA045143F4801332D322FA0CFE10EB5A
:10A6B0000E0023FA0CFE41EB0E01CCF1200E03FA42
:10A6C0000EFE10EB0E0051F10001B1F5801FCCF130
:10A6D000200E32D201EB045112FA0EF2BDE8104006
:10A6E00058BF7047401C38BF5FEA420218BF70472E
:10A6F000002814BF20F0010041F100014FEA41039E
:10A7000013F5001F38BF7047A1F1C04100F0B2BB84
:10A71000012A43EB0302ACF1200CDCF11F0E32BF27
:10A720004FF0000E23FA0CF310EB030041EB045141
:10A73000B4EB115FD0D0A1EB045101F580114908B1
:10A740005FEA300001EB04510ED350F1000038BF36
:10A7500012FA0EFE08D1BDE81040C9E7401C38BF10
:10A760005FEA4202CAD1C3E7BDE810404FEA4103A5
:10A7700013F5001F38BF7047A1F1C04100F07ABB4C
:10A780009EEA445F08D011EA5E0FBDE8104004BFA6
:10A7900001F0004100207047BDE8104070B500F0A6
:10A7A0001BFB00BF64FBBE3E0000E0FF02494FF010
:10A7B000000000F000BE00BF0000F87F491058BF45
:10A7C000C1F140415B1058BFC3F140438B42EFF3EE
:10A7D000008070472DE9C04130B4DFF8A0C23CEAE8
:10A7E000111418BF3CEA131400F0EC8081EA030551
:10A7F0001CEA111444EAD57418BF1CEA131500F0C2
:10A80000C780A4EB05044FF0004545EAC12145EAA5
:10A81000C32341EA505143EA525304F17F749942F1
:10A8200004F500344FEAC0204FEAC22208BF90422C
:10A8300000F09C804FEA13650FF24016765D4FEAF8
:10A84000134506FB05F7C7F1807706FB07F74FEACC
:10A85000D737A7FB03687642C8F58038A7FB06CE3A
:10A8600038BFA8F1010807FB08E64FF0000EA6FB71
:10A87000028CE6FB03CEDCF1000CCEF1004E38BFBB
:10A88000AEF1010EA6FB0C584FF000074FF000058B
:10A89000E6FB0E87A1FB08C6A0FB07CE16EB0E0653
:10A8A00045F10005E1FB076515F1E04E7EBFA4F51B
:10A8B00080345FEA46066D4116F1800745F10005D8
:10A8C0004FEA17274FEA066647EA0567A6F1DE4614
:10A8D000B6F1805F4FEA15251FD9384624F0010CE8
:10A8E00005EBC471BCF1FE6F01EB0C1102D8F0BC9A
:10A8F000BDE8008124425CBF01F5801E9EEAC47F52
:10A9000002D4F0BCBDE80081244238D4F0BCA1F1EF
:10A91000C041BDE8004100F0ADBA4FEAD22242EAA0
:10A9200043524FEAD323A7FB02864FEAD02040EAE6
:10A93000415007FB03661EEA0E0F4FEAD12105FBCB
:10A94000026658BFA6EB0056B6EB00564FEA520E11
:10A950004EEAC37E18EB0E0E56EB530EBDD518EB28
:10A9600002085E417F1C55F10005B6E74FF48015E3
:10A970004FF000074FF000064FF00008ADE7F0BCC5
:10A980004FF0000001F1C04101F00041BDE800813D
:10A9900011EA0C1F0CEA131500D00CE013EA0C1F8F
:10A9A00000F025804FF00000F0BC81EA030101F0C7
:10A9B0000041BDE80081F0BCBDE8004181EA03012F
:10A9C00000F058BAF0BCBDE8004170B500F004FAE0
:10A9D000097EFC3E00F007B881EA03014FF0000059
:10A9E00001F00041704781EA030100F043BAF0BC76
:10A9F000BDE800414FF0000021497047FFFDFBF921
:10AA0000F7F5F4F2F0EEEDEBE9E8E6E4E3E1E0DEA1
:10AA1000DDDBDAD8D7D5D4D3D1D0CFCDCCCBCAC813
:10AA2000C7C6C5C4C2C1C0BFBEBDBCBBBAB9B8B73A
:10AA3000B6B5B4B3B2B1B0AFAEADACABAAA9A8A82D
:10AA4000A7A6A5A4A3A3A2A1A09F9F9E9D9C9C9BFB
:10AA50009A999998979796959594939392919190A6
:10AA60008F8F8E8E8D8C8C8B8B8A89898888878737
:10AA70008685858484838382828181800000FF07AC
:10AA80000000F87F51EA030C17D41CF5801F58BF53
:10AA9000BCF5801F00F10680994218BF704708BFBF
:10AAA0009042704707D711F5801F58BF13F5801FDC
:10AAB00019D499427047894270471CF5801F08D508
:10AAC000BCF5801FF7D58B4218BF704708BF824284
:10AAD00070474FF4001C1CEB410F38BF1CEB430FB9
:10AAE00001D28B42704770B500F076F9922449008C
:10AAF0004FF000514FF08053FFF760BE4FEA410323
:10AB00004FEA5353A3F58063D3F11E03C8BFD3F1BB
:10AB1000210C0CDD4FF0004242EAC12242EA5052C1
:10AB200032FA03FC8CEAE17CACEBE1707047102B4D
:10AB3000C4BF0020704703F5787CBCF1FF3F04D010
:10AB40006FF0004282EA2100704770B500F044F9CE
:10AB50004992248000207047F2E700004FEA115329
:10AB6000A3F58063D3F11E03A8BFD3F1200C08DB4B
:10AB70004FF0004242EAC12252EA505232FA03F048
:10AB8000704709420BD4102BC4BF0020704703F557
:10AB9000787CBCF1FF3F05D04FF0FF3070474FF09D
:10ABA0000000704770B500F017F900BF499224808B
:10ABB00000207047F0E710F0004248BF4042B0FA72
:10ABC00080F310FA03F10AD0C3F11D0303F580638B
:10ABD0004FEA415002EB035202EBD12170474FF094
:10ABE00000007047B0FA80F310FA03F10AD0C3F105
:10ABF0001D0303F580634FEA41504FEA035202EB15
:10AC0000D12170474FF000007047000051EA030C5B
:10AC100017D41CF5801F58BFBCF5801F00F10680BB
:10AC2000994218BF704708BF9042704707D711F587
:10AC3000801F58BF13F5801F19D49942704789426D
:10AC400070471CF5801F08D5BCF5801FF7D58B42D7
:10AC500018BF704708BF824270474FF4001C1CEBBE
:10AC6000410F38BF1CEB430F01D28B42704770B5C8
:10AC700000F0B2F8922449004FF000514FF0805399
:10AC8000FFF79CBDDFF848C170B51CEA111E1EBF5E
:10AC90001CEA13159EEA0C0F95EA0C0F00F06F806A
:10ACA00081EA030423EA4C134EEAD47E21EA4C11D4
:10ACB00041F4801143F48013AE44A1FB024CA0FB8D
:10ACC0000365AEF17F7E361955EB0C05A1FB034CF5
:10ACD0004CF10003A0FB021C16EB0C06654153F17E
:10ACE0000003094218BF46F0010613F4007F0BD1A0
:10ACF0004FEA03314FEA0530340341EA155140EA87
:10AD000016506FF003020AE04FEAC3214FEAC52054
:10AD1000F40241EA555140EA56506FF0020202EB4C
:10AD20002E4201EB025585EACE710AD05FEA440C4F
:10AD300018BF24F0004450F1000041F1000120EA66
:10AD4000D47040F2FE7C624500D270BDA84214BFB0
:10AD50004FF080444FF04044002E08BF0024BEF165
:10AD6000806FA8BFA1F1C041BDE8704080F2828031
:10AD70004FF0000001F1C04101F0004170479EEA30
:10AD80000C0F0CEA131518BF95EA0C0F06D04FF004
:10AD9000000081EA030E0EF0004170BD00F01CF8C7
:10ADA0008900013E00F007B800F009B84FEA430CF3
:10ADB0005FEA5C5C08D081EA030100F05BB84FEA0F
:10ADC000410C5FEA5C5CF6D14FF00000014970472E
:10ADD0000000FF070000F87F0EF1020E2EF0030EB8
:10ADE0005EF8046B364205D4012A43EB030515F5E2
:10ADF000001F12D8012841EB010C1CF5001F0CD8D4
:10AE00000ED14FEAD17C15F5001F0CEB4C0C0CF168
:10AE1000020C08BF4CEBD37C04E04FF0080C01E0BF
:10AE20004FEAD37C0CEB4C0526FA05F606F0070634
:10AE3000B6F1040C06D20EEB860CBDE870404CF067
:10AE4000010C6047DFE80CF0090B02024FF00041F3
:10AE50004FF00000A1F5002170BD194610460128F1
:10AE600051EB010418BFD4F5001484BF002001F099
:10AE7000004170BD0808A0F500114FEA310170478C
:10AE800053EA010C17D41CF5801F58BFBCF5801F76
:10AE900000F106808B4218BF704708BF824270479E
:10AEA00007D713F5801F58BF11F5801F19D48B42A7
:10AEB00070479B4270471CF5801F08D5BCF5801F6A
:10AEC000F7D5994218BF704708BF904270474FF4BA
:10AED000001C1CEB430F38BF1CEB410F01D2994201
:10AEE00070470FB40CBC03BCFFF7C1BE91EA030F5F
:10AEF00010B581F000413FF5B9AB83F0004300F09D
:10AF0000EFB800002DE9F04101F5801CBCF5001FF1
:10AF1000C0F2C3804FEA115C21EA0C510CF1FD0C28
:10AF200041F480115FEA5C0C0CF5C07C01D3400059
:10AF300049413DA4890241EA905187028E0E0A0CD4
:10AF4000A45D04FB04F602FB06F6C6F14046A4FB32
:10AF50000662F60D46EA422606FB06F4A4FB012330
:10AF60005242C3F1404338BF5B1EA6FB024200249D
:10AF7000E6FB0324D20B42EA4446A6FB0623A1FBD0
:10AF800002E2A3FB07E4A4184FF0000252F1000212
:10AF9000E3FB01426442C2F1404E38BFAEF1010E04
:10AFA000A6FB04234FF00002E6FB0E32A2FB034691
:10AFB0004FF00004B61954F10004E2FB0264A1FB57
:10AFC00006E6A4FB07E816EB08064FF0000858F168
:10AFD0000008E4FB01687642C8F1405838BFA8F188
:10AFE0000108A2FB06E4A3FB08E52D194FF00004BD
:10AFF00054F10004E2FB0854A1FB05E6A7FB04E8BA
:10B0000018EB06084FF0000656F10006E1FB048637
:10B0100018F1200556F10006A809A8F11B08B1098E
:10B0200008F03F08B8F10A0F40EA86601CD901EB2E
:10B030000C51BDE8F08100BFFCF5EEE8E2DDD8D3AD
:10B04000CFCBC7C3C0BDB9B6B4B1AEACA9A7A5A399
:10B05000A19F9D9B9A9896959392908F8D8C8B89AA
:10B060008887868584838281A0FB006800FB01F2CB
:10B0700008EB4208B8EB872807D5341858EB0104D1
:10B08000D5D5401C51F10001D1E7341A78EB010409
:10B09000CDD4401E71F10001C9E75FEA4C0C5FEAB4
:10B0A0009C5C0DD105D34FF0000001F00041BDE8DC
:10B0B000F081BDE8F04170B5FFF78EFE6DDBFFBE9D
:10B0C000BDE8F0414FF00000004970470000F87FF4
:10B0D00010B591EA030F48BF83F000433FF5C6AABD
:10B0E000841A71EB030C07D212198CF0004C43EB5D
:10B0F0000C03001B61EB0C01DFF8A4E14FEA1154D3
:10B10000A4EB135C1EEA430F18BF9EEA445F00F0F5
:10B11000B08023EA6E03524221EA0451C3EB6E036E
:10B1200038BF5B1EDCF1200E25D322FA0CFE10EB9B
:10B130000E0043FA0CFE41EB0E01CCF1200E03FA97
:10B140000EFE10EB0E0051F10001CCF1200E29D4BF
:10B1500012FA0EF201EB0451BDE8104058BF7047DF
:10B16000401C1CBFB2F1004F704700280CBF491CA7
:10B1700020F00100704712EB020E43EB030218BFF0
:10B180004FF0010E4EEA4202ACF1200CDCF11E0E33
:10B1900054D943FA0CFE10EB0E0051F1FF31CCF103
:10B1A0001E0ED5D50EF1010E12FA0EFE404141EBF6
:10B1B000010101EB445C5FEA5C5C10D910EBDE70CE
:10B1C00001EB045138BFBEF1004FBDE8104018BF7D
:10B1D000704700280CBF491C20F00100704730D296
:10B1E0004FEAD42C11F5001124F400641BD0B1FAFD
:10B1F00081F20B3AA41AA41ED2F12003914030FA36
:10B2000003F31943904001EBCC71002C01EB045186
:10B21000BDE81040A8BF704701F1C0414FF00000E9
:10B2200001F000417047B0FA80F310FA03F100D149
:10B2300010BDE41A173C4805C90AE4E701EB0451C4
:10B2400010BD491001EB0451BDE810404FEA300039
:10B2500002E04FF0000170474A0008BF0042F8D0FA
:10B26000B2F5001F28BF704701F000414FF0000009
:10B2700070479EEA445F07D011EA5E0FBDE81040B8
:10B2800004BF002100207047BDE8104070B5FFF7F3
:10B29000A3FD00BF40DFF63E83F00041104670473B
:10B2A0000000E0FF43004FEAD30C4FEA3C0C434060
:10B2B0001FBF40070CF1605113F0FE4F70471CF0A8
:10B2C000006F03D100200CF0004170470CF00043E8
:10B2D00043EA507010B540EACC0000F022F800BFFD
:10B2E000000000924FEA0001FFF7C4BD4FF000419B
:10B2F0004FF00000A1F5002170470000B0FA80F384
:10B3000010FA03F2C3F19D030AD0D90501EB122014
:10B31000530638BF704700F1010008BF20F001005C
:10B3200070470EF1020E2EF0030E5EF8044B24421D
:10B3300004D44FEA4102B2F17F4F11D84FEA4003E3
:10B34000B3F17F4F0CD80ED14FEAD07CB2F17F4FD2
:10B350000CEB4C0C0CF1020C08BF4CEBD17C04E064
:10B360004FF0080C01E04FEAD17C0CEB4C0324FABF
:10B3700003F404F00704B4F1040C06D20EEB840CC1
:10B38000BDE810404CF0010C6047DFE80CF0070806
:10B3900002024FF00040A0F5800010BD08464200B8
:10B3A00018BFD2F1807288BF00F0004010BDFDF7D9
:10B3B00020B8FDF79DBA0CF00F03092B08BF082039
:10B3C00000F059800A2B0BD0082B18BF704708BF1C
:10B3D0001CF0400F0AD04FF000004FF00001704702
:10B3E0001CF0400F18BF4FF0004070471CF0100FCA
:10B3F00008D020F0704300F07F4242EAD3014FEAC8
:10B400004370704700F0604021F07F4242EA000242
:10B4100001F07F4040EA727070474FF0FF0C4CF42F
:10B42000E06C1CEA11531CBF9CEA030C9445C2BF9C
:10B43000DA4201EB02517047002B0DD0BCF1000F36
:10B440000FD0002A01F00041A4BF41F0E04141F0DB
:10B450007F614FF00000704701F000414FF00000A5
:10B46000704750EA01334FF09B0C18BF4CF0806CD2
:10B470007FF49CA970471CF4801F11D01CF4E02FAE
:10B4800003D06FEACC31490070474FF04050EFF3E2
:10B49000008222F0704242EA000282F30088704784
:10B4A0004FF0000070470103070F1FFFFF1F0F073A
:10B4B00003010000000000E0E00000FCFC000000D0
:10B4C00000000000000000000000003F3F000038C6
:10B4D0003800003F3F00003F3F00003F3F000000BA
:10B4E0000000000000000000F808E8E8E8E80808AC
:10B4F000E8E8E8E80808E8E8E8E80808F820E000F4
:10B5000000000000000000001F1017171717101090
:10B510001717171710101717171710101F04070009
:10B520000000000000000000C0E0F0F8FCC05F5523
:10B5300055D5755555555FC0000809090B0505051A
:10B540000B09090000EACC0011F200FC2424E41FDE
:10B55000E485660000070A0700020B0403040E00DE
:10B56000B3CF0012D2FE5190122400FF8080000160
:10B57000000F00000101010F000000BFC600888815
:10B58000FF4824E4243F24E4040000080F000808D6
:10B59000050205080800BCBC000000000000000017
:10B5A000000000000000000000000036360000002F
:10B5B000000000000000000000A3BA00000000002E
:10B5C00000000000000000000000000000005838EB
:10B5D000000000000000000000000000A3AC00001C
:10B5E000000000000000000000000000000000005B
:10B5F000001824241800000000000000000000A132
:10B60000A300000000FE0000000000000000000099
:10B6100000000000003300000000000000000000F7
:10B620000000A3A100000038340282C27C38000070
:10B63000000000000000000000003737000000009C
:10B640000000000000A3BF00008080BEAAAAAAEAF2
:10B65000AAAAAABE80800000048584945C54272492
:10B6600024544C4484050400EACC004042CC000041
:10B67000F888888808FF0809CA080000003F906819
:10B680001F10209F4027182641F000B3CF0024242C
:10B69000A4FEA3220022CC0000FF00000000080648
:10B6A00001FF00010404040404FF02020200BFC6FB
:10B6B00000101010FF109008888888FF888888087C
:10B6C000000444827F01808040432C102846818002
:10B6D00000BCBC001010FF109000FE5252D252521B
:10B6E000525E000042827F8140308F929392FE92A0
:10B6F00093968000CED50000002424242424FC222C
:10B7000022222322000000020202020242827F0261
:10B7100002020202020200CAD6000000F01010105D
:10B7200010FF10101010F000000000000F040404BF
:10B7300004FF040404040F000000D6D00000000041
:10B74000000001E21CE0000000000000008040203A
:10B75000100C03000000030C3040808000C8EB0098
:10B7600000FE0222428272022242827202FE000027
:10B7700000FF100806010E100806014E807F000031
:10B78000CDF800404042CC000444645C47F444449B
:10B790004404000040201F2044444444447F444467
:10B7A000444400C1AC00101010FF1050445465C652
:10B7B0004464544440000444827F0182824A5623F8
:10B7C00022524E820200BDD3000000FE222222FE41
:10B7D00000FE828292A29E000080601F0242827F51
:10B7E00000FF402F102C438000B7FE00000090881F
:10B7F0004C57A42454548C84000000000101804262
:10B80000221A07024282423E01010100CEF100806D
:10B81000809E9292929EE0809EB2D2929E8000087C
:10B8200008F4949292F10001F2929494F80800C600
:10B83000F7001060028C0008080809FA08080808D8
:10B84000000004047E0140404141417F41414141AB
:10B850004000D7A200808080FE8282FE8080FE822F
:10B8600082FE8080000080403F00407F80601F405B
:10B87000807F000000B2E1000000F8888888880816
:10B8800008FF08090AC8080080601F0010201F80F8
:10B89000402116182641F800B3C900080808F80826
:10B8A00008081010FF101010F000001030101F08D2
:10B8B0008848300E014080403F0000B9A60000409B
:10B8C000301E101010FF10101010100000008181A9
:10B8D0004121110D0301030D112141818100CAA7EE
:10B8E0000000FE02FA02FE4020D8171010F01010DF
:10B8F000008047300F1067804021160816214080D5
:10B9000000B0DC00080889EA1888000404FC04047C
:10B9100004FC0000020100FF01864020180740805F
:10B92000403F0000B3F5001010F01F10F00040E0A1
:10B930005847405060C0004022150816210000FE04
:10B9400042424242FE0000CABC00008060F807008C
:10B950000000FF40201008040000010000FF000468
:10B9600002013F40404040407800BBAF0004044427
:10B97000C44F4444C424242FB42404040040442469
:10B9800024150C04FE040C152424444000B2CB0002
:10B990000000F8494A4C48F8484C4A49F800000071
:10B9A00010101312121212FF1212121213101000A2
:10B9B000B5A500404042CC0000FC24A4242222A3D0
:10B9C0006200000040201F2058475048454245482B
:10B9D000504000B7B5000000FE0202F2121212F24F
:10B9E0000202FE00000000007F20202724242427DC
:10B9F00020207F000000BBD800000022322AA6A22F
:10BA0000622111098101000000004222130B4282D1
:10BA10007E02020A1223460000CFB5002030AC633C
:10BA2000300088C8A8998E88A8C88800226722128A
:10BA3000128040300F00003F40407100CDB30080C5
:10BA400080848484FE82838280FF808080800000E6
:10BA5000804020180700000000FF0000000000C91F
:10BA6000FD002030AC6330000202FE0202625AC6C2
:10BA70000000226722121240308F80432C102C438A
:10BA80008000BCB60008C8B88FE8888840300FC86E
:10BA9000082818000008180808FF048440300E0128
:10BAA0000E30408000C8ED00008060F80780601C08
:10BAB0001010FF1010100000010000FF0002020231
:10BAC0000202FF0202020200BCFE00004042445893
:10BAD00040407F40405048C600000000404444447D
:10BAE00044444444444444FF000000B5B100080805
:10BAF000E8292E28E80808C80C0BE8080800000010
:10BB0000FF0949897F00000F40807F000000C7B017
:10BB10000000FE20203F2000FC24E4242223E20039
:10BB200000807F0101FF80601F8041261826418030
:10BB300000B0E6000010101010D030FF30D0101010
:10BB40001010000010080402090808FF0808090284
:10BB500004081000B1BE00808080BEA2A2A2A2A2F2
:10BB6000A2A2BE80808000000000060504040444F8
:10BB700084443C00000000BAC500404042CC004074
:10BB8000A09E8282829EA02020000000003F90881C
:10BB900040432C10284641808000C9E800809090E6
:10BBA000484C57242424544C4480808000000000DA
:10BBB000FF4949497F494949FF00000000B1B800E9
:10BBC000008060F80700042424252624242404008F
:10BBD000010000FF000000F94949494949F9000006
:10BBE000D0C500000000FC54545655545454FC0079
:10BBF0000000004030000339414145594141730084
:10BC0000083000CFA2000000007F49494949494956
:10BC1000497F000000008141211D214181FF898968
:10BC2000898989818100CAC700000282824222126A
:10BC3000FA0622224242820000010100FC444444F0
:10BC400045444444FC00000100B7F100001010908E
:10BC500010101116101010D010100000404040407D
:10BC6000435C4040504C434040404000C1A2000073
:10BC7000FE92929292FE0000FE020202FE0000007E
:10BC80003F20100A04180000FF000408070000BC51
:10BC9000B400003E22E2223E0010885724548C005B
:10BCA0000000407E403F22220001FE424242FE014F
:10BCB0000100C2B700001088C43380824222121AE9
:10BCC0002622408000020100FF00404242427E42A4
:10BCD0004242424000BEB6000484E45C44C400F228
:10BCE0009292FE9292F2020002017F10103F808F2A
:10BCF00054245F4484878000D3B20000FE02FA021D
:10BD0000FE0080FF80A090888680008047300F1062
:10BD1000670000FF40230C10204000D5CB0080803E
:10BD200080BEA2A2A2A2A2A2A2BE80808000000029
:10BD30000006050404044484443C00000000BAC525
:10BD400000108C4404E40495A64424148444940C08
:10BD50000002027A414143427E42424243F80000DF
:10BD600000C3DC000484E45C44C40002F2828282EA
:10BD7000FE80800002017F10103F0008080808487C
:10BD800088403F00C2EB00C808090EE808405E503A
:10BD900050DF50505E4000206F201C131000FE0248
:10BDA0007F027E82FE0000B6CB000000FC0404048B
:10BDB000040404040404FC00000000007F20202090
:10BDC0002020202020207F000000BFDA00404424F3
:10BDD000A4948C84FF848C94A4244440004040406C
:10BDE0005F4A4A4A4A4A4A4A5F40404000B2E90034
:10BDF000404042CC0020D04C4B48C80808F8000016
:10BE00000000007F20101F1212125F80403F0000D0
:10BE1000D1AF00404042CC00202222A26222222246
:10BE20002000000040201F20444E45444444454625
:10BE30004C4000D4CB00001088C433004042424242
:10BE4000C24242424000020100FF00000000408068
:10BE50007F0000000000D0D000808080BEA2A2A29F
:10BE6000A2A2A2A2BE8080800000000006050404F9
:10BE7000044484443C00000000BAC50000000000F7
:10BE800000000000002F0000000007000700001461
:10BE90007F147F1400242A7F2A120062640813236F
:10BEA00000364955225000000503000000001C2206
:10BEB0004100000041221C000014083E0814000844
:10BEC000083E0808000000A06000000808080808F4
:10BED000000060600000002010080402003E51498C
:10BEE000453E0000427F400000426151494600212A
:10BEF00041454B31001814127F1000274545453944
:10BF0000003C4A494930000171090503003649499E
:10BF1000493600064949291E000036360000000057
:10BF200056360000000814224100001414141414A2
:10BF3000000041221408000201510906003249594B
:10BF4000513E007C1211127C007F49494936003E67
:10BF500041414122007F4141221C007F4949494122
:10BF6000007F09090901003E4149497A007F08081C
:10BF7000087F0000417F4100002040413F01007FD9
:10BF800008142241007F40404040007F020C027FA5
:10BF9000007F0408107F003E4141413E007F0909B7
:10BFA0000906003E4151215E007F091929460046DD
:10BFB000494949310001017F0101003F4040403FB4
:10BFC000001F2040201F003F4038403F00631408FE
:10BFD00014630007087008070061514945430000D9
:10BFE0007F41410000552A552A55000041417F00FC
:10BFF00000040201020400404040404000000102F1
:10C000000400002054545478007F484444380038D9
:10C010004444442000384444487F00385454541861
:10C0200000087E0901020018A4A4A47C007F080473
:10C0300004780000447D4000004080847D00007F43
:10C04000102844000000417F4000007C0418047860
:10C05000007C0804047800384444443800FC24245C
:10C0600024180018242418FC007C08040408004844
:10C070005454542000043F444020003C4040207C65
:10C08000001C2040201C003C4030403C0044281054
:10C090002844001CA0A0A07C004464544C44141408
:10C0A0001414141400000000000000000000000040
:10C0B00000000000000000F8000000000000003355
:10C0C0003000000000100C06100C060000000000FC
:10C0D0000000000040C07840C0784000043F0404E5
:10C0E0003F040400007088FC08300000001820FFA6
:10C0F000211E0000F008F000E018000000211C03E1
:10C100001E211E0000F00888700000001E2123245C
:10C110001927211010160E0000000000000000007A
:10C1200000000000000000E018040200000000070A
:10C130001820400000020418E00000000040201811
:10C1400007000000404080F0804040000202010FE4
:10C1500001020200000000F0000000000101011FC8
:10C1600001010100000000000000000080B070002C
:10C1700000000000000000000000000000010101BC
:10C18000010101010000000000000000003030004B
:10C190000000000000000000806018040060180625
:10C1A0000100000000E010080810E000000F10205F
:10C1B00020100F00001010F8000000000020203FA9
:10C1C0002020000000700808088870000030282433
:10C1D00022213000003008888848300000182020D4
:10C1E00020110E000000C02010F8000000070424F9
:10C1F000243F240000F8088888080800001921203E
:10C2000020110E0000E0108888180000000F112097
:10C2100020110E0000380808C83808000000003F50
:10C22000000000000070880808887000001C2221AF
:10C2300021221C0000E010080810E000000031225C
:10C2400022110F00000000C0C000000000000030FC
:10C25000300000000000008000000000000080604E
:10C2600000000000000080402010080000010204CF
:10C2700008102000404040404040400004040404B6
:10C280000404040000081020408000000020100872
:10C2900004020100007048080808F00000000030A7
:10C2A00036010000C030C828E810E0000718272435
:10C2B00023140B000000C038E0000000203C2302E3
:10C2C0000227382008F8888888700000203F202046
:10C2D00020110E00C0300808080838000718202078
:10C2E0002010080008F808080810E000203F20206F
:10C2F00020100F0008F88888E8081000203F202050
:10C300002320180008F88888E8081000203F200043
:10C3100003000000C030080808380000071820207B
:10C32000221E020008F808000008F808203F21013A
:10C3300001213F20000808F8080800000020203FE5
:10C340002020000000000808F8080800C080808055
:10C350007F00000008F888C028180800203F20014E
:10C360002638200008F8080000000000203F2020A8
:10C370002020300008F8F800F8F80800203F003FBF
:10C38000003F200008F830C00008F808203F2000D7
:10C3900007183F00E01008080810E0000F102020E8
:10C3A00020100F0008F808080808F000203F2101BD
:10C3B00001010000E01008080810E0000F18242414
:10C3C00038504F0008F8888888887000203F200087
:10C3D000030C30200070880808083800003820213D
:10C3E00021221C00180808F8080818000000203F47
:10C3F0002000000008F808000008F808001F2020AE
:10C4000020201F000878880000C83808000007387E
:10C410000E010000F80800F80008F800033C0700CF
:10C42000073C0300081868808068180820302C0337
:10C43000032C30200838C800C83808000000203F0E
:10C440002000000010080808C838080020382621FD
:10C4500020201800000000FE020202000000007F01
:10C4600040404000000C30C000000000000000010F
:10C470000638C00000020202FE00000000404040FA
:10C480007F0000000000040202020400000000001F
:10C49000000000000000000000000000808080809C
:10C4A0008080808000020204000000000000000084
:10C4B000000000000000808080800000001924221D
:10C4C00022223F2008F8008080000000003F112059
:10C4D00020110E000000008080800000000E11205E
:10C4E00020201100000000808088F800000E11203C
:10C4F00020103F200000808080800000001F22224A
:10C5000022221300008080F0888888180020203FB5
:10C51000202000000000808080808000006B9494C8
:10C520009493600008F8008080800000203F210084
:10C5300000203F2000809898000000000020203F4D
:10C5400020200000000000809898000000C080803B
:10C55000807F000008F8000080808000203F2402D7
:10C560002D302000000808F8000000000020203FC7
:10C57000202000008080808080808000203F20007C
:10C580003F20003F8080008080800000203F21000D
:10C5900000203F200000808080800000001F2020BD
:10C5A00020201F00808000808000000080FFA120EC
:10C5B00020110E000000008080808000000E1120FD
:10C5C00020A0FF80808080008080800020203F218C
:10C5D000200001000000808080808000003324243F
:10C5E00024241900008080E0808000000000001FEB
:10C5F000202000008080000000808000001F20209C
:10C6000020103F20808080000080808000010E305C
:10C610000806010080800080008080800F300C03BD
:10C620000C300F0000808000808080000020312EC0
:10C630000E312000808080000080808080818E709C
:10C640001806010000808080808080000021302C4E
:10C650002221300000000000807C02020000000067
:10C66000003F404000000000FF000000000000000C
:10C67000FF0000000002027C800000000040403FFC
:10C680000000000000060101020204040000000096
:10C690000000000060010000010000002000000018
:10C6A00020000000002C0000200000000306010B09
:10C6B0000405020925262734350000010001000188
:10C6C0000001000000400000000002000000040023
:10C6D0000000080000001000A4550020A45600200F
:10C6E000A4570020A45800200B0000000C000000FC
:10C6F0000D0000000E0000000F0000001000000000
:10C700001100000038000000390000003A0000006D
:10C710003B0000003B00000000010203040506008E
:10C7200004000000080000001000000020000000CD
:10C730004000000080000000000100000100020035
:10C7400004000800100020004000800000010002EA
:10C7500000040008001000200040008000010203D7
:10C760000405060708090A0B0C0D0E0F0100000056
:10C77000020000000400000008000000100000009B
:10C7800020000000400000008000000000010000C8
:10C79000000200000004000000080000001000007B
:10C7A000002000000040000000800000060708098B
:10C7B0000A17171717172828282828280003030600
:10C7C00001040602050003051F1C1F1E1F1E1F1F5C
:10C7D0001E1F1E1F1C1D1E323637000001000000E8
:10C7E000020000000400000008000000100000002B
:10C7F0002000000000000000000000003031323353
:10C800003435363738394142434445464030580084
:10C8100030313233343536373839616263646566B6
:10C820004030780004000008000000000000000212
:10C83000000100001000000004FA97999999D93F6F
:10C84000AF788E1DC571CC3F9FC678D0099AC33F83
:10C85000935555555555E53F599322942449D23F58
:10C86000DE03CB966446C73F44523EDF12F1C23F1F
:10C87000000000000000F03F000000000000F83F52
:10C8800000000000000000000000004003B8E23F8C
:10C89000000000000000000006D0CF43EBFD4C3E3E
:10C8A000033333333333E33FFFAB6FDBB66DDB3F33
:10C8B0004D268F515555D53F01411DA96074D13F7B
:10C8C00065DBC9934A86CD3FEF4E454A287ECA3F75
:10C8D0003E5555555555C53F93BDBE166CC166BFF7
:10C8E0002CDE25AF6A56113FF16BD2C541BDBBBEF0
:10C8F000D0A4BE726937663E000000000000000050
:10C9000030313233343536373839616263646566C5
:10C91000787000303132333435363738394142435C
:10C92000444546585000000002400000000000A0AE
:10C930000000000005400000000000C800000000EA
:10C940000C4000000000409C000000001940000066
:10C950000020BCBE0000000034400000BFC91B8E98
:10C9600000000004B5400000504BCFD06607E2CF76
:10C97000010000006C4100003E8251AADFEEA734A6
:10C9800001000000D9420000DCB5A0E23A301F9758
:10C99000FFFFFFFFB4450000FD25A0C8E9A3C14F7C
:10C9A000FFFFFFFFFF3F00000000008000000000CD
:10C9B000FF3F000000000080000000000D0A2A2A4E
:10C9C0002A2A2A2A2A2A2A2A2A2A2A2A2A2A2A2AC7
:10C9D0002A2A2A2A2A2A2A2A2A2A2A2A2A2A2A2AB7
:10C9E0002A2A2A2A2A2A2A2A2A2A2A2A2A2A2A2AA7
:10C9F0002A2A2A2A2A2A2A2A2A2A2A2A000000003F
:10CA00000D0AB0E6C8A8B9E9CAF4203A20EACCB3C6
:10CA1000CFBFC6BCBC20323031372F382D32303238
:10CA2000372F38202E0909090909090D0ABCBCCA8B
:10CA3000F5D6A7B3D6203A204D722E2057616E67E7
:10CA400020203133363335353133363138202E001E
:10CA50002A4745542A20496170466C61673A5B2534
:10CA6000635D21202052756E4170704E756D3A5B8A
:10CA700041505025635D2120204A756D70526573C9
:10CA8000756C743A5B25635D212020426F6F74568C
:10CA90006572733A5B25735D212020417070566585
:10CAA00072733A5B25735D2120204373713A5B25D5
:10CAB000735D21202045633230566F6C3A5B2573DD
:10CAC0005D21202053696D49636369643A5B257376
:10CAD0005D212020467470557365726E616D653AF4
:10CAE0005B25735D21202046747050617373776FEE
:10CAF00072643A5B25735D212020467470466F6C2A
:10CB00006465723A5B25735D21202046747049503C
:10CB10003A5B25735D21202054637049503A5B25B0
:10CB2000735D212020546370506F72743A5B2573DB
:10CB30005D210000B2CECAFDB2BBBACFB7A82100BA
:10CB4000C3FCC1EEB8F1CABDB4EDCEF321000000C4
:10CB5000C3FCC1EEB2BBD6A7B3D600007175616E3F
:10CB60002E73756E696E672E636F6D002F67657427
:10CB700053797354696D652E646F0000504F5354A0
:10CB800020687474703A2F2F2573257320485454ED
:10CB9000502F312E310D0A436F6E74656E742D5413
:10CBA0007970653A6170706C69636174696F6E2F3A
:10CBB0006A736F6E3B636861727365743D5554466A
:10CBC0002D380D0A486F73743A25730D0A636F6E22
:10CBD00074656E742D6C656E6774683A25640D0A11
:10CBE0000D0A2573000000007B226D6163223A224A
:10CBF0002573227D00000000415445300D0A0000DD
:10CC000041542B4342430D0A0000000041542B5174
:10CC1000504F57440D0A000041542B474D520D0A06
:10CC20000000000041540D0A000000004154265647
:10CC30000D0A0000415426570D0A0000453A2030E5
:10CC400000000000453A2031000000002B43424321
:10CC5000000000004F4B0000504F57455245442004
:10CC6000444F574E000000004552524F5200000002
:10CC700041542B5149435347503D25642C312C22BC
:10CC80002573222C22222C22222C310D0A00000096
:10CC900041542B435245473D320D0A0041542B432A
:10CCA000475245473D320D0A0000000041542B43D6
:10CCB0005245473F0D0A000041542B434752454718
:10CCC0003F0D0A0041542B51494143543F0D0A0086
:10CCD00041542B51434349440D0A000041542B5108
:10CCE0004E57494E464F0D0A0000000041542B4359
:10CCF00053510D0A0000000041542B514944454155
:10CD000043543D25640D0A0041542B51494143547D
:10CD10003D25640D0A0000002B435245473A0000B0
:10CD20002B43475245473A002B514E57494E464FE9
:10CD30003A0000002B4353513A0000002B51494167
:10CD400043543A002B5143434944000041542B5172
:10CD500049434C4F53453D25642C31300D0A0000AA
:10CD600041542B51494F50454E3D312C25642C22C6
:10CD7000544350222C222573222C25642C25642C0C
:10CD8000310D0A0041542B514953544154453D3112
:10CD90002C25640D0A00000041542B514953454E87
:10CDA000443D25642C25640D0A0000002B51495395
:10CDB000544154453A0000002B51494F50454E3ADA
:10CDC000000000003E00000053454E44204F4B0041
:10CDD0002573000041542B51485454504346473D5D
:10CDE00022636C6F73657761697474696D65222C59
:10CDF0003130300D0A00000041542B51485454503A
:10CE000055524C3D25642C36300D0A0041542B51AF
:10CE1000485454504346473D22636F6E74656E74A8
:10CE200074797065222C310D0A00000041542B5199
:10CE3000485454504346473D22726571756573747A
:10CE4000686561646572222C310D0A0041542B51D2
:10CE5000485454504346473D22636F6E746578745E
:10CE60006964222C320D0A0041542B51485454500D
:10CE7000504F53543D25642C362C360D0A000000CB
:10CE800041542B5148545450524541443D360D0AAB
:10CE9000000000002B5148545450504F53543A2036
:10CEA000302C3230300000002B5148545450524541
:10CEB00041440000434F4E4E4543540008D0020801
:10CEC000000000205C0600006CC1010834D3020899
:10CED0005C06002074860000C8C101081001000033
:10CEE00043000000F8FFFFFF00404040404040404A
:10CEF000404041414141414040404040404040402D
:10CF000040404040404040404005020202020202D0
:10CF1000020202020202020202202020202020201F
:10CF20002020200202020202020290909090909033
:10CF300010101010101010101010101010101010F1
:10CF40001010101002020202020288888888888865
:10CF50000808080808080808080808080808080851
:10CF60000808080802020202400000000000000059
:10CF700000000000000000000000000000000000B1
:10CF800000000000000000000000000000000000A1
:10CF90000000000000000000000000000000000091
:10CFA0000000000000000000000000000000000081
:10CFB0000000000000000000000000000000000071
:10CFC0000000000000000000000000000000000061
:10CFD0000000000000000000000000000000000051
:10CFE0000000000000000000000000001C00000025
:10CFF00043000000F8FFFFFF0C0000000E000000DF
:10D000000F0000002E0000000130320432301E50AC
:10D01000CB020834041A400451320C6201174BDF72
:10D02000010801011F0302010105570C1302011F32
:10D0300001030202098B0C1303011F020403030BFB
:10D04000BF0C1A04241E0104040DF30C180B050177
:10D0500001080605051027E00819381E0705051107
:10D060005B0C180A07010106080505128F0C1955FB
:10D070001F0705080813C30C180A0901020A0A0948
:10D080000914F70C18160A010209090A0A152BE1FE
:10D0900001080B01030C0C0B0B165F0C180A0C019A
:10D0A000030B0B0C0C17930C180A0D01040F0E0D3B
:10D0B0000D18C70C180A0E01040D0F0E0E19FB0CEB
:10D0C00028110F01040E0D0F0F1A2FE20108100195
:10D0D0000510011A630C2D11010611011AB70C2D50
:10D0E00012010712011E07E40108130329011A5D4A
:10D0F0000C2D14010914011AB10C2D15010A15018A
:10D10000280907E5010816010B16011A5D0C2D17F9
:10D11000010C17011AB10C2D18010D18011AD70CAA
:10D120002D19010E1901280923E601081A010F1A09
:10D1300001290C812230500D3132312E34312E37FD
:10D14000392E3837180A581B70177CCB02085C043C
:10D150001A6C041AE804C11F0CCC02088A022819B0
:10D16000081AFF011A68081A041032011A240C3236
:10D170000AAA541C2203191F111A2C0C190B115A3C
:10D180003C1C2A441C193529141AF8642908B9389A
:10D19000193532045A3438E91C32050A15181C4274
:10D1A00006598CDA4C1C411AD00C2940CB44CDA82E
:10D1B00029C40A159054293B5AAC1CAA18381919CD
:10D1C00029140A159C3829C45AB81CDA2038298435
:10D1D0005ADC1CAA281C198929C45AEC1CDA3438D8
:10D1E00032070A15707032081A08301ADC5DB91C53
:10D1F000195432091AF80C1A900CE91C320A5AC454
:10D2000054DA3C70411A60142AC8CCD9A819031109
:10D210001A4C140A11648C293B1A841C29E8DAACD4
:10D220005429681A98142A1478D95432045AD01CF4
:10D23000DAC81C414B4CCE54E970291F0A152C1C2E
:10D24000298C5AD48CE91C298C0A150C38298C1A83
:10D25000F8381A580C1AB424A98C293029A80912B4
:10D260003832061A6830323CE9385A07383250DA18
:10D27000941C32081A80143264DAA81C1E1D2B027A
:10D28000084F0413A0262A205F13A0521A2009E297
:10D2900068280901020209020A0A0C0A17030A0394
:10D2A0000B0B0214380140124412401A48041A4C65
:10D2B0000412501B4004141A04141A04141A0414FF
:10D2C0001EC1330208CB041AD5041ADF0441120828
:10D2D0001C02401C041A30041A44041A58041A6C24
:10D2E000041A800419E51B401C041A30041A440473
:10D2F0001A5804111A08681A0C041A10041A140493
:10D300001A18041A1C041A2004011212401A0404E8
:10D310001A08041A0C041A100412143D40020406E0
:10D320007C19BC2A040415060708098CA24A04DEED
:04D33000591471001B
:040000050801C131FC
:00000001FF
